:10000000004000202D6A00006D6A00006F6A000049
:1000100000000000000000000000000000000000E0
:10002000000000000000000000000000716A0000F5
:100030000000000000000000736A0000756A000004
:10004000776A00003D4D0000A96E0000776A00004D
:10005000776A000000000000776A0000776A0000FD
:10006000776A000079710000C52C0000776A0000F3
:10007000776A0000776A0000776A0000776A0000FC
:10008000776A000011730000776A0000776A000049
:10009000776A0000776A0000776A0000776A0000DC
:1000A000776A0000776A000000000000000000008E
:1000B0000000000000000000000000000000000040
:1000C00010B5064C2378002B07D1054B002B02D02E
:1000D000044800E000BF0123237010BD640200202B
:1000E00000000000E0DB0000044B10B5002B03D043
:1000F0000349044800E000BF10BDC04600000000F6
:1001000068020020E0DB0000164B002B00D1144BEE
:100110009D46402292029A1A924600218B460F4633
:100120001348144A121A0AF09BFE0F4B002B00D002
:1001300098470E4B002B00D0984700200021040068
:100140000D000D48002802D00C4800E000BF0AF066
:1001500047FE2000290006F0C5FE0AF01BFEC0463F
:100160000000080000400020000000000000000027
:10017000640200209C2F002000000000000000000E
:100180000123034010D104280CD90268120909D0B8
:10019000531E9B001A1DC1180979002902D0013392
:1001A0009342F8D1180070470023FBE70378002B37
:1001B00003D05AB2002A01DB013070473F2293433B
:1001C000C03B59424B41C01803789343802BF4D174
:1001D0000130F9E710B500240378002B01D120008D
:1001E00010BDFFF7E3FF0134F6E770B5002204000D
:1001F0000D00411C092003F075F8002806D00123EA
:100200006200134343600023A34200DB70BD9A00E9
:10021000A958821891600133F6E770B5012803DC14
:100220001C2000F0A1FE70BD01230D6811201D42AD
:10023000F7D04868184206D1042804D90F23026871
:100240001340042B01D00E20EBE702F0B5FE6D1039
:100250000400002D03DDFFF7BDFFA84206DA1220DF
:10026000DFE72000FFF7A2FF0400013D012DF8D1D8
:1002700020787F2809DDDF280BDCF8233F22DB0014
:10028000800118406378134018430123400018434D
:10029000C9E7EF280BDCFC22637812019B011340B5
:1002A0003F220007000C0343A0781040ECE7F7283A
:1002B00012DCFC22637892021B031340E0228004CC
:1002C000520310403F221843E3781340FC220343BB
:1002D000A07812018001E8E701204042D5E7F0B59F
:1002E000070085B00D001C20012F06DD4C6801239E
:1002F00022001A40019203D10D2000F035FE54E097
:10030000022F02D08A681A42F6D001232E681E42BC
:1003100000D07EE0042E00D87BE01C41002C00DCE5
:100320001C000F2332681340092B29D173685B101E
:100330000193022F05D0AB68019A5B109A4200DD51
:100340000193019B01221F1B0137FB43DB171F4059
:10035000791C092002F0C6FF061E09D001237F0088
:100360001F4303002A68083347600199A14202DA5B
:10037000300005B0F0BD0134A100515802C3F4E7CC
:10038000042B46D1300002F017FEFFF723FF029046
:10039000022F04D0AB685B10984200DD0293029BF1
:1003A0009C4204DD002003F009F80600E0E730007D
:1003B00002F002FE0700019B9C4222DC3000019704
:1003C00002F0FAFD03903800FFF7F0FE029B0134C3
:1003D0000700A342F7DA019BC71A380002F0EEFFCC
:1003E000061EC5D002F0E8FD0400286802F0E4FD16
:1003F000039A019B991A41183A0020000AF014FD53
:10040000B6E73800FFF7D2FE019B070001330193E6
:10041000D1E7212071E7F8B54D680F00EB0706D44E
:10042000042D04D90F232E683340092B03D00B2051
:1004300000F09AFDF8BD6B6836095C10731EA3428C
:100440000FD80321200008F0C7FB6421642803DCD7
:100450000100032800DA03212800891902F072FF45
:1004600005002B6800201B09013B9C42E2D23A6840
:10047000A31C9B005A510123013464001C436C608F
:10048000D8E7F0B585B0012803DC1C2000F06CFD36
:100490002AE001244D682200022806D08B682342FE
:1004A00003D05C10002C00DC140001231D4200D09E
:1004B00073E0042D00D870E00F272B680E683B40D6
:1004C000042B27D1033B1E4205D1042E03D93368E8
:1004D0001F40042F01D00E20D8E72800FFF750FE60
:1004E000A04203DA0120404205B0F0BD280002F02E
:1004F00063FD0700300002F05FFD013C0100381988
:100500000BF064F80028EDD00123C01B013040003F
:100510001843E9E7092B40D16B685B1000939C42BC
:10052000E0DC01231E4230D1042E2ED933683B403B
:10053000042B2AD1300002F03FFD012302900193E9
:100540000397671CBB00E858864203D101986400FA
:100550002043C9E7019B18420ED104280CD9036837
:10056000039A1340042B07D102F026FD01000298E4
:100570000AF0F6FF0028E9D0009B3C009F42E0DD36
:10058000B0E71C00009B9C42ACDC631C9A00AA589C
:10059000B242F6D164000120DAE7212076E710B5F7
:1005A00002F0EEFC43000120184310BD10B57F2976
:1005B00002DC0170013010BD1A4B99420CDC402363
:1005C0008A115B42134303703F230B408021494251
:1005D000194341700230EEE7134B994210DC20239F
:1005E0000A135B4213433F24802203708B11524253
:1005F0002340214013430A43437082700330DAE7FB
:100600000A4B9942D7DCF0230370603B4370113BE7
:100610008A11FF3B1A4382703F2211401943C17077
:100620000430C8E7FF070000FFFF0000FF0F0100D4
:10063000F0B50D0085B0002803DC1C2000F094FC10
:100640000DE009680122080010400AD002AC1141F7
:100650002000FFF7ABFF011B200002F0BBFE0400EF
:100660001AE004293FD90F230C682340092B3AD103
:100670004B685B10019303239C46019B9A420EDD5D
:1006800002F09CFE041E07D02E68012502F094FCA7
:100690002F00019B9D421DDD200005B0F0BD013201
:1006A0009300CC580123234001D10D20C6E76410EC
:1006B0007F2C0DDD0D4E0223B44209DD0C4E634646
:1006C000B44205DD00270B4EE30FA6427B419B00A1
:1006D000C018D2E70135AB00F1583942E5D04910D6
:1006E000FFF764FFD5E72120A8E7C046FF07000019
:1006F000FFFF0000FF0F010010B5040001200840BB
:1007000010D104290DD90F230A681340042B08D1F6
:10071000080002F051FC010020000AF021FF4342D2
:10072000584110BD0020FCE7F7B50F00012803DC9D
:100730001C2000F019FCFEBD01264D682E4006D19C
:10074000042D04D90F222B681A40092A01D00B204E
:10075000EFE76A681B095410A34200D85C1E396891
:100760001E48FFF7C9FF01230190002813D1396803
:100770001B48FFF7C1FF002811D0002C0DD001232A
:10078000621C013C9C409200535123436B6004E087
:100790000136B200AB50B442FADA0020CBE73B6836
:1007A0000D20DA07C5D55B10002B11DD9C420FDB55
:1007B0009B00A200291DEB1889180433994209D126
:1007C0000123013C9C40AA181C4353606C60E4E781
:1007D0001220AEE758681860EFE7C046EBC400008F
:1007E000EFC40000002310B50C000B70C30705D543
:1007F0000D49421020000AF077FE08E00B4900285E
:1008000002D0042804D10A4920000AF08DFE10BD50
:100810000428FCD90F2302681340042BF7D102F0FF
:10082000CBFB04490200E5E7F0CD0000F4C4000072
:10083000FAC40000FFC40000F0B593B003900300B9
:1008400002911C20012B1DDD029B01251B681C0051
:100850002C4000D0A8E0042B00D8A5E01A680F2394
:100860001A40092A48D10194019A029992008A58A3
:1008700016002E4005D1042A03D910681840092813
:1008800004D0222000F070FB07002CE052685210C8
:10089000A418019A013201920199039A8A42E3D184
:1008A000611C012202F01EFD071E01D100271AE083
:1008B00064002543456005000835029AB300D1580D
:1008C0004B680A685B1012099A4200D8531E002236
:1008D00093420BDCDA43D21713409B00ED18019BC7
:1008E00001369E42E9DB380013B0F0BD90000C18D1
:1008F000A46801322C50EBE7042A55D12F002600C2
:100900001D00029AB300D058384237D1042835D997
:1009100003682B40042BB4D1FFF732FC039B013654
:100920002418B342EDD1200002F048FD071EBDD0CF
:10093000039B029D9B00EB18041D029301232E686C
:100940001E4222D1042E20D90F2233681340042BDB
:100950000DD13000FFF714FC0190300002F02CFBA9
:10096000019A010020000AF05FFA019BE418029B43
:100970000435AB42E2D100232370B4E705A9FFF7A9
:1009800031FF05A80AF0F6FDC8E705A93000FFF71A
:1009900029FF05A80AF0EEFD0600020005A92000C7
:1009A0000AF042FAA419E2E7212000F0DDFA7DE71F
:1009B000F0B50D0095B0002806DC1C2000F0D4FA3C
:1009C0000400200015B0F0BD0C68012123000B408D
:1009D000009306D1042C04D922680F331A40092A47
:1009E00001D00B20EAE7626852100392002A03DC70
:1009F000009802F0E3FCE3E73F4A019201280BD0A4
:100A00006868084208D1042806D902681340042BFC
:100A100002D102F0D1FA019001980AF0ABFD060074
:100A20000F27039B0834013B04935E43039B029012
:100A30009B001B19059301232068184251D10428FB
:100A40004FD903683B40042B52D1FFF799FB059B1C
:100A500004343618A342EED1300002F0AFFC041E7D
:100A6000AFD02B680593029B002B03D0686802F07F
:100A7000A3FA0190200002F09FFA0500009B059A5E
:100A80009B00D3189F68380002F096FA01230600F5
:100A90001F4201D1042F04D807A93800FFF7A2FE96
:100AA00007AE30000AF066FD0700020031002800A2
:100AB0000AF0BAF9029BED19002B0AD0049B009AA8
:100AC000934206DD2800029A01990AF0ADF9029BD3
:100AD000ED18009B01330093009A039B9342CDD104
:100AE0006FE707A9FFF77EFE07A80AF043FDAEE710
:100AF00002F062FAF9E7C0464FC8000010B50024C2
:100B0000A04207DD0B6801341C4003D05C10E343B6
:100B1000DB171C40611C0122092002F0E3FB0028C6
:100B200003D0012364001C43446010BD0B6870B502
:100B300018000125284032D1042B30D90F241A681F
:100B400049681440092C16D15C6812092C41A24254
:100B500000D8541E844205DC02200132904206DB9C
:100B600000200FE085005D19A9600130F2E78400E4
:100B700019510130F2E7032C11D1294203D113207E
:100B800000F0F2F970BD4910FF29F8D812090433BA
:100B900092009A189A42E3D919700133FAE70B20B0
:100BA00000F0E2F9DCE700000123F7B500264D680C
:100BB0000F002B400093B3420DD11E00042D0AD923
:100BC0000F222B681A40092A0FD16A681B09561098
:100BD000B34200D85E1E3968CB0713D54C10002CE9
:100BE00001DDA64219DA12202EE0042A04D12800E1
:100BF000FFF7C6FA0600EEE7009E032AEBD11E09B6
:100C0000B600E8E72E48FFF777FD002814D00AF079
:100C100007FC310008F0C6F84C1C009B002B4CD19F
:100C2000042D4AD92A680F331340092B10D10134FF
:100C3000A40064592000FEBD39682248FFF75CFD1E
:100C400034000028E9D1113000F08EF90400F1E7FA
:100C5000042B2AD1280002F0AFF90600FFF7BAFAF8
:100C6000A042C0DB012C1ADC280002F0A5F900909C
:100C70003000FFF79BFA851B280002F09FFB041E43
:100C8000D8D002F099F90190786802F095F9009BAC
:100C90002A00F11A411801980AF0C6F8CAE7300094
:100CA000FFF784FA013C0600DCE7032B05D12C1981
:100CB000E478023B64001C43BCE70B20C4E7C04659
:100CC000E4C40000EFC40000F7B54C680F00012039
:100CD000210001402AD1042C28D90F222368BE68A4
:100CE0001A40092A13D162681B0955100191AB42C1
:100CF00000D85D1E39682848FFF7FEFC002829D07F
:100D00000F2322681340092B19D1012313E0032A72
:100D10000CD1064203D1132000F026F9FEBD72105B
:100D20000192FF2AF7D81D09AD00E3E70B20F3E796
:100D300001339A00A6509D42FADA0020EEE7032B19
:100D4000FBD1230001331A1BAA42F6DC6A46127952
:100D5000DA70F7E73968CB0706D54910002901DDBD
:100D60008D4209DA1220D7E70C48FFF7C5FC2900AD
:100D7000002801D11130CFE70F2322681340092B3F
:100D800003D1013189000E51D7E7032BD5D16B4632
:100D90001B796418E370D0E7EBC40000EFC40000D7
:100DA00010B501240868204216D1042814D90F2256
:100DB00003681A40092A01D1406810BD032A03D1F3
:100DC0001809C0002043F8E7042A05D102F0F4F81E
:100DD000FFF700FA4000F5E70B2000F0C5F8ECE75C
:100DE00010B5034A0A21034804F0B2F810BDC0460A
:100DF00094C400008CC40000F0B585B0039301904A
:100E000002912C4E2C4B002A02D002223270013A61
:100E100000251A601B68F554019B9D4201DB05B05B
:100E2000F0BD029AAB00D058234B1C68C8239B002E
:100E300037191C1B0123184206D0204A43102100F9
:100E400038000AF01FFB09E01D4A002802D00428E0
:100E50001BD11C4A210038000AF014FB30000AF0B4
:100E600089FB154A039B1060002B0CD0019B013BB2
:100E7000AB4208DD144B984205D8431C1360202276
:100E800032540022F2540135C6E704280FD90F234B
:100E900002681340042B04D102F08EF80B4A0300C1
:100EA000CDE7092B04D14368094A5B10C7E701234A
:100EB000084AC4E7A5020020C8050020F0CD0000C4
:100EC000F4C40000FAC400001F0300000FD40000A7
:100ED00064C7000073C7000010B50124044002D0AD
:100EE0004410200010BD04280CD90F2302681340C1
:100EF000042B07D102F060F821000A220AF002FC5C
:100F00000400EEE70D22014B1A70EAE7A40200206C
:100F10000123020010B51A4015D1042801D9026836
:100F200012090B4011D1042901D90B681B090024B7
:100F3000934206D104309B000431C318984206D373
:100F40000124200010BD0022EBE70023EFE7047826
:100F50000A78002C01D1002AF2D0013001319442EC
:100F6000ECD00024EDE70000014B18700020704722
:100F7000A402002070B501F093FD094C0100251D6D
:100F80001F2228000AF00EFB28000AF0F3FA0423BF
:100F900004308008000118432060200070BDC04666
:100FA00080020020C368F0B59D00836889B05D1998
:100FB0000300183306930369069A9F00069B02906C
:100FC000DF19436901939B00D3180393CD4B1B7822
:100FD000002B26D17F222B68CB491C1213409B008B
:100FE0005B58043501929F46029B587804F08CFBB5
:100FF0000023029A137027E0C24B1B78002B10D1FC
:101000002B68019A1C121340BF4A9B009B58043561
:10101000E9E7069B3A1DD11ABA4BD82928DD1A22D6
:101020001A70029BB74C9B6821780193EA1A029BC5
:1010300092109B7812021A43029B587804F06CFBC2
:101040000023029A23701370029B069A9B680193F7
:10105000ED1A029BAD10DD60069BFE1A029BB610D6
:101060001E61039B9B1A029A9B10536109B0F0BD4D
:101070001B783C60002B01D01700D2E72B68019948
:101080001C120B40A0499B005B5817000435AAE7CF
:10109000069B3A1DD11A9B4BD82902DD1A221A70E1
:1010A000BFE728681B78291D3860002B02D0170085
:1010B0000D00B6E76B6801991C120B4092499B002A
:1010C0005B58170008358EE7069B3A1DD11A8D4BE9
:1010D000D82902DD1A221A70A3E7A4001B782C1964
:1010E0003C60002B01D017009BE72B6801991C1274
:1010F0000B4085499B005B581700043573E7069B3E
:101100003A1DD11A7F4BD82902DD1A221A7088E7BE
:101110007E49A40061581B783960002B01D017006C
:101120007FE72B6801991C120B4077499B005B58A5
:101130001700043557E7043F744B3A68A400E250A7
:10114000704B1B78002B00D06BE72B68019A1C12A8
:1011500013406D4A9B009B58043544E76B4BA40039
:10116000E058FFF7B9FE043F06003868FFF7B4FE09
:1011700036180120654B76000643E650614B1B781C
:10118000002B00D04DE72B68019A1C1213405E4AD9
:101190009B009B58043526E7069B3A1DD11A594BF4
:1011A000D82902DD1A221A703BE70698039C012118
:1011B000A04202D221000C3909681B783960002B4B
:1011C00001D017002DE72B6801991C120B404E49E6
:1011D0009B005B581700043505E7069B3A1DD11AA2
:1011E000484BD82902DD1A221A701AE7069903988B
:1011F00081420FD203000C3B1B6845495B10641809
:10120000E41AA40023583B603E4B1B78002B05D00A
:10121000170006E7182119700023F4E72B680199DD
:101220001C120B4038499B005B5817000435DAE666
:10123000069B039A934219D213000C3B1B68344A55
:10124000043FA4185B10E31A039A39689B00995075
:101250002C4B1B78002B00D0E3E62B68019A1C1264
:101260001340294A9B009B580435BCE61822254BA5
:101270001A70EDE7069B039A93422DD2244B3E1F32
:10128000E31814000C3C04932368049A5B10D31AEF
:10129000039A9B009858FFF71FFE07903068FFF7EE
:1012A0001BFE2468049B64101C1B079BA4001F18D2
:1012B00001207F00039B0743E7503700114B1B7849
:1012C000002B00D0ADE62B68019A1C1213400E4A89
:1012D0009B009B58043586E618220A4B1A70EDE7EE
:1012E000069B3A1DD11A074BD82902DD1A221A7023
:1012F00097E60399A40061581B783960002B09D048
:1013000017008EE6A402002064C50000802D002096
:10131000FDFFFF3F2B6801991C120B40D7499B0032
:101320005B58170004355EE6043F039B3A68A4004F
:10133000E250D34B1B78002B00D072E62B68019A49
:101340001C121340CD4A9B009B5804354BE6039B6F
:10135000A4001C192368043F38685E10FFF7BCFD29
:1013600036180120C64B76001B7806432660002BFA
:1013700000D056E62B68019A1C121340BF4A9B000E
:101380009B5804352FE6069BA4003F1BBC4CBB4278
:101390000CD82378002B00D043E62B68019A1C124E
:1013A0001340B64A9B009B5804351CE6B54801F033
:1013B000F3FD2378002B00D033E62B68019A1C1232
:1013C0001340AE4A9B009B5804350CE6A300ED1871
:1013D000002C00DA38E6AA4B1B78002B00D020E660
:1013E0002B68019A1C121340A44A9B009B58043599
:1013F000F9E5043F3B68042B04D1A300ED18002C51
:1014000000DA21E69E4B1B78002B00D009E62B6802
:10141000019A1C121340994A9B009B580435E2E53F
:10142000043F3B68042B06D0A200AD18002C02DA62
:10143000002B00D108E6924B1B78002B00D0F0E582
:101440002B68019A1C1213408C4A9B009B58043550
:10145000C9E53A1F13685B10013B002B06DD012133
:101460005B00A4000B432D191360EDE5844B1700BE
:101470001B78002B00D0D4E52B68019A1C12134076
:101480007E4A9B009B580435ADE53A00069B0C3222
:10149000D31AD82B03DD1A22794B1A70C1E5FF232A
:1014A00061005B001940FE3BFF3B19433960029924
:1014B00006988968241204916D1A0299AD108978F2
:1014C0002D020D4303999D40091A891099401D432F
:1014D0000B43BB60029B7D609C70E4B26A4BE400EE
:1014E0000392E358029A9360654A1278002A03D067
:1014F00008331D00039F94E51D00019A9B680C357D
:101500001C1213405D4A9B009B58039F6BE53B1FD9
:101510001C68039A069B93422DD10A20E3070CD442
:10152000042C13D90F2322681340042B11D120005F
:1015300001F042FD0AF01EF80630643003F098FD19
:1015400000280FD1043D069B03937DE50720042C62
:10155000F3D02000431E9841FA234042FF33184045
:101560000730EAE7029B2100587804F0E7F80023EF
:10157000029A1370E7E7039B039A0C3B1B680299DE
:101580005B109B00D31A0C3B1C601F1D1300083B13
:101590001B685A108A70D2B23B49D2005B00555882
:1015A0009B0A029A9B009560ED18039B069A043BE8
:1015B0001B685B109B00D3180393314B1B78002BE7
:1015C00000D02EE52B68019A1C1213402B4A9B0079
:1015D0009B58043507E53B1F1868FFF77DFCA40006
:1015E00006003F1B1E2827DC00280DDC244B1B783F
:1015F000002B00D015E52B68019A1C1213401F4ADE
:101600009B009B580435EEE401F038FA033E36188F
:1016100001F034FA1D4B801B9842F9D8184B1B7807
:10162000002B00D0FDE42B68019A1C121340134AD2
:101630009B009B580435D6E40123029A137001F0F5
:101640001DFA029B0A3886195E60FDE43B1F18688C
:10165000FFF742FCA40006003F1B002818DC084BE3
:101660001B78002B00D0DCE42B68019A1C1213407D
:10167000024A9B009B580435B5E4C04664C500008F
:10168000A402002085C70000882500203F420F00EB
:10169000CA4B984203DD1D22C94B1A70C1E40123D5
:1016A000029A137001F0EAF9FA239B005E43029B51
:1016B0000A3E30185860C7E4A300FF1A0023200038
:1016C0001A003900FFF798FBBE4EBF4C316820006E
:1016D00001F080FEBD4B31681860200003F0E2FE8F
:1016E0003168200004F031F83168200002F06DF814
:1016F000B34B1B78002B00D093E42B68019A1C128B
:101700001340B34A9B009B5804356CE4AC4BA400D7
:101710001B783F1B002B00D083E42B68019A1C121E
:101720001340AB4A9B009B5804355CE4029803F0DD
:1017300003FDA34B1B78002B00D072E42B68019AA9
:101740001C121340A24A9B009B5804354BE43B1FDC
:101750001B68002B3ED13B000C3B1B68DA072CD5E5
:10176000390001225B105800083902430A60002B3F
:1017700044DD012259001143381F01603900083946
:1017800009681141CB1A39000C390968114224D07B
:101790009B189340A4001343039AA350884B1B78D3
:1017A000002B00D03DE42B68019A1C121340884A9C
:1017B0009B009B580435FFF716FC042B06D90F221B
:1017C00019680A40092A01D15B68C9E719227C4BD4
:1017D0001A7026E45B10013BC9E7042909D90F22DE
:1017E00008680240092A04D102339B005B58A40018
:1017F000D2E71922724B1A70FFF713FC0435CDE7BC
:10180000A300069AFB189B1AD82B13DC0122631E37
:10181000002C14DC6A4B1B78002B01D0FFF701FC75
:101820002B68019A1C121340694A9B009B5804358F
:10183000FFF7D9FB1A22624B1A70FFF7F2FB3A60EE
:101840001C000437E3E7069A3B1D9B1A5C4ED82B1D
:1018500003DD1A233370FFF7E4FB069B039AA40011
:1018600093422AD23B1F1868FFF736FB011E21DD89
:10187000039B0C3B1A68521082421BDB9007801AB4
:10188000544B4018C018039B8000C2583B1B1A6081
:101890004B4B3F1B1B780437002B01D0FFF7C1FBDC
:1018A0002B68019A1C121340494A9B009B5804352F
:1018B000FFF799FB20233370EAE71823FBE7434B3C
:1018C000A4001A683B1B1F001A603D4B04371B78AD
:1018D000002B01D0FFF7A5FB2B68019A1C121340C7
:1018E0003B4A9B009B580435FFF77DFBA3009C46B9
:1018F000FE1A002C17DC1C22314B1A7000233360B7
:101900006346FF1A2E4B04371B78002B01D0FFF7DC
:1019100088FB2B68019A1C1213402D4A9B009B5890
:101920000435FFF760FB002033685A108300F1583C
:1019300001230B4003D10D21214A1170DFE749102B
:101940008A4200DD0A0001308442EFDC01235200AC
:101950001343D4E7A3009C46FE1A002C17DC1C227C
:10196000174B1A70002333606346FF1A144B043779
:101970001B78002B01D0FFF754FB2B68019A1C1237
:101980001340134A9B009B580435FFF72CFB0020A3
:1019900033685A108300F15801230B4003D10D2105
:1019A000074A1170DFE749108A4200DA0A00013065
:1019B0008442EFDC012352001343D4E780EE36006B
:1019C000A4020020C8050020A50200200800002075
:1019D00064C50000FCFFFF3F3B00083B1868FFF7B1
:1019E0007BFA3B1F06001868FFF776FA0023864251
:1019F00000DA0433A4003A1B17001360E34B0437EA
:101A00001B78002B01D0FFF70CFB2B68019A1C12EE
:101A10001340DF4A9B009B580435FFF7E4FA3B0074
:101A2000083B1868FFF758FA3B1F06001868FFF7D5
:101A300053FAF30FC217B0425341A4003A1B1700E8
:101A40009B001360D14B04371B78002B01D0FFF7AC
:101A5000E8FA2B68019A1C121340CD4A9B009B5850
:101A60000435FFF7C0FA3B00083B18683B1F1968B4
:101A7000A600BE1B0423814202D0042802D8002302
:101A8000336016E001231842F9D10F2302681A408F
:101A9000042AF4D1033A1142F1D10429EFD90A689A
:101AA0001340042BEBD1FFF733FA431E984180001B
:101AB0003060B64BA4001B783F1B0437002B01D0CD
:101AC000FFF7AFFA2B68019A1C121340B04A9B0033
:101AD0009B580435FFF787FA3B00083B18683B1F0B
:101AE0001968A600BE1B0023814202D0042802D838
:101AF0000423336016E001231842F9D10F23026852
:101B00001A40042AF4D1033A1142F1D10429EFD941
:101B10000A681340042BEBD1FFF7FAF9434258410E
:101B200080003060994BA4001B783F1B0437002BCA
:101B300001D0FFF776FA2B68019A1C121340944AE1
:101B40009B009B580435FFF74EFA3B00083B186892
:101B5000FFF7C2F93B1F06001868FFF7BDF9F3173E
:101B6000C20F86425341A4003A1B17009B0013602A
:101B7000864B04371B78002B01D0FFF752FA2B68F5
:101B8000019A1C121340824A9B009B580435FFF7B0
:101B90002AFA3B00083B1868FFF79EF93B1F060036
:101BA0001868FFF799F90023864200DD0433A4008A
:101BB0003A1B17001360754B04371B78002B01D0BC
:101BC000FFF72FFA2B68019A1C121340704A9B00F2
:101BD0009B580435FFF707FA3B1F1B68A400043B22
:101BE0005A1E93413A1B17009B001360674B043742
:101BF0001B78002B01D0FFF714FA2B68019A1C12F6
:101C00001340634A9B009B580435FFF7ECF93B00F7
:101C1000083B1868FFF760F93B1F06001868FFF7DC
:101C20005BF932180120A4003B1B1F005200024345
:101C30001A60564B04371B78002B01D0FFF7F1F9DF
:101C40002B68019A1C121340514A9B009B58043583
:101C5000FFF7C9F93B00083B1868FFF73DF93B1F48
:101C600006001868FFF738F9321A0120A4003B1B60
:101C70001F00520002431A60444B04371B78002BAC
:101C800001D0FFF7CEF92B68019A1C121340404A8D
:101C90009B009B580435FFF7A6F93B00083B1868EA
:101CA000FFF71AF93B1F06001868FFF715F9020045
:101CB0000120A4003B1B1F007243520002431A6024
:101CC000324B04371B78002B01D0FFF7AAF92B68A1
:101CD000019A1C1213402E4A9B009B580435FFF7B3
:101CE00082F93B1F1868FFF7F7F8061E17D11F226D
:101CF000264B1A70A4003B1B1F001E60234B0437A9
:101D00001B78002B01D0FFF78CF92B68019A1C126D
:101D100013401F4A9B009B580435FFF764F93B00B2
:101D2000083B1868FFF7D8F8310006F055FF012688
:101D300040000643DEE73B1F1868FFF7CDF8061E9C
:101D400017D11F22114B1A70A4003B1B1F001E60ED
:101D50000E4B04371B78002B01D0FFF762F92B687C
:101D6000019A1C1213400A4A9B009B580435FFF746
:101D70003AF93B00083B1868FFF7AEF8310007F06E
:101D800011F8012649000E43DEE7C046A4020020F8
:101D900064C500003B1F1868FFF79EF8C217801843
:101DA00050400122A4003B1B1F004000104318605C
:101DB000F64B04371B78002B01D0FFF732F92B6864
:101DC000019A1C121340F24A9B009B580435FFF7FE
:101DD0000AF9A300FE1A3068012C24D1FFF77CF821
:101DE0000494079009F01CFB0799002900DC0121ED
:101DF00006F0D8FF049BA400C91801234900194329
:101E0000E24B3F1B1B7831600437002B01D0FFF7FA
:101E100008F92B68019A1C121340DD4A9B009B585D
:101E20000435FFF7E0F8FFF757F804907068FFF704
:101E300053F8049B0130C31A0793D3E7A300FE1A9B
:101E400031002000049301F047FC049B3060FF1A2E
:101E5000CE4B04371B78002B01D0FFF7E2F82B683C
:101E6000019A1C121340CA4A9B009B580435FFF785
:101E7000BAF83B00083B1868FFF72EF83B1F060036
:101E80001868FFF729F802000120A4003B1B1F007F
:101E90003240520002431A60BC4B04371B78002BBF
:101EA00001D0FFF7BEF82B68019A1C121340B84A04
:101EB0009B009B580435FFF796F83B00083B1868D9
:101EC000FFF70AF806003B1F1868FFF705F8320015
:101ED00002430120A4003B1B1F00520002431A6072
:101EE000AA4B04371B78002B01D0FFF79AF82B6818
:101EF000019A1C121340A64A9B009B580435FFF719
:101F000072F83B00083B1868FEF7E6FF06003B1F2F
:101F10001868FEF7E1FF320042400120A4003B1B9D
:101F20001F00520002431A60984B04371B78002BA5
:101F300001D0FFF776F82B68019A1C121340944ADF
:101F40009B009B580435FFF74EF83B1F1868FEF7BF
:101F5000C3FFC0430122A4003B1B1F0040001043ED
:101F600018608A4B04371B78002B01D0FFF759F813
:101F70002B68019A1C121340854A9B009B5804351C
:101F8000FFF731F83B00083B1868FEF7A5FF060095
:101F90003B1F1868FEF7A0FF32008240510001226B
:101FA000A4003B1B1F000A431A60784B04371B78C0
:101FB000002B01D0FFF735F82B68019A1C12134053
:101FC000734A9B009B580435FFF70DF83B00083B14
:101FD0001868FEF781FF06003B1F1868FEF77CFFBC
:101FE0003200024151000122A4003B1B1F000A43A2
:101FF0001A60664B04371B78002B01D0FFF711F8ED
:102000002B68019A1C121340614A9B009B580435AF
:10201000FEF7E9FF3B000C3B1868FEF75DFF3B0055
:10202000083B06001868FEF757FFF1170200C317B8
:10203000300006F009FF3B1F049005911868FEF779
:102040004BFF02000498059906F0B2FE4300012000
:10205000A4003E1B370018434C4B30601B780437FC
:10206000002B01D0FEF7DDFF2B68019A1C121340F4
:10207000474A9B009B580435FEF7B5FFA300FE1AA4
:10208000310020000493FEF739FD049B3060FF1AF5
:102090003E4B04371B78002B01D0FEF7C2FF2B68A4
:1020A000019A1C1213403A4A9B009B580435FEF7D4
:1020B0009AFFA300FF1A39002000FEF737FD334BCB
:1020C0001B78002B01D0FEF7ACFF2B68019A1C1285
:1020D00013402F4A9B009B580435FEF784FFA30052
:1020E000FE1A310020000493FEF75EFD049B306071
:1020F000FF1A264B04371B78002B01D0FEF791FF07
:102100002B68019A1C121340214A9B009B580435EE
:10211000FEF769FFA300FF1A39002000FEF7D4FD87
:102120001A4B1B78002B01D0FEF77BFF2B68019A1E
:102130001C121340164A9B009B580435FEF753FFB0
:10214000A300FE1A310020000493FEF729FE049B31
:102150003060FF1A0D4B04371B78002B01D0FEF7BF
:1021600060FF2B68019A1C121340094A9B009B5880
:102170000435FEF738FF069B3E1DF31A034CD82B9F
:1021800008DD1A232370FEF74CFFC046A40200208E
:1021900064C5000000F07CFC430001201843237854
:1021A0003860002B02D03700FEF73BFF2B68019A06
:1021B0001C121340F44A9B009B5837000435FEF76D
:1021C00012FF069B3E1DF31AF04CD82B03DD1A2399
:1021D0002370FEF726FF00F051FCED4B4000184045
:1021E0000123184323783860002B02D03700FEF714
:1021F00018FF2B68019A1C121340E34A9B009B585E
:1022000037000435FEF7EFFE0123A600BE1B2000B9
:102210001A003100FEF7F0FDDE4C2068643002F059
:1022200027FF002802D1043DFEF70EFF029B216824
:102230005A78D94803F097FA0123029A37001370AD
:1022400000F01CFCD54B22681B680632534318185B
:10225000029B5860FEF7F8FEA600BE1B200001237B
:1022600000223100FEF7C8FDCA4C2068643002F03D
:10227000FFFE0028D7D0C84803F06CF8DCE7A400C4
:102280003E1BFEF777FE3700C04B30601B780437EB
:10229000002B01D0FEF7C5FE2B68019A1C121340DB
:1022A000B94A9B009B580435FEF79DFEA4003E1BD7
:1022B000300000F01CFC3700B44B30601B78043752
:1022C000002B01D0FEF7ADFE2B68019A1C121340C3
:1022D000AD4A9B009B580435FEF785FEA4003E1BCB
:1022E000300000F006FC3700A84B30601B78043744
:1022F000002B01D0FEF795FE2B68019A1C121340AB
:10230000A14A9B009B580435FEF76DFEA300FE1A00
:1023100031002000049300F0EFFB049B3060FF1AB3
:102320009A4B04371B78002B01D0FEF77AFE2B68FE
:10233000019A1C121340944A9B009B580435FEF7E7
:1023400052FEA4003F1B380000F008FC8F4B1B78A6
:10235000002B01D0FEF765FE2B68019A1C1213407A
:10236000894A9B009B580435FEF73DFEA300FE1AE8
:1023700031002000049300F019FC049B3060FF1A28
:10238000824B04371B78002B01D0FEF74AFE2B68E6
:10239000019A1C1213407C4A9B009B580435FEF79F
:1023A00022FEA4003F1B380000F042FC774B1B7854
:1023B000002B01D0FEF735FE2B68019A1C1213404A
:1023C000714A9B009B580435FEF70DFE0121200049
:1023D00000F016FC6D4B1B78002B01D0FEF721FEA0
:1023E0002B68019A1C121340674A9B009B580435C6
:1023F000FEF7F9FD0021200000F002FC634B1B7882
:10240000002B01D0FEF70DFE2B68019A1C12134021
:102410005D4A9B009B580435FEF7E5FDA4003E1B7A
:10242000300000F027FC3700584B30601B78043731
:10243000002B01D0FEF7F5FD2B68019A1C1213400A
:10244000514A9B009B580435FEF7CDFDA4003E1B6E
:10245000300000F023FC37004C4B30601B78043711
:10246000002B01D0FEF7DDFD2B68019A1C121340F2
:10247000454A9B009B580435FEF7B5FDA4003F1B61
:10248000380000F0E5FB414B1B78002B01D0FEF734
:10249000C8FD2B68019A1C1213403B4A9B009B58B5
:1024A0000435FEF7A0FDA4003F1B380003F076FCC6
:1024B000364B1B78002B01D0FEF7B3FD2B68019A39
:1024C0001C121340304A9B009B580435FEF78BFDCD
:1024D000A4003E1B300003F0F9FC37002B4B3060AA
:1024E0001B780437002B01D0FEF79BFD2B68019A67
:1024F0001C121340244A9B009B580435FEF773FDC1
:10250000A4003F1B380003F0F9FB204B1B78002B85
:1025100001D0FEF786FD2B68019A1C1213401A4A5F
:102520009B009B580435FEF75EFDA4003E1B300067
:1025300003F0FAFB3700154B30601B780437002B93
:1025400001D0FEF76EFD2B68019A1C1213400E4A53
:102550009B009B580435FEF746FDA300FF1A390087
:10256000200001F0E1FB094B1B78002B01D0FEF7A6
:1025700058FD2B68019A1C121340034A9B009B587C
:102580000435FEF730FDC04664C50000A4020020FB
:10259000FEFFFF7FC8050020A502002004000020E8
:1025A000A300FF1A3900200001F0FAF99F4B1B78B5
:1025B000002B01D0FEF735FD2B68019A1C12134049
:1025C0009B4A9B009B580435FEF70DFDA300FF1AA4
:1025D0003900200001F0E0FA944B1B78002B01D069
:1025E000FEF71FFD2B68019A1C121340904A9B00B6
:1025F0009B580435FEF7F7FCA300FF1A39002000B2
:1026000001F0F2FA894B1B78002B01D0FEF709FD8F
:102610002B68019A1C121340854A9B009B58043575
:10262000FEF7E1FCA300FE1A31002000049303F042
:10263000F2FC049B3060FF1A7C4B04371B78002BA4
:1026400001D0FEF7EEFC2B68019A1C121340784A69
:102650009B009B580435FEF7C6FCA300FE1A310010
:102660002000049303F0DFFC049B3060FF1A6F4BE3
:1026700004371B78002B01D0FEF7D3FC2B68019A9E
:102680001C1213406A4A9B009B580435FEF7ABFCB2
:10269000A300FE1A31002000049303F0CCFC049B3D
:1026A0003060FF1A614B04371B78002B01D0FEF716
:1026B000B8FC2B68019A1C1213405D4A9B009B5882
:1026C0000435FEF790FCA300FE1A310020000493AD
:1026D00003F0CCFA049B3060FF1A544B04371B788C
:1026E000002B01D0FEF79DFC2B68019A1C121340B1
:1026F0004F4A9B009B580435FEF775FCA300FF1A58
:102700003900200001F084F9484B1B78002B01D0E0
:10271000FEF787FC2B68019A1C121340444A9B0069
:102720009B580435FEF75FFCA300FF1A3900200018
:1027300001F082FA3D4B1B78002B01D0FEF771FCB3
:102740002B68019A1C121340394A9B009B58043590
:10275000FEF749FCA300FE1A31002000049301F0AB
:10276000E9F9049B3060FF1A304B04371B78002BCB
:1027700001D0FEF756FC2B68019A1C1213402C4A1C
:102780009B009B580435FEF72EFCA300FF1A39006E
:10279000200001F09BF9254B1B78002B01D0FEF7A0
:1027A00040FC2B68019A1C121340214A9B009B5845
:1027B0000435FEF718FC069B029AFB1A9B10136166
:1027C000A300FF1A3900200002F0D6FB174B1B783C
:1027D000002B01D0FEF725FC2B68019A1C12134038
:1027E000134A9B009B580435FEF7FDFB069B029A9B
:1027F000FB1A9B101361A300FE1A31002000049302
:1028000002F0BAFB049B3060FF1A084B04371B78B8
:10281000002B01D0FEF705FC2B68019A1C12134017
:10282000034A9B009B580435FEF7DDFBA402002001
:1028300064C500000023F7B55A1E0192002B07DA89
:1028400001F088FA02F08CFE02F0ECFF19230193EC
:1028500000263000194B1968B14212DD184B1A6876
:1028600001328A420FDAF0241A601D68154F6C435A
:10287000E35D002B1FD0E419022B06D12000FEF7E8
:1028800091FB019BD8E70022EDE7012B0DD1002839
:1028900001D100F0F3F8F0226A43BB185B680A49E3
:1028A000C31A8B4201D80223BB54F0235D43054B6E
:1028B000EB5C022BE2D00136CCE7C046CC05002011
:1028C00000000020281C00203F420F0001220021B0
:1028D0000A4B0B481A61195004301950A2210420E8
:1028E000C9005850C121C0208900800258501A6088
:1028F000044BFC311960044B1A70704700A0004073
:102900000405000000E100E0F3050020042070470A
:10291000F8B550C9012322001A40101E2DD03340B3
:10292000181E2AD0641000201C2C26D81D4B7610AF
:1029300035009E4200DD1D001B4F3B5D012B05D085
:102940000121200004F064FC01233B55174B1B7848
:10295000002B01D1FFF7BAFF0023154A9E420DDC80
:10296000FF2514491448D65CB44202D15E0070526F
:10297000D5540133042BF6D10420F8BDD15C8C4230
:1029800003D10C4A5B009D52F6E70133042BF5D1CD
:102990000023D15CFF2901D1D454F2E70133042B89
:1029A000F7D1E9E788130000D4050020F3050020E3
:1029B0001C0000200E000020DC050000F8B530C926
:1029C000012623003340181E1BD02B003340181E55
:1029D00017D0344100201C2C13D8174F3B5DB34255
:1029E00004D03100200004F013FC3E5569100800AB
:1029F000124A1038124B904204D9012252421A60F6
:102A00000420F8BD1C600F4806F0E6F80E4B188055
:102A10000E4B1B78002B02D1FFF758FFF0E7012285
:102A20000B4B9A64A922D2009A588018A82280B22F
:102A3000D2009850E4E7C046D405002090860100FB
:102A40001800002020A107000C000020F305002042
:102A500000A000400420704701220020054B0649D9
:102A60001A615850043103305850083180185850BA
:102A70001A60704700800040040500000122034BEB
:102A80001A64A822D20098587047C04600800040BF
:102A900010B5FFF7F3FFFA21890006F013F810BD17
:102AA00000487047D8C700001D20704770B5054E1C
:102AB0000400335C0D008B4202D004F0A9FB3555B5
:102AC00070BDC046D405002070B50024064D635D7E
:102AD000012B05D10021200004F09AFB002363554F
:102AE00001341D2CF2D170BDD405002070470D209B
:102AF00070473B2070470000F8B501240B680600C2
:102B00000D00234204D10D20FEF72EFA2000F8BD5F
:102B10005B102000052BFAD80E4A9B009C580E4FE4
:102B20003B5D002B05D00021200004F071FB002349
:102B30003B55012E06DD6B68042B03D102212000DA
:102B400004F066FB200004F011FA01244000204349
:102B5000DDE7C046C0C70000D4050020F8B5012657
:102B60000568354202D04468344203D10D20FEF797
:102B7000FBF9F8BD6D101C2DFBD80A4F7B5D012BB6
:102B800004D03100280004F043FB7E550649641050
:102B90008C4202DCE143C9172140280004F06CFAA2
:102BA000E7E7C046D4050020FF03000070B501240C
:102BB0000D68254204D10D20FEF7D6F9200070BD26
:102BC0006D101C2D17D80024012804DD4C68043C2E
:102BD00063425C416400094E735DA34204D021004E
:102BE000280004F015FB7455280004F045FB030091
:102BF0000420012BE3D00020E1E7C046D4050020EB
:102C000070B504000D001C280ED8084E335C012B53
:102C100004D0012104F0FCFA0123335529002000DF
:102C20004D1EA94104F012FB70BDC046D405002022
:102C3000036810B5DA0703D40D20FEF795F910BD2F
:102C40004168581004394A425141FFF7D9FFF6E76D
:102C500037B569460A00064B30CB30C20368022004
:102C6000042B02D100F098FF37BD00F0BDFFFBE759
:102C700098C7000010B5084C6379002B05D00021DF
:102C8000052004F0C5FA00236371052004F0F4FA6E
:102C900043425841800010BDD405002010B5084CB7
:102CA000E37A002B05D000210B2004F0B1FA0023B9
:102CB000E3720B2004F0E0FA43425841800010BD5B
:102CC000D4050020F7B5304D304E6B6C002B15D07D
:102CD000A8240023E40037596B642D4B18680028A2
:102CE0000CDB2C4B19784A425141C9B2197004F0DF
:102CF000ADFA294B1B88DF19BFB23751AB6C002BE3
:102D000039D00021254B264FF458A9643A780C3469
:102D10000193244D8A4206D02B68032B03D8224A04
:102D2000D05C04F093FA2B68204A0133134004D599
:102D30000422013B5242134301331B4900228C46BB
:102D40002B60042B18D06046C05C591CFF2802D1B0
:102D50000B000122F5E7002A00D02B60012104F0CE
:102D600075FA01233B702B68114A5B009B5AE418EB
:102D7000019BA4B2F450F7BD01235B422B600023FA
:102D80003B700C4BF3E7C046FCA0004000A00040A5
:102D900018000020F20500200C000020440500006F
:102DA000F1050020D00500201C0000200300008059
:102DB0000E00002050460000084B094AFF201A80F0
:102DC0005A809A80DA800023064A07491370074A1E
:102DD000087048708870C870136070470E0000203B
:102DE000DC050000F10500201C000020D0050020BB
:102DF0000122024B52421A607047C0461800002060
:102E000010B5034A0421034802F0A2F810BDC046E1
:102E1000A0C7000030CF0000E12170B5490214487E
:102E200003F09CFEFFF718FE0A2004F099F8002337
:102E3000FF21104A995401331D2BFBD101220020A0
:102E40000D4B01001A6004230C4A0D4D1468002C30
:102E5000FCD02C680002013B20431160002BF5D10F
:102E60000122084B1A6004F035F801F0BFF870BD7C
:102E7000B01B0020D405002000D0004000D100404D
:102E800008D5004004D00040F8B50B4E07003000D4
:102E90000D0003F0ABFE0400A84200DD2C003D0055
:102EA000EB1B9C4205DD300003F0AAFE28700135C3
:102EB000F6E72000F8BDC046B01B002010B50100A9
:102EC000014803F053FE10BDB01B002010B5054CA7
:102ED000200003F059FEE1212000490203F03EFEEC
:102EE00010BDC046B01B0020C3070CD4064B1B68A6
:102EF000834208D8054B1B68984204D8031F1B68FF
:102F0000002B00D018007047FC050020F8050020B9
:102F10000023012210B50A48990001334250642B66
:102F2000FAD1084C084B00211A602000074A07F02C
:102F300097FF074B074A6360074B1A6010BDC046F6
:102F4000802D00200006002008000020D409000089
:102F50003027000004060020F405002010B5044BC3
:102F6000044A1A60044B054A1A60FFF7D1FF10BDEE
:102F7000FC05002000060020F8050020D40F0020EA
:102F8000044B1B68186800090238C343DB1718405C
:102F90007047C046F405002000B59BB0020005490B
:102FA00001A808F0A1FA01A802F0F0F902F03AFC39
:102FB000FCE7C0463FC800000A4BC20704D40428FF
:102FC00004D8094B00D0094B180070470F22036842
:102FD0001A40031D042AF7D0054B092AF4D0054BEB
:102FE000F2E7C04625C80000FAC40000F4C400009F
:102FF00038C800002FC800000020064A0649131FE9
:10300000186013681B0902339B00D2188A42F6D35A
:103010007047C04604060020D40F0020F7B50F24E7
:103020000126304B304A1968304B314D186813680F
:103030001F002740072F25D813681B0902339B0068
:10304000D218AA42F3D300242A4EA500AD1928684D
:10305000FFF74AFF01342860642CF6D1264C206823
:10306000FFF742FF2060254C2068002802D0FFF7C0
:103070003BFF20600025224B1B680093009B9D4274
:1030800013DBF7BD1B099B00D3189A42D4D01F68ED
:10309000374208D1B94206D2B84204D3043F3F6850
:1030A000002F00D01F60043BEFE7F0236B43154A6D
:1030B0009B181A78002A01D10135DFE71F693C23EC
:1030C00000266B43DB199B0001930136BB1BF3D435
:1030D000019BB4001C1B0B4B1C19A069FFF704FFDC
:1030E000A061F2E7FC05002004060020F80500209E
:1030F000D40F0020802D002008000020D40F0020D5
:10310000CC050020281C0020F7B50124204244D122
:10311000224B1B689C4698423FD3214B1B6801936E
:1031200098423AD8031F1B68002B36D1020003686F
:1031300000941B09002B0FD10099131F19609042B6
:103140002BD015682B1F1B68990069180C68013B70
:1031500014600A602A00EDE79D0055192968009C5B
:10316000214218D18C4516D8019C8C4213D30E1FD6
:103170003468002C0FD10F680F343C40072C07D95E
:103180002F60151F2B600B680A601B090A00D1E72E
:1031900000993160CEE7013BCCE7F7BDFC0500208C
:1031A000F80500200D49F0B50B000F260C4D1868EE
:1031B0001C1F276802090232002F0BD000208B420F
:1031C00000D0080020609000091892009B18AB42C4
:1031D000EDD3F0BDB0431860F7E7C0460406002009
:1031E000D40F0020F8B5114C26000F2233681F09B8
:1031F00013420DD07D1CAD00A64204D02A00310040
:10320000200007F01AFE00226319043564191A60C1
:103210000237BF00064BF6199E42E6D31B1B9B10DC
:10322000013B1B012360034B1C60F8BD040600201A
:10323000D40F0020F4050020F0B59BB0FFF71EFC72
:1032400000240700204AA300D0580134FFF75CFF98
:10325000642CF7D11D4B1868FFF756FF1C4B1868FC
:10326000002801D0FFF750FF00261A4B1B689E4232
:1032700016DBFFF797FFFFF7D1FEFFF7B3FFFFF76E
:10328000FDFB154BC21B1B6814491B6801A81B09D9
:10329000023B08F029F901A802F078F81BB0F0BD54
:1032A000F02575430E4BED182B78002B01D101361C
:1032B000DBE72B695C1E002CF9DBA300EB18986997
:1032C000FFF722FF013CF6E7802D002008000020D8
:1032D000D40F0020CC050020F405002005C8000014
:1032E000281C0020F7B5164D4F1C2B6806001B68E4
:1032F0000C0001921B099F420ADBFFF79DFF2B6820
:103300001B681B099F4203DB0A20FDF72DFEFEBD53
:103310002868A71CBA00DB1B81181B010B60296001
:103320000021031F19600F231E40030024012643C0
:1033300040C3083A9A189A42E9D9019902C3FAE7B8
:10334000F4050020F7B503000122134004000D002E
:103350000193002B2AD1164B1B68834226D8154BAC
:103360001B68834222D90F23134F3860006818402E
:10337000FFF7B8FF019B3C68061E3B6016D0236830
:1033800004301B099D4200DD1D00AA00211D251FE0
:1033900007F04AFDFFF730FE2E60FFF73FFE0023E7
:1033A0002B6022680F339A43226034002000FEBD58
:1033B000FC050020F8050020D40F00200323043072
:1033C00010B5C11719400918891000220420FFF711
:1033D00089FF10BD70B5050008000C00FFF7EEFF77
:1033E0000023002804D170BDE95CC21811710133BB
:1033F000A342F9DBE343DB171C40002304192371CC
:10340000F1E7F0B50C009BB0022804DC1C20FDF7AE
:10341000ABFD1BB0F0BD01230868184206D104289B
:1034200004D90F2601683140042901D00E20EEE7AF
:1034300061680D001D40F9D10429F7D90A683240AE
:10344000042AF3D1A2681A4201D10D20DFE7FFF769
:10345000B3FD06006068FFF7AFFDA768010001AC8F
:103460007F103000257002F096FF3900642322009F
:1034700002F0F6FF200008F07DF801002000FFF7C1
:10348000A9FFC6E710B51C4CA544041E02D1FFF7E6
:1034900095FF0BE002F098FE0138062828D805F0C9
:1034A000FDFA090911182904240000208023DB00FB
:1034B0009D4410BD200002F003FF011B2000FFF718
:1034C00089FFF3E7200002F0A9FE43000120184322
:1034D000ECE780226946D200200002F0B6FE684682
:1034E00008F048F801006846E9E704210348E6E7E8
:1034F0000020CCE70420D9E700FCFFFF88C80000CB
:1035000070B50C00022803DC1C20FDF72DFD70BDFA
:1035100001230868184206D1042804D90F25016840
:103520002940042901D00E20EFE761681942FAD141
:103530000429F8D90A682A40042AF4D1A2681A4258
:1035400001D10D20E1E7FFF737FD05006068FFF7C7
:1035500033FDA46801006410280002F01CFF210064
:1035600002F059FFFFF78EFFD1E770B50D0001287B
:1035700003DC1C20FDF7F8FC70BD01240868204224
:1035800006D1042804D90F2102680A40042A01D078
:103590000E20EFE76A682242FAD1042AF8D91368AC
:1035A0000B40042BF4D1FFF707FD06006868FFF716
:1035B00003FD0100300002F0EEFE02F070FF40005B
:1035C0002043D9E7F8B507000C001C20012F0BDDC4
:1035D00001250868284206D1042804D90F21026871
:1035E0000A40042A03D00E20FDF7BEFCF8BD626835
:1035F0002A42F8D1042AF6D913680B40042BF2D1E1
:10360000FFF7DAFC06006068FFF7D6FC0100022F26
:1036100014D0A4682C4211D06410300002F0BBFE1C
:10362000050002F0D1FD012811D1002C02DD013589
:10363000012C06D12800FFF725FFD7E701246442BB
:10364000EBE7280002F048FE013C0500F0E7022805
:10365000F0D1002CEEDD0135012CEBD0002228004A
:10366000110002F06BFE02F037FE013C0500F3E7AB
:1036700010B501240868044016D04410200005F05D
:103680003FFD134905F00AFC07F0F0FA03F038FF9C
:103690000022104B06F0A4FC03F0DAFE07F076FAE5
:1036A00043000120184310BD04280CD90F230268E1
:1036B0001340042B07D1FFF77FFC21000A2208F0FA
:1036C00021F80400DAE70D20FDF74EFCD6E7C046EE
:1036D000D30237390000D040086870B501240500D6
:1036E000254006D1042804D90F2302681340042B77
:1036F00003D00E20FDF738FC70BDFFF75DFC0378AA
:103700002900233B5A4253411022C01807F0FAFF08
:1037100080239B05C218044B9A4201D91420E9E783
:1037200040002043E8E7C046FFFFFF3F10B5034AD3
:103730000621034801F00CFC10BDC04658C800002B
:1037400050C800000020704710B51E20FDF70CFC8B
:1037500010BD10B51E20FDF707FC10BD10B51E20D2
:10376000FDF702FC10BD10B51E20FDF7FDFB10BDDE
:1037700010B51E20FDF7F8FB10BD10B51E20FDF79B
:10378000F3FB10BD10B51E20FDF7EEFB10BD10B50C
:103790001E20FDF7E9FB10BD10B51E20FDF7E4FB70
:1037A00010BD10B51E20FDF7DFFB10BD10B51E20AB
:1037B000FDF7DAFB10BD10B51E20FDF7D5FB10BDDF
:1037C00010B51E20FDF7D0FB10BD704710B5034AA1
:1037D0000E21034801F0BCFB10BDC046C4C8000068
:1037E00034C900000120034B1860034B1B68834061
:1037F00018437047F80F0020D80F0020F0B5EFF302
:1038000010810123194083F31088134C134AA446F6
:103810001268134E013A9340124F134A002B17D0EF
:10382000146803420FD03D682C60C046C046C046B5
:10383000C046C046C046C046C0460C4C1568246809
:1038400025605B08EAE765462C6014683460F8E799
:1038500081F31088F0BDC04608050050200000200C
:103860000C050050E40F0020EC0F0020E00F0020BA
:1038700030B585B001AD0C220649280007F0D4FA16
:103880000024285D01210134FFF710F90C2CF8D138
:1038900005B030BDF3C90000F7B56A46394B01AD3C
:1038A00013801C239370384B2B800A23AB70FFF7D7
:1038B000E5F8364B364CC0182368984201D20023F5
:1038C00023602668002E3DD16B469F5D01213800A4
:1038D000FFF7ECF801360021380003F0B7FC032EA7
:1038E000F2D10026AF5D01213800FFF7DFF8013685
:1038F0000121380003F0AAFC032EF3D1C8200138BF
:10390000C046C046C046C046C046C046C046C04687
:10391000C046C046C046C046F1D100212878FFF716
:10392000C5F868780021FFF7C1F8A8780021FFF7F3
:10393000BDF8FFF7A3F8FA2300251B01C01820608B
:103940002800FEBDFFF79AF8236800259842F7D3B8
:10395000032003F00BFB0600042003F007FB3618DE
:103960000A2003F003FB0B4B9B1B181A0A4BA842BF
:1039700006DB18600023094A236013600125DFE796
:103980001D60F7E71A1B0000030400001027000069
:10399000F00F0020E3030000D80F0020F80F0020F4
:1039A0000022054B10B51A60044B1B68934201D0EE
:1039B00002F0AAFB002010BDF40F0020D41A002052
:1039C00010B5041E10DA00240A4BA400E2580123AB
:1039D0009340094A09491360094A1160094A0A4992
:1039E00011600A4A136010BDFFF75EF8A042EADDDD
:1039F000EAE7C0469CD60000EC0F00200805005006
:103A0000E40F0020E00F00200C05005018050050C6
:103A10002B4BF7B51B680C00002B03D10120404253
:103A2000FFF7CEFF24680126250035401AD0FF227B
:103A30006310120260121040DAB21043FF221B0220
:103A40001204134018431F4B1B68202B06D1B440AF
:103A50001D4BA40EA400E35800021843FFF7CEFE4E
:103A60000020FEBD042CFBD90F2322681340092B34
:103A7000F6D1FF2763683F025B100193019B9D42D3
:103A8000EEDAAB00E3189B68334216D05A10581296
:103A9000D1B238400843FF21120209040A40104302
:103AA000084A1268202A06D15B009B0E06499B003B
:103AB000020258581043FFF7A1FE0135DEE7C04669
:103AC000EC0F002020000020DCCB00000200086882
:103AD00010B5C3070FD540101823012A03DD4A682B
:103AE000042A00D10833054A1360FEF7FFFFFFF7F1
:103AF00067FF002010BD01204042EDE720000020BC
:103B000010B50124044002D04410200010BD042848
:103B10000CD90F2302681340042B07D1FFF74CFA8E
:103B200021000A2207F0EEFD0400EEE70D20FDF76C
:103B30001BFAEAE70868F8B5C3071AD5FFF7E0FFF4
:103B40000300203B5E2B23D805200122584300238D
:103B5000104E451DA84217D005211024375C3C4269
:103B600000D09B180139520064100029F7D10130B0
:103B7000F0E704280CD90F2203681A40042A07D161
:103B80001B0905D00079DBE701205B001843F8BD75
:103B90000120FCE7FFC9000070B508680D00FFF7C1
:103BA000AFFF04006868FFF7ABFF621E0100042A44
:103BB00014D8451E042D11D805236B439B180122F0
:103BC00015009D402B00064805682B430360054BFC
:103BD0001B68002B02D0200002F097FA002070BD75
:103BE000F40F0020D41A002070B508680D00FFF70C
:103BF00087FF04006868FFF783FF621E0100042A44
:103C000013D8451E042D10D805236B439B180122A1
:103C10009A400748036893430360064B1B68002BD8
:103C200003D00022200002F070FA002070BDC046D0
:103C3000F40F0020D41A0020F0B5050089B0086800
:103C40000C00FFF75DFF0690022D36DD6068FFF780
:103C500057FF0190A068FFF753FF04000127231DC1
:103C6000661E0793731C0293079B9E4235D0052363
:103C700073430593019B019D05330493049BAB4261
:103C80001ED0042E16D86B1E042B13D80122059BC0
:103C90002349013B5B199A409446224A0B681068FD
:103CA000069A3A4003920DD062461A430A600122F6
:103CB00000280DD17F000135E0E701240194CDE714
:103CC000029ECFE7624693430B600028F2D0039A2E
:103CD0000299280002F019FAECE7019B1E1D042E40
:103CE0001AD8012C18D1002505273B0021006B4371
:103CF0009B1999400B000A4A013511689943094BF9
:103D000011601B68002B05D0019B0022581D290063
:103D100002F0FBF9052DE8D1002009B0F0BDC04646
:103D2000F40F0020D41A0020086810B5C30703D58B
:103D3000FFF7E6FE054B1860054B1B68002B03D010
:103D4000024B186802F0E2F9002010BDF40F0020C9
:103D5000D41A00207FB5A04C2368002B0AD19F4ABB
:103D60001268002A06D19E4B1B68002B01D0FFF77A
:103D700093FD7FBD9B4D2A68002A26D1984A126880
:103D8000002A1BD0FFF788FD0028F2D0FFF770FD56
:103D9000924B24681A681C60002A16D0002C14D19B
:103DA00001AD0C229049280007F03EF8285D002163
:103DB0000134FEF77BFE0C2CF8D1DAE7874A126853
:103DC000002AE5D1002BE3D0E0E700211A2003F020
:103DD0003DFA00211B2003F039FA00211C2003F0DA
:103DE00035FA2E68012E5CD0022E00D1A2E0002E02
:103DF00050D101363100794C03202368994303F0F8
:103E000025FA0420216801404B42594103F01EFA73
:103E1000102123680A2019404B42594103F016FA39
:103E200080212368090119404B425941062003F0C3
:103E30000DFA80212368090219404B42594107209D
:103E400003F004FA80212368490219404B4259418A
:103E5000092003F0FBF980212368890219404B42B5
:103E60005941192003F0F2F980212368C902194051
:103E70004B425941182003F0E9F9802321681B03C4
:103E800019404B425941172003F0E0F931001A2044
:103E900003F0DCF92B680321581C04F083FF296030
:103EA00067E702214D4C1720236819404B425941C6
:103EB00003F0CCF908212368182019404B425941DE
:103EC00003F0C4F980212368C90019404B425941CD
:103ED000042003F0BBF980212368490119404B42BB
:103EE00059410A2003F0B2F980212368C901194021
:103EF0004B425941032003F0A9F98021236889032B
:103F000019404B425941092003F0A0F98023216850
:103F10001B0419404B425941192003F097F9310015
:103F2000062003F093F93100072003F08FF93100E8
:103F30001B20ADE72021294C1720236819404B4254
:103F4000594103F083F940212368182019404B425E
:103F5000594103F07BF980212368192019404B4215
:103F6000594103F073F980212368490019404B42FD
:103F70005941092003F06AF980212368890019401A
:103F80004B425941072003F061F9802123688901E0
:103F900019404B425941062003F058F9802123680B
:103FA000490319404B4259410A2003F04FF980213F
:103FB0002368C90319404B425941032003F046F9D5
:103FC000802321685B0419404B425941042003F0CF
:103FD0003DF901211C205BE7F40F0020E80F0020D1
:103FE000F80F0020DC0F0020F3C90000012010B5FD
:103FF0004042FFF7E5FC10BD10B5034A0921034814
:1040000000F0A6FF10BDC046DCCC000024CD0000AF
:1040100030B502248025094B094AED009C505C59BB
:10402000002CFCD0A124E400884202D30021995046
:1040300030BD8025ED0018514019F5E700E0014042
:104040000405000010B5002806D1C020B0214002B0
:104050008902FFF7DDFF10BDB02080218002C90278
:10406000F7E7000043425841064B40421840B02356
:104070009B02C018036800201A0E532A01D11B02AC
:10408000180A704700C0FEFF30B501248025054B9B
:10409000054AED009C505C59002CFCD001600021C9
:1040A000995030BD00E001400405000043425841F2
:1040B000074B40421840B0239B02C018A62310B5FE
:1040C0000902DB05090A1943FFF7DEFF10BDC046F0
:1040D00000C0FEFF70B5012480250D4B0D4EED0094
:1040E0009C515C59002CFCD0002902DC00229A5122
:1040F00070BD557814782D02254394780139240435
:104100002543D478043224062C4310C0ECE7C04683
:1041100000E001400405000070B505004B680A008E
:104120009C1C2100A400FFF7D5FF281970BD0000DA
:10413000134B1B68002B0CD08022B023D2029B02B1
:1041400000280BD11A1D5B681B0E522B00D11000EA
:104150007047B022C02392025B02F1E782420DD980
:1041600003681B0E522B09D1436802339B00C01811
:10417000824203D903681B0E522BE9D00020E7E7E7
:10418000FC10002070B50020FFF7D2FFFF260500CD
:10419000002801D1280070BD03681C143440FFF7CB
:1041A000C7FFDA2CF4D10500F2E700008022F0B559
:1041B0005200A1B00021674806F052FE8022002183
:1041C0005200654806F04CFE644BFF271B681A003E
:1041D000049353425A4110000592FFF733FF049CA9
:1041E0000020631E9C415E4B64421C405D4BE41802
:1041F000FFF7C8FF0600002E2DD10498FFF732FF0D
:10420000411C0598FFF752FF059A574D534B2C6000
:104210001A60FEF75BFE514B64201B68A0215A42D6
:1042200053414F4A5B421340B0222C6892029B18C4
:10423000E41A6043490204F0CFFCA02252020300BA
:1042400000924A49220007A807F04EF907A801F09A
:104250009DF821B0F0BD3268131412123A403B4071
:1042600003921A000A3A092A49D83A4B039A995CF0
:10427000002931D110223E4806F0F2FD35002B68AE
:1042800003991A123A40914209D11A143A400B2A62
:1042900027D0132A2DD00A2A01D1354B1D602800C2
:1042A000FFF746FF051EEAD1314B196800290FD0F0
:1042B0002000FFF731FF04002D4B5B1959680029DE
:1042C00003D02000FFF728FF040004350C2DF3D1A4
:1042D000204B0121039A99543000FFF729FF060073
:1042E00089E73B40022BDADC214A9B00D3185D6052
:1042F000D5E7102200211E4806F0B2FDCFE71A00D4
:10430000153A082AE8D8144A0399525C002AE3D1E6
:104310003500152B00D01500300003681A143A4000
:10432000152A0FD01D2A00D10025FFF701FF002814
:10433000F3D1002D04D020002900FFF7EDFE04008A
:10434000054BC6E7039A1B123B409A42EDD105008C
:10435000EBE7C046FC0F002004110020FC100020F9
:1043600000C0FEFF04C0020000110020BDCD00000F
:10437000102F0020F0B50020B7B00024FFF7D8FEC2
:10438000270005002600002D2ED1284D2868FFF7B4
:1043900069FE32003B0001900094254904A807F013
:1043A000A3F804A800F0F2FF224B64201C682B68DD
:1043B000A0215A425341204A5B421340B02292024C
:1043C0009B18E41A6043490204F006FCA022520242
:1043D000030000921949220004A807F085F804A8F8
:1043E00000F0D4FF37B0F0BDFF226B6829689C460F
:1043F0000233FF180B12013613409C4200DA1C00F6
:10440000FF200A140240039262460140019200918B
:10441000039A0B4904A807F067F804A800F0B6FF58
:104420002800FFF785FE0500ADE7C046FC10002020
:104430002ECE00000011002000C0FEFFD8CD0000ED
:104440001ACE000070B50020FFF70CFE040001201A
:10445000FFF708FE844200DA04000A4B1D686A4236
:10446000554128001D60FFF7EDFDA0226B4252026E
:104470001340054A28009B18044A611C1360FFF78B
:1044800015FE70BDFC10002004800100001100200A
:10449000F8B50020FFF7E6FD07000120FFF7E2FD79
:1044A0003E00204D0643204C0DD18021C020C90282
:1044B0004002FFF7ADFD01213000FFF7F7FD1B4B78
:1044C0002E6023601DE0874209DD0023B0212B60B0
:1044D000164B8902236023680020012517E0012381
:1044E00080212B60124BC9022360F4E7120E522A7E
:1044F00008D0002800D023600E4800F047FFFFF7E7
:10450000A1FFF8BD28005A68023292009B188B4226
:1045100005D21A68561CE9D10028F2D0D1E72160F3
:10452000EFE7C046FC1000200011002004800100CD
:1045300004C00200F3CD0000F0B585B00392032261
:104540000333DC17294D1440E4182B68284F5A42D6
:10455000534180225B42D202A4103B409B18A21C14
:104560000291244E910000910190316800980A1840
:10457000934215D2FFF71AFE2B685A42534180220C
:104580005B421F40D202BF183368009A9B189F42BB
:1045900006D2194800F0FAFE0025280005B0F0BD4B
:1045A000029B356819066B461A7BA423DB0513436F
:1045B000FF222F00090C1943019B12041B04134016
:1045C00019432800FFF760FD0837281D21003760D8
:1045D000FFF75AFD002C04D00A9A21003800FFF79B
:1045E00079FD009B083BFF183760D6E7FC100020E0
:1045F00000C0FEFF0011002097CD000010B5FFF7AE
:10460000D5FD10BD70B59AB0FFF742FFFF221E4CDA
:10461000D2000021200006F023FCFF25FFF7B2FDA9
:104620000026002814D10200C300E3580130591EAF
:104630008B41D218FF28F7D1144901A806F054FF86
:1046400001A800F0A3FE124800F0A0FE1AB070BD51
:1046500003681A142A400A2A0AD11A122A40FF2A89
:1046600003D0D200A1180B71A050FFF761FDD8E76D
:10467000132AFAD11B122B40FF2BF6D0DB00E218D5
:104680001671E650F1E7C0468825002063CE000091
:1046900077CE00000021094B094A59600131516071
:1046A00059680029FCD0002119610123936002227E
:1046B000044B8131FF315A501A607047FC100040A2
:1046C0000010004000E100E00222064B0121DA6701
:1046D0000022054B5A61054A11615A69002AFCD033
:1046E0007047C04604E100E0FC10004000100040AC
:1046F00010B5044C2378002B01D0FFF7E5FF002014
:10470000207010BD05120020802301205B055B6E28
:104710005B001843704700000120024B1B685B00E0
:1047200018437047881200200120024B1B685B0071
:1047300018437047240000200120024B1B685B00D7
:10474000184370478C12002070B504000D0016004D
:10475000FEF79EF9802301215B055A6E2670002624
:1047600053006170E1706272010A5A0A6071A171AE
:10477000A272010C5A0C000E5B0EA6702571E1713D
:104780002072E272237370BD10B5044C200006F055
:10479000F1FE01002000FEF71DFE10BD9112002069
:1047A0000E4B10B51B680E4C5A1C0FD00D4C002B35
:1047B0000CD00D4C012B09D00C4C022B06D0094C0F
:1047C000042B03D00A4C052B00D1074C200006F027
:1047D000D1FE01002000FEF7FDFD10BD28000020E5
:1047E0000FCF000008CF00001ACF00001FCF00003D
:1047F00014CF000070B5214C2278002A3DD1204B07
:1048000001215A608022D20511605A68002AFCD02A
:10481000002207201B4B1C4901255A5004395850CF
:1048200008315A5019481A4958501A491A485A50CA
:104830001A495A50A622D2009D50082218495A50AF
:1048400004315850022017495850174917485850FA
:10485000174804395850182016495850C12189006A
:104860005A500539FF395858921802435A50124984
:10487000124A9950FFF70EFF257070BD05120020F7
:10488000FC000040001000400C05000074696275D7
:104890001C05000024050000200004022C05000077
:1048A00014050000340500003C050000FFFF000077
:1048B000211001005405000006120020040500002C
:1048C00070B50E4B06001B78002B01D1FFF792FF4D
:1048D00000200B4D2C7884420ED00A4B20221978F0
:1048E0000323091B1940084B4901C918300006F081
:1048F0009BFA0120013C2C7070BDC04605120020BF
:10490000901200200412002006120020002370B52F
:1049100088B0984235DD0D6801262C0034409C4259
:104920002FD12300042D2CD90F222B681A402300ED
:10493000092A26D16A683F2A23DD6846FFF7C0FFAF
:10494000230000281DD06B4619783300A14203DBF9
:104950006B461B5D5B003343A200AA1801349360D1
:10496000202CF2D1092169444A780B7812021A43AB
:104970008B781B041A43CB781B061343024A13603F
:104980000423180008B070BD8C12002070B5454B90
:104990008AB01B78002B01D1FFF72CFF02AC20005E
:1049A000FFF78EFF002802D100200AB070BD2378E7
:1049B0000B2BF9D96378012BF6D1E378012BF3D1D6
:1049C00000231120384E394D33602B706844237911
:1049D000374A417813600278090211438278120441
:1049E0001143C27812060A4332490A60002B0ED1E5
:1049F000152169444A780B7812021A438B781B04FC
:104A00001A43CB781B0613433360002318E0012BB5
:104A10001AD1152169444A780B7812021A438B780F
:104A20001B041A43CB781A211B06134333600E2351
:104A3000627C6944934200DD130000229A422CD12B
:104A400000220420EA54B0E7022B03D1627B10332A
:104A50001621EEE7042B0DD1152108226944684682
:104A600006F0E2F90098019902F062FC06F08EF877
:104A70003060CAE7052BC8D1152108226944684671
:104A800006F0D2F90098019902F052FC06F07EF887
:104A90003060627D0A231E21CBE7885CA854013276
:104AA000CCE7C04605120020881200209112002099
:104AB000280000208C12002010B5134B04001B7836
:104AC000002B01D1FFF796FEFFF7FEFD00200F4AF5
:104AD0000F49104B5450586001301060586800283E
:104AE000FCD0002018610130906018690028FCD0CB
:104AF000094B0A481B785B011B185350FFF7E4FD74
:104B0000FFF7C8FD10BDC046051200200010004090
:104B100004050000FC1000400412002006120020D2
:104B200010B588B000281DDD0A68012113000B4074
:104B300018D1042A16D90F2014682040092811D151
:104B400050683F280EDD9800101880680024084245
:104B500001D04010C4B26846C4540133202BF2D1B6
:104B6000FFF7AAFF002008B010BD000010B5002814
:104B700013DD0C68E30710D56410532C0DD8084BD7
:104B80001B78002B01D1FFF735FEFFF79DFDA12318
:104B9000044ADB00D450FFF77DFD002010BDC04665
:104BA000051200200010004010B500280EDD0C6832
:104BB000E3070BD56410FF2C08D8054B1B78002B9E
:104BC00001D1FFF717FE034A034BD450002010BD5C
:104BD00005120020001000402405000013B5002835
:104BE00014DD0C68E30711D5094B64100093094BE1
:104BF0000193072C0AD8084B1B78002B01D1FFF733
:104C0000F9FD6B46054A1957054BD150002016BDDA
:104C1000E2ECF0F4F8FC0004051200200010004063
:104C20000C05000070B588B0002820DD012408685C
:104C300004401CD104281AD90F2302681340042B06
:104C400015D1FEF7B9F9060006F094FC050012280C
:104C500000D912252A0002210D326846FFF774FDA3
:104C60006B465D73A54205DC6846FFF725FF002013
:104C700008B070BD2300325D6B449A730134F1E7D4
:104C8000F0B50D008BB0012832DD08680122040068
:104C900014402DD104282BD90F2301680B40042B7D
:104CA00026D16B68134223D0FEF786F96E680700A1
:104CB0007310019306F05EFC05000E2800D90E2546
:104CC0002A000121113202A8FFF73EFD6A4612793F
:104CD00002AB5A7302AA73129373019B76141B0ED4
:104CE000D67313745574A54205DC02A8FFF7E4FEE1
:104CF00000200BB0F0BD3A5D02A963189A7401342C
:104D0000F1E730B589B0002814DD0C68E30711D550
:104D1000102268460021FFF717FD6B466A466510B2
:104D20005D73684663122D0E64149373D473157407
:104D3000FFF7C2FE002009B030BD0000174B184A33
:104D40005968002903D00021596001319160196927
:104D500000291FD0002018618023DB00D35811499F
:104D6000012B18D1A923DB00D3585B420B600E49FD
:104D70000B78032B01D801330B7003200B490B7800
:104D8000013303400B700A495B015B18094953501A
:104D90000123936070470860FAE7C046FC100040AA
:104DA0000010004024000020901200200412002077
:104DB000061200200405000010B5034A1021034824
:104DC00000F0C6F810BDC04688CE00007FCE0000BF
:104DD000044A05491368C85401339B059B0D1360B1
:104DE0007047C046C0160020C012002070B5114C9C
:104DF000114A2368834202DC0023236016E0155C1D
:104E0000411C2E00FA3E012E05D899420FDA555C5E
:104E1000013D1F2D01D90800ECE70100151A565C71
:104E20006E5401318B42FADC181A206070BD157087
:104E3000FAE7C046CC1A0020CC16002010B5FDF7CA
:104E40001DFE064B1A68824201D900221A601B68B7
:104E5000C31A034898428041404210BDBC12002052
:104E6000204E000010B5094C094A2368126893428D
:104E700000D110BD074AD05CFEF720F80028F8D01A
:104E8000236801339B059B0D2360ECE7C4160020CB
:104E9000C0160020C012002010B50400064B074ABF
:104EA0001B6812689B1ADB439B059B0DA34200DB2A
:104EB00010BDFFF7D7FFF1E7C0160020C416002091
:104EC00070B50020FFF734F9FF260500002801D156
:104ED000280070BD03681C143440FFF729F9DA2C50
:104EE000F4D10500F2E7F7B5050056680191B0006E
:104EF000441C06301700FFF7CFFFFB20FFF768FFC9
:104F00001C20FFF765FFE8B2FFF762FFE0B2241252
:104F1000FFF75EFFE0B2FFF75BFF6B461879FFF724
:104F200057FF0025AE4200DCF7BDAB00FB189C68C4
:104F30000135E0B2FFF74CFF2012C0B2FFF748FF87
:104F40002014C0B2FFF744FF200EFFF741FFE9E74E
:104F500070B5074E3368092B08DC0C255D43054C02
:104F60000133285164196160A260336070BDC0468E
:104F7000C8160020202F0020F0B587B002900C004A
:104F8000012803DC1B20FBF7EFFF45E0244B0868FA
:104F90000093C30709D4042807D90F2302681340DC
:104FA000042B02D1FEF708F800901D4B60680193B6
:104FB000C30709D4042807D90F2302681340042B20
:104FC00002D1FDF7F9FF01900027164B1B680493EF
:104FD000049BBB42D6DD0C267E43134B0099F6188A
:104FE000306806F0BDFA051E05D17368B6680593F2
:104FF000059B9D4201DB0137EAE730680199039682
:1050000006F0AEFA0836002808D121000298039B6A
:10501000083102385B68984707B0F0BD0135E7E713
:105020004FC80000C8160020202F002010B5FBF745
:10503000D7FEFEF7E1FFFDF7E3FEFEF777FBFEF795
:10504000C5FBFFF7B9FE00F07DFE01F061F810BD71
:10505000962210B512010021034805F001FF00223D
:10506000024B1A6010BDC046281C0020CC05002051
:10507000064B074A1B6812689B1ADB439B059B0D76
:105080000122834200DC002210007047C01600207D
:10509000C4160020F8B505000C0016001F1E0ED126
:1050A0000320FFF7E5FF002808D0FA20FFF790FE65
:1050B000E8B2FFF78DFEE0B2FFF78AFEF8BD501DA3
:1050C000FFF7D6FF0028F9D0FB20FFF781FEE8B2FA
:1050D000FFF77EFEE0B2FFF77BFEF0B2FFF778FE4F
:1050E0003012C0B2FFF774FE3C00E31B9E42E5DDC8
:1050F0002078FFF76DFE0134F7E7000070B500245B
:10510000F0250B4B1B68A34202DCFFF7A1FF70BD2B
:105110002B006343074A9B181A78002A05D0597858
:10512000002311201A00FFF7B5FF0134E9E7C0465C
:10513000CC050020281C0020F8B507000024F0252D
:105140002B0063430C4A01349E18B74211D03178CA
:1051500000290BD00133D15C002311201A00FFF786
:1051600099FF2A000021300005F07AFE0A2CE7D1D1
:10517000F8BD024B1C60F9E7281C0020CC0500207C
:10518000F0B5150001222F005E4C1740A544019098
:105190000291002F11D005AB1A706A105A70120ECE
:1051A0001A710522691299706D140299DD70FFF76A
:1051B00071FFCF239B009D44F0BD042D1ED90F230A
:1051C0002A681340042B25D1023B04AA280013713E
:1051D000FDF7F2FE040006F0CDF94B4B984200D9E2
:1051E0001800B84204DC421C05AB02990198DEE7C6
:1051F00001377B1EE35C05AAD355F2E7042D7CD171
:10520000032304AA043D13716B425D4105AB557144
:105210000222EAE7092BCCD1042205AB1A706A6896
:10522000511000916946521209789A70009A59708B
:105230001F2A01DD202200926A46127806ACDA703D
:10524000009BBB4202DC05ABE21ACEE70126BB00A5
:10525000EB189868064006D1042837D90F23026856
:105260001340022B0CD101232370431063704212B0
:105270001B0E4014A270E070237105340137DFE784
:10528000042B21D1023B2370FDF796FE039006F01C
:1052900071F9A31C0C2809D86070864201D19C19B1
:1052A000ECE7039A925D9A550136F6E70C2262709C
:1052B000039A925D9A550136092EF9D12E23E37295
:1052C000237363730E34D9E7012B07D1032304380A
:1052D00023704342584160700234CFE7092B09D153
:1052E000053B23704368E6705A105B126270A3702E
:1052F0000434C3E726700134C0E7002D00D058E71E
:105300007EE7C046C4FCFFFF2303000070B5020027
:105310000024F0210D4E0800604380194578954225
:1053200003D001340A2CF6D170BDF022002105F023
:1053300097FD074A1368013BA34200D11460002384
:1053400029001A001120FFF7A5FEEDE7281C002018
:10535000CC05002010B5B2B002236A4604001370D9
:1053600006F008F9C72800D9C7200023984207DCB7
:10537000421C6B46FE211420FFF78CFE32B010BD9C
:10538000694601335A1EA25CCA54EFE730B5B3B088
:1053900002236A460500137006F0ECF80400C728E3
:1053A00000D9C72400239C420BDC20003230FFF7D9
:1053B00073FD621C6B46FF211420FFF76BFE33B0B8
:1053C00030BD694601335A1EAA5CCA54EBE700009F
:1053D000F7B5234B06001B68F02100930023009AC9
:1053E0009A4211DC0024F0231A00624301920199D1
:1053F0001C4A55182F78002F12D001340A2CF3D1F3
:105400001948FFF7C3FF29E00A005A4315488218DC
:105410005078B04202D11278002A1FD10133DEE762
:10542000F0223900280005F01BFD02230D4A0199E6
:10543000EB6053540D4AF1008A58009B6E70AE70B9
:10544000AA602F616F61A34202DC054B01341C602E
:10545000002331001A001020FFF71CFEF7BDC046E4
:10546000CC050020281C002021D400008825002025
:1054700010B5FFF743FEFF24084AE3005B429B1888
:10548000074AD35C043B012B03D8E043C0B2FFF7CB
:105490009FFF013C002CEFD110BDC046FC0700006F
:1054A00088250020F7B50F00FF247F2501901E4AB4
:1054B000E300D31A1D4A9A181278062A01D0032A4B
:1054C00020D1FF22D2009B18186883682B401C2B28
:1054D00018D1C3681A002A40042A13D102692A404D
:1054E000192A0FD11B0A01339B000C30C018FDF79D
:1054F00063FD03780600002B10D006F03BF8002374
:10550000B84209D0013C002CD1D1F7BD019AF15C21
:10551000D25C9142F6D101339F42F7DCE043C0B246
:10552000FFF756FFEEE7C04688250020FC07000085
:1055300070B50500FF24084AE3005B429B18074A48
:10554000D35CAB4203D1E043C0B2FFF741FF013C63
:10555000002CF0D170BDC046FC070000882500205B
:10556000F7B5FDF78BFA514B1A68824201D9002238
:105570001A601A684E49821A8A4200D883E018607D
:10558000FDF786FA071E00D101370020FDF772FBF8
:1055900001900020FDF782FB019B0090454C464D99
:1055A000002B14D02368002B00D07AE02B682760F2
:1055B000002B00D171E0414B01261B78002B63D1F9
:1055C0000920FFF7B5FF3E4B1E703C4B1E70009B41
:1055D000002B12D02B68002B0FD123682F60002BDB
:1055E0001ED0374B01261B78002B52D10920FFF724
:1055F0009FFF334B1E70314B1E702368002B0FD062
:105600002F4E3278002A0BD19F4200D227602368A8
:10561000FB1A312B04D90720FFF78AFF01233370CF
:105620002B68002B0FD0254E3278002A0BD1BB42BD
:1056300000D92F602B68FF1A312F04D90820FFF7FB
:1056400077FF012333702368002B0CD0019B002BC4
:1056500009D11B4E3378002B02D10720FFF768FFDA
:105660000023236033702B68002B0CD0009B002B91
:1056700009D1124C2378002B02D10820FFF758FFE4
:1056800000232B602370F7BD0720FFF751FF0C4B61
:105690009CE70820FFF74CFFADE7009B002B9CD157
:1056A000ABE7009A002A95D1AAE7C046B8120020BD
:1056B0000F270000A8120020B0120020B412002012
:1056C000AC12002037B500240500FFF717FD01A834
:1056D0000194FDF7BDFA21002000FEF761F9FEF705
:1056E00039FBFDF769FBFDF783FBFEF77FFCFDF758
:1056F000EBF9A54204D0FDF70BFC0248FFF746FE8C
:1057000037BDC04612D40000002310B501001A00B6
:105710001120FFF7BFFC10BD07B56B461970694635
:105720005A7013128B701314120ECB700A716B46E1
:10573000010005221320FFF7ADFC07BD10B50A00DC
:1057400001001220FFF71CFD10BD70B50500080018
:105750000C003230FFF7A0FB2B00220000211B20A1
:10576000FFF798FC70BD10B50C0003001100142069
:105770002200FFF78FFC10BD012370B5FF24084AFB
:1057800041185B42884201D3D84370BD06781D0A98
:10579000234073409B009B5801306B40F2E7C046AA
:1057A000F4CF0000002313B501930B4BC20004009B
:1057B000D058002805D0436808309900FFF7DCFF77
:1057C00001900920FFF768FB01AB0422210017209C
:1057D000FFF760FC13BDC04688250020F7B5019097
:1057E000FFF76EFB01250400FF276D42002C01D15D
:1057F0002800FEBD266833143B40152B0DD1210037
:105800000198083105F0ACFE002801D135123D4069
:105810002000FEF78DFC0400E8E71D2BF8D10125E0
:105820006D42F5E7F0B580279DB0FFF71BFBA54C57
:10583000A54D2068FF00391A4019FDF725FB2368A4
:105840000600C3182360002B0ED11DB0F0BD2068E8
:10585000391A2818FDF718FB236806001B18236067
:10586000FDF70CF9994B1860002EF0DC2B78FA2B21
:1058700000D037E12368022B07DCFFF7DFFA0028AE
:10588000E3D00120FFF7B2FADFE76878AC7802389E
:1058900018282BD803F00CF919002C003000340024
:1058A000370040002A004A007C0086008A00A000E1
:1058B000F10002012A002A002A002A002A002A00F8
:1058C0002A002A002A002A001001FF2C0ED02000F6
:1058D000FFF71CFD00227E4BE100CA505B181A71D5
:1058E0002100009213001320FEF726FE0320C9E7D3
:1058F0002000FFF76DFDF9E72000FFF707FDF5E752
:10590000FFF7B6FDF2E7FFF7F9FB0020FFF7DAFE3D
:105910007048FFF73BFDE9E7632CE7D86E4BA20028
:10592000D25821001520FFF72BFCDFE7FFF7C8FA5C
:10593000FF270400002CD9D025682B143B40152BE1
:1059400004D02000FEF7F4FB0400F3E72000083049
:1059500005F010FE06000530FFF79EFAFB20FFF76A
:1059600037FA2D121D20FFF733FAE8B2FFF730FAAD
:10597000F0B2FFF72DFA3012C0B2FFF729FA250076
:105980002B1B9E42DDDD287AFFF722FA0135F7E76F
:1059900000211D2000910B000A00FEF7CDFDFDF750
:1059A000B7FAA3E72000FFF7FDFE9FE7FDF778F8C1
:1059B00003AC4A4A64210090494B200005F062FD87
:1059C00002232000237005F0D5FD230002000021F2
:1059D0001620FFF75FFB89E700243D4AE300D55816
:1059E000002D27D06B689E00701DFFF755FA2B0025
:1059F00000253200083321000120FFF74BFB2F0068
:105A0000FFF75EFA2E00002818D1002F04D03A00CC
:105A100001212000FFF767FA002D04D02A0002219F
:105A20002000FFF760FA002E04D032000021200091
:105A3000FFF759FA0134FF2CCFD157E7FF21036854
:105A40001A120A40A24209D11A140A400B2A08D19C
:105A50000B400CD0012B0CD0022B0CD0FEF768FBB6
:105A6000D1E7132AFAD100252F002E00F6E7060011
:105A7000F4E70700F2E70500F0E70024FFF73EFB3C
:105A80002200210000942300DA20FEF755FDFF22BA
:105A90002100D2000E4805F0E3F980E7012C02D185
:105AA000FEF768FC22E7022C02D1FEF7A7FD1DE7F6
:105AB0000120FFF707FE19E7002321001A001A2032
:105AC00087E7C046CC1A0020CC160020BC1200206C
:105AD00088250020F4D30000802D00200BD4000086
:105AE00006D40000FB2B00D0CBE62268042A00DCA1
:105AF000C3E62E79E878574B360206439E4200DD16
:105B0000BFE6331D9A4200DCB7E6EB5CFE2B00D00B
:105B1000B7E66B78AC78771E1B2B61D019D8072BB2
:105B200047D0082B1CD0012B18D1FF2C16D02000F9
:105B3000FFF7ECFB6D79484AB31E009221002A0062
:105B40000A20FEF7F9FC454BE400E0501B191D71DB
:105B500004E01D2B56D048D31E2B6AD0701D91E651
:105B6000632CFBD86A79022A13D0032A1BD0012A9E
:105B7000F4D1E979AB79090219432B7AA4001B040B
:105B800019436B7A1B060B435B001343344AA35043
:105B9000E4E7002FE2DDB11E2F48FDF71BFC304B80
:105BA000A400E050DAE7AB79A4005A1E93419B00B1
:105BB000ECE7632FD2DC03AD3A002A49280005F058
:105BC00033F900232800EB55FFF708FE0028C5DB5A
:105BD000234B8000C25821001520FFF7D1FABDE702
:105BE00039002048FFF75EFCB8E7FF2CB6D06A7991
:105BF000022AB3D818490B2000912100B31EFEF7EA
:105C00009BFCABE7632F00DD6327002303A99F42C2
:105C10000ADCFB430022DB173B40CB181A7015202F
:105C200000917B1C2100EAE7EA185279CA5401333B
:105C3000EDE7012C92D1002F90DD6B79002B03D082
:105C40001C00322B00DD322464235C43064B1C60B5
:105C500084E7C046F6030000D21600208825002005
:105C6000802D0020D1160020040000200122094BC5
:105C70001A60094A1368002BFCD00322074B1B68EB
:105C8000D8171040C0180123801006384000184370
:105C90007047C04600C0004000C1004008C5004039
:105CA0000120704710B5064C200000F041FD054969
:105CB000200000F065FD0122034B1A6010BDC046B4
:105CC000F81A0020801A0600D01A002010B5012111
:105CD0000D20FCF7EBFE01210E20FCF7E7FE002172
:105CE0000F20FCF7E3FE044C200000F05DFC1021C7
:105CF000200000F075FC10BDD81A002010B5046813
:105D00000D20E30703D56410FF2C03D91720FBF700
:105D10002BF910BDFFF7DAFFE1B2024800F082FC78
:105D20000020F6E7D81A002010B5FFF7CFFF0021BA
:105D3000034800F077FC43000120184310BDC04623
:105D4000D81A002010B5034A08210348FFF700F9CC
:105D500010BDC04638D4000078D400000D4B70B59B
:105D60001B6804000E001500002B01D1FFF79AFFFD
:105D7000E1B2094C200000F09AFDF1B2200000F0E1
:105D80009DFCE9B2200000F099FC200000F0FAFD33
:105D900070BDC046D01A0020F81A002010B50124AA
:105DA0000368234205D04168214202D08268224222
:105DB00003D10D20FBF7D8F810BD5810802801D969
:105DC0001520F7E74910FF2901D91620F2E75210F4
:105DD000FF2A01D91720EDE7FFF7C0FF0020EBE70E
:105DE000F7B501221400904222DD0D682A421FD02F
:105DF0001D4B15411B684C68002B01D1FFF752FF6A
:105E0000E9B201272500194E3D40300000F04FFD5A
:105E1000002D0FD03C413000E1B200F04FFC3000CB
:105E200000F0B0FD0024A04202D02320FBF79CF834
:105E30002000FEBD042CF2D90F2322681340092B49
:105E4000EDD163685B100193019BAB42E7DDAB00D2
:105E5000E3189968394204D04910C9B2300000F003
:105E60002DFC0135F0E7C046D01A0020F81A0020BA
:105E7000144B70B51B6805000E00002B01D1FFF715
:105E800011FF114CEDB22900200000F010FDF1B21D
:105E9000200000F013FC0021200000F013FD00287A
:105EA00001D0404270BD01222900200000F0FAFC20
:105EB000200000F0F4FB0028FAD0200000F0F4FBF2
:105EC000F0E7C046D01A0020F81A002010B50124CF
:105ED0000368234202D04168214203D10D20FBF721
:105EE00043F810BD5810802801D91520F7E7491054
:105EF000FF2901D91620F2E7FFF7BAFF400020433F
:105F0000EFE70000002370B5344D0400EB56013379
:105F10000BD10D211D20FFF7ABFF5A2814D1012210
:105F20002A212A703D38FFF719FF0023EB56022B78
:105F30002AD0032B49D0012B4CD121001D20012454
:105F4000FFF796FF644225E00F211920FFF790FF2D
:105F5000332805D102235F222B7020211A38E2E773
:105F60000D211E20FFF784FFC7280AD1032300223A
:105F70002A21A9382B70FFF7F1FE1B222A211E20AF
:105F8000D1E700232B70D0E7012C13D12921192050
:105F9000FFF76EFF7F2801DD0138FF3803007F33F4
:105FA00001DA7F20404264237F21584302F014FE2F
:105FB000604370BD032C0BD12B211920FFF758FF34
:105FC000043CE7E72D211920B9E721001E20B6E7A0
:105FD000052CF7D0012400206442E4E72C000020C7
:105FE00070B50120FFF78EFF04000320FFF78AFF42
:105FF00005000520FFF786FF6D43644340436419A5
:10600000201804F0F9FD01F0C3FA04F0BFFD4300CD
:106010000120184370BD10B50120FFF773FF430046
:106020000120184310BD10B50320FFF76BFF43009C
:106030000120184310BD10B50520FFF763FF430092
:106040000120184310BD0000F8B501231C00984240
:1060500029DD0F683B4226D04E6835001D4022D115
:10606000042E20D90F2231680A40092A1BD17368F7
:106070005C10202C00DD2024134B1B68002B01D169
:10608000FFF710FE7F10F9B2104F2200380000F029
:1060900009FCA54214DA380000F001FB002804D105
:1060A00001246D002C432000F8BD380000F0FCFAFC
:1060B0000122AB004000F31810439860AD18E8E7E8
:1060C00064000125EEE7C046D01A0020F81A00202F
:1060D0000020704701207047002070470020704763
:1060E0000120704700207047002070470020704753
:1060F0000020704700207047002070470020704744
:1061000000207047002070477047704770470000BC
:1061100010B5034A0E210348FEF71AFF10BDC04612
:10612000C8D4000038D500000378013B1F2B00D9EC
:1061300070470130F8E710B5FFF7F6FF0378002B42
:106140000BD00130222B11D10378002B03D0421C3D
:10615000222B03D11000FFF7E7FF10BD5C2B03D10A
:106160004378002B00D0821C1000EDE73A2BF2D0D0
:106170002C2BF0D07B2B0BD1FFF7D6FF0378002B15
:10618000E9D07D2B01D10130E5E7FFF7D4FFF5E73A
:1061900020225B2B14D1FFF7C7FF0378002BDAD046
:1061A0005D2BF0D0FFF7C7FFF7E7202BD3DD2C2BBB
:1061B000D3D0190091435D29CFD0222BCDD001300F
:1061C0000378002BF1D1C6E7002210B5904216D01B
:1061D000FFF7AAFF03780422222B10D0023A7B2B70
:1061E0000DD0013A5B2B0AD019003039023209294F
:1061F00005D92D2B05D14178303909290AD810004D
:1062000010BD0522742BFAD00132662BF7D0013273
:106210006E2BF4D0581E83415A42F0E770B5FFF759
:1062200083FF037801222D2B01D18018023A00232D
:106230000A2502E06B430130CB1801783039CCB22B
:10624000092CF7D95A43100070BDF8B50C001500A1
:10625000FFF76AFF0378222B02D000232370F8BDDA
:106260000D236A1E210008250C260A279C460130B2
:106270000378222B02D100230B70F0E7002BFAD019
:10628000441C5C2B0BD14378841C622B0ED0662BF4
:106290000ED06E2B0ED0722B0ED0742B0ED0002A87
:1062A000E9DD0B70013A01312000E1E72B00F6E750
:1062B0003300F4E73B00F2E76346F0E70923EEE73B
:1062C00010B50400FFF737FFA04202D90378202B56
:1062D00000D910BD0138F7E710B5002815D00378B4
:1062E000002B13D0FFF720FF2021037802008B43FF
:1062F00000205D2B09D01000FFF71DFF03782C3B19
:106300005A425341C018FFF70FFF10BD1800FCE7B9
:106310000300002070B50C0081420EDD1A785B2A64
:106320000BD1581CFFF700FF0125AC4205D0FFF749
:10633000D3FF002801D00135F7E770BD70B50C0020
:106340001500002901D000230B70002820D003780D
:10635000002B1ED0FFF7E8FE037806002C2B03D19C
:106360000130FFF7E1FE0600337800207D2B0FD0CF
:10637000844204D02A0021003000FFF766FF30007D
:10638000FFF7D9FE03783A2B02D10130FFF7CCFE9C
:1063900070BD1800FCE7F0B50D0004009DB02E782C
:1063A000002E35D02E21280005F0CCF8071E14D081
:1063B000431B0193303E092E14D82800FFF72EFF0F
:1063C00001002000FFF7A4FF0400002C20D0002FC4
:1063D0001ED0019B0133ED18E1E7280005F0CAF853
:1063E0000190E7E723787B2B11D1601C642203A97D
:1063F000FFF7A4FF041E0BD0019A290003A805F0A3
:10640000C0F80028E1D02000FFF795FEEEE7002459
:1064100020001DB0F0BD70B5050000200C008142C9
:106420001DDD2800FFF7D0FE0300681C012B14D0EF
:106430000020022B13D10022681C1100FFF77EFF01
:10644000012C0CD0FFF748FF00221100FFF776FF68
:10645000013CF5E7FFF740FF013C012CFAD170BD8C
:10646000F8B5050000200C0016001F0081420DDD6C
:106470002800FFF7A9FE03000020022B06D1681CAC
:106480003A003100FFF75AFF012C00D1F8BDFFF7A9
:1064900023FF3A003100FFF751FF013CF4E710B54C
:1064A0000024A04218D0FFF73FFE03787B2B0AD1CF
:1064B000013000221100FFF741FF00280CD0FFF748
:1064C0003AFE0134F5E75B2B06D10130FFF704FFFC
:1064D000002801D00134F9E7200010BD10B5FCF709
:1064E0009BFCFCF73BFDFEF7A1FD0448FEF74EFFC9
:1064F000FEF788F8FEF7BCFF10BDC046C1D500000E
:1065000010B5FCF797F910BD70B5002504AC2478E0
:106510000573A94205D10A4B0A4A23210A4804F00F
:1065200015FC01600949920052589B0002715B58AA
:10653000A40083716358856043710223C37170BDE9
:10654000D9D500003ED60000E7D500009CD600005B
:10655000037B002B04D14373837303610133037303
:10656000704700001FB50191A02100240068C900F8
:10657000D2B24450012A10D0A24209D0032A0AD034
:10658000074A8350074B019AC250012343501FBD55
:1065900002221343F4E70422FBE70622F9E7C04690
:1065A000540500002405000010B50400FFF7D0FFDB
:1065B000A1222368A179D20099506179064A20006E
:1065C0009950217904329950044B19685A689B6894
:1065D000FFF7C8FF10BDC0460C050000EC1A0020F4
:1065E0004BB2002B0FDB80233F290FD81F290FD878
:1065F0000F290FD807290FD803290FD81B060168C8
:10660000074A8B50704780239B04F8E7DB04F6E7CA
:106610001B05F4E75B05F2E79B05F0E7DB05EEE71A
:10662000240500000368074A99501A00FC32D1681B
:106630000029FCD0A321C90058580023C0B2D36060
:106640007047C0461C05000007B58022074BD205E5
:106650001A6000229A6002321A710F230C320093E2
:106660000349023B0348FFF74FFF07BDEC1A002028
:1066700000300040D81A0020F8B505000E001700C1
:106680000024BC4208D02B68315D1B682800984765
:10669000002801D00134F4E72000F8BD704710B5A0
:1066A0001C3000F0A9F910BD10B51C3000F096F9AF
:1066B00010BD10B51C3000F0A5F910BD70B5437EBB
:1066C0000D00002B01D1002070BD6430040000F0EB
:1066D000A2F90028F7D12000290000F070F901206C
:1066E000F2E70000F7B50193FA23002504009B00B0
:1066F00083600D4B4560083303601C300F001600AB
:1067000000F052F92000643000F04EF9074A27618A
:10671000B600B35820006375019B9B009B586576BB
:10672000A576A375FEBDC0467CD600009CD60000B1
:106730000123A022C375837D0E49C133FF33D205E7
:106740009B009950437DC133FF339B009950CC226D
:106750000169094B5204CA5005220169243BCA5001
:10676000827D01690833CA500269417D034BD150D3
:106770007047C0460C060000240500000C05000010
:10678000A022002310B50469D200A3500A4CA142F4
:106790000FD90A4C8C425B4109495B420B40CD2129
:1067A000C9045B18046907496350052103699950BE
:1067B00010BDCC235B04F5E7A086010090D0030058
:1067C000000098FD24050000F7B5040000200D002E
:1067D0000193824265D01600402A00D94026270046
:1067E0001C37380000F0F6F8B1232269DB00D550E1
:1067F00080220123216992008B50A27E002A03D1BE
:1068000022691362226913600025731EAB4207D10F
:10681000019B002B04D08022022123699200995011
:10682000012223691A622369FC33DA68002A02D143
:106830009A6A002AF9D09A6A002A0BD1DA60A32357
:106840002269DB00D1583800C9B2013500F0B7F831
:10685000B542DAD3019B2269002B0FD11300FC3320
:106860009B6A002B0AD10133A376D3612369FC33E1
:10687000DA6C002AFCD00022DA640AE0002301214D
:10688000A37651611A002369FC3399680029FCD072
:106890009A602369FC339A6A002A01D000229A6226
:1068A000E8B2FEBD10B50123FFF78EFF10BD030057
:1068B000AC3310B504001970643000F08BF801237C
:1068C000637610BD0023020070B5AC3243760D0034
:1068D0001178B12204000069D20081508022216920
:1068E00092008B5022690133136222699360260063
:1068F0006436300000F080F8002812D0300000F03C
:106900006DF81E4B2269D0502369FC331A6A002AA5
:1069100002D19A6A002AF9D09A6A002A01D11A6231
:10692000E5E723690122002D0DD11900FC31896AA8
:10693000002908D1DA612369FC33DA6C002AFCD023
:106940000022DA6407E05A612369FC339A68002A5E
:10695000FCD000229A6000202369FC339A6A8242AC
:106960000BD098622169064A8B588B501800022B75
:1069700003D0181F431E9841033070BD1C05000052
:10698000C404000010B50121FFF79CFF10BD0000FA
:1069900010B51323142202490248FFF7A3FE10BDCD
:1069A00000400040F81A002010B5402200210400E9
:1069B00004F056FA002320002364636410BD10B570
:1069C0003F24026C531C2340446C9C4201D08154F0
:1069D000036410BD0023036443647047436C026C7E
:1069E000934206D03F21C25C01330B404364100048
:1069F000704701204042FBE7036C406C181A00D539
:106A000040307047436C026C934201D0C05C7047C9
:106A100001204042FBE73F22036C406C01331340EE
:106A2000181A43425841C0B27047000003210A4877
:106A300002680A430260094802680A430260084982
:106A4000084A094B9B1A03DD043BC858D050FBDCB5
:106A500000F012F8F9F758FB2405004054050040F7
:106A6000ECDB00000000002064020020FEE7FEE7EF
:106A7000FEE7FEE7FEE7FEE72D4B10B51A68D2B23F
:106A8000012A0FD12B4A126812070BD12A4AE0249F
:106A90001168F0220800104021422DD127490968D1
:106AA00011422CD01A68D2B2012A12D121490968A8
:106AB00009070ED1F020204909680140402908D17A
:106AC0001E490968014204D18020C121C005C900C6
:106AD00042501B68DBB2012B0DD1164B1B681B0704
:106AE00009D1154B1A68F0231A40A02A0FD1134A76
:106AF00012681A420ED010BD3028CFD0D2E7104A0B
:106B0000104911608021104A09021160CAE7D02A99
:106B1000F1D1ECE70D4B1A68012A04D00C4A1A6037
:106B20001A68012AFCD1C0220A4B1A60E3E7C0466A
:106B3000E00F00F0E40F00F0E80F00F0EC0F00F0C1
:106B400004050040DFFF07C0186C004000EC064061
:106B50007593000014EC06400120704710B50368DF
:106B60001322DB69984710BD70470000054B02698E
:106B7000D1500369FC331A6A002AFCD0002201209C
:106B80001A6270471C050000030010B55C331A78C8
:106B90001F231A401E3B19009140114AD167C2229F
:106BA000042104699200A150026953600269D36014
:106BB000A02300220169DB00CA5001230169094AB0
:106BC0005B428B500169084A8B5001690C3A8B502B
:106BD000016908328B501430FFF7FCFE10BDC0462F
:106BE00004E100E00C0500001405000010B51430AD
:106BF000FFF702FF10BD10B51430FFF703FF10BD03
:106C000010B51430FFF7EAFE10BD0000030070B5A8
:106C10005E331A780469724BE25003005D331A78D0
:106C20000469704BE250030061331C7802696E4BBB
:106C3000012C00D09EE005005F352E78A225ED00E6
:106C40005651020060321578A1220669D200B55073
:106C50000269D4509623DB00994200D88CE0962339
:106C60001B01994200D88AE096235B01994200D823
:106C700088E096239B01994200D885E0E1239B019F
:106C8000994200D882E09623DB01994200D880E047
:106C9000E123DB01994200D87DE096231B02994253
:106CA00000D87AE0E1231B02994200D877E09623CE
:106CB0005B02994200D874E0E1235B02994200D85C
:106CC00071E0E1239B02994200D86EE0474B994264
:106CD00000D86CE0E123DB02994200D86AE0E122AF
:106CE000002312038A425B41414A5B4213408022E7
:106CF00052059B1801693F4A8B50A0230422016969
:106D0000DB00CA5000210369FC33D9600369FC33FE
:106D10001962012301690B6001698B60C12104695B
:106D2000890062501F215C3002780A409340623132
:106D3000314AFF3153500021415600293CDA0F23DC
:106D40000B40083B2D4C9B089B001B190324214042
:106D5000A140FC348C40DD69A5432C00C0258D404A
:106D600029002143D9611F23017819401E3B8B4024
:106D7000136070BD00246CE79E23DB02BAE79D23FD
:106D80001B03B7E71E4BB5E71E4BB3E7EC239B0392
:106D9000B0E71D4BAEE71D4BACE71D4BAAE71D4B03
:106DA000A8E71D4BA6E71D4BA4E71D4BA2E78023D8
:106DB000DB049FE71B4B9DE78C080F4BA400E418F6
:106DC00003230B40FF21C025DB009940AD0066592D
:106DD0008E433100C0269E4033000B436351C2E70F
:106DE0000C050000140500006C05000090D00300A5
:106DF00000D0BEFE2405000000E100E000ED00E050
:106E000000B013000050270000A04E0000F07500F5
:106E100000509D0000F0EB0000903A0100E0D70127
:106E200000B0AF0300705F07F7B5009308AB1B78A5
:106E300000250193FA2304009B0083600E4B4560FC
:106E40000833036014300F001600FFF7ADFD230078
:106E50005C3327611E70009B084A9B0099582300F1
:106E60005D331970019B20009B009A5823005E330C
:106E7000DD701A70FEBDC04620D700009CD6000011
:106E8000036910B51A00FC32D2680400002A0AD047
:106E9000A322D20099581430C9B2FFF790FD002206
:106EA0002369FC33DA6010BD10B50248FFF7E8FF34
:106EB00010BDC046B01B0020162307B50222009368
:106EC0000249013B0248FFF7AFFF07BD0020004029
:106ED000B01B002010B5002801D004F07DFA10BDD1
:106EE0007047000010B500F011F8FFF7F9FF01201E
:106EF00000F000FAFFF7F2FAFFF702FB024B002B5B
:106F0000FAD000E000BFF7E700000000C420114BFA
:106F100080001A5810491140C02212020A431A5028
:106F2000C0218022490092025A501A608023A32275
:106F30000021DB05D20099500122F9309A60074BFD
:106F4000FF301950C12002318000195040301950D3
:106F50001A60704700E100E0FF00FFFF00100140F1
:106F6000014B18607047C04678000020F7B5002339
:106F700020285AD8384B8000C258042A5BD007D842
:106F8000022A54D055D80423012A09D000234CE00A
:106F9000062A54D051D31A2A53D002231B2AF5D1E2
:106FA0002E4A116808294ED909294FD00A240226F1
:106FB000A02001252A4AC00015502A482A4D0768FA
:106FC0001C20BF00074029480197006857590090CE
:106FD00027481B0207401F43C02300989B02034021
:106FE000FF2057515759000207401F43019B1F4381
:106FF000009B58016023184007433E43565101252A
:107000001C4B156058680028FCD000205860A12354
:107010000125DB00D3585560A025ED0050511BB26F
:10702000A14202D015D2611ACB401800FEBD082340
:10703000B6E71023B4E72023B2E74023B0E780236C
:10704000AEE70123ACE708240026B1E70C000126D7
:10705000AEE7091B8B40E8E79CD6000074000020D7
:1070600000700040300000200405000034000020C3
:10707000FF00FFFFFC700040F0B520285BD8364BC6
:107080008000C258354B1E68002E30D1C227344BC9
:10709000BF00D859334C03250440C02000022043D0
:1070A000D851C02480206400800018512E4F1860F1
:1070B0002E4B803CD859FF3CA043D8510437D859B7
:1070C000A8432043D8510837D8590C35A8438446E3
:1070D000072065462843D851A820C0001E50C12073
:1070E0008026800076021E501C601C4B1C601425FC
:1070F00000202B001E4C2E0046433659771C1BD116
:107100004343E250A0230325C132FF329200DB0546
:10711000D550184B1A68082A14D114234343E31896
:107120009A6812485132FF32920059601150DA6861
:10713000C1239B00C250F0BD9642E1D0013003282C
:10714000D9D1F8E7082A02D9083AD140E5E708235F
:107150009A1A9140E1E7C0469CD60000141C00201A
:1071600000E100E0FF00FFFF040500000090004088
:1071700038000020780000202149F0B54A6C2148F1
:10718000002A14D0A025A12600230124ED05F60035
:10719000C258571C06D0C7187F68002F02D027009E
:1071A0009740AF5114333C2BF2D100234B64A02302
:1071B0000121DB0500260F009C4614234B43C31816
:1071C0001A1F1268104C0E4D920014195219526C6D
:1071D000002A10D01A00143A1268551C09D0103B2E
:1071E0001B68FF2B05D03B00934065461A00074BF8
:1071F000EA50FC34666401310429DED1F0BDC0469A
:10720000FC90004038000020009000400C05000079
:1072100000B5202810D80C4A8000835803290BD8C9
:10722000A0220800C133FF33D2059B0001F036FCD9
:10723000020905070021D15000BD0C21FBE7042104
:10724000F9E70321F7E7C0469CD6000020280AD8BA
:10725000074B8000C25801239340A022D205002989
:1072600002D1044953507047A121C900FAE7C04632
:107270009CD600000C05000003000020202B0AD83B
:10728000A021A222C905D2008858034A9B009B581E
:10729000D8400123184070479CD60000F7B506007F
:1072A0000D000C008B180193019B671B9C4207D0BB
:1072B000336821781B683000984701340028F3D1E7
:1072C0003800FEBD0849094A094B10B51B688858AB
:1072D000FA22190A1B0618439200002301F0B4FD9C
:1072E0004904C00B084310BD001001400405000014
:1072F000181C002070B5041E09D0FFF7E3FF05003D
:1073000000F014F8FFF7DEFF401BA042F8D370BD79
:107310000022044B9A60044A13680133DBB2136005
:107320007047C046FC100140181C00207047000048
:10733000F0B5C64600B5CB0F9846404A4B005B0DF2
:107340009A1882B00D000400132A2FDC002A49DBB2
:107350003B4F17413E000E40064323D07F083900C3
:1073600029400C430AD03749BD438C4663445C42F4
:107370005C418023DB021341E4071D434146CE00FC
:1073800031492B008E1922003468756820002900CD
:1073900001F000FF009001910098019922002B005C
:1073A00003F090F802B004BC9046F0BD332A08DD2B
:1073B0008023DB009A42F5D102000B0001F0EAFEC7
:1073C000F0E7224A9446012263445242DA400242E4
:1073D000E8D052080242D1D094438022D2051A410B
:1073E0001443CBE74B005B080343DBD00B031B0BC1
:1073F0001C436342234380244D0C24031B0B234076
:107400006D042B4319004346DA000F4B9B181C6890
:107410005D6802000B002000290001F0BBFE009017
:1074200001910098019922002B0003F04BF842468D
:107430004B005B08D60733431900B3E701FCFFFF9D
:10744000FFFF0F00EEFBFFFF50D70000EDFBFFFF3B
:10745000F8B5274A4B005B0D9A180C000700132A59
:1074600010DC002A36DB234B13410B423AD0802438
:1074700024031441002064189C43060025003000BA
:107480002900F8BD332A0EDD80230600DB000D0045
:107490009A42F4D102000B003800210001F07AFE7C
:1074A00006000D00EBE7144D0600AC4601256344D1
:1074B0006D42DD40AC4663460D000342DFD033230E
:1074C0009A1A323B93401818874200D94C1C6346E5
:1074D0009843D2E7C90FCC070020531CCDD1074BEE
:1074E0001C43CAE706000D000028C0D1C7E7C0460C
:1074F00001FCFFFFFFFF0F00EDFBFFFF0000F03F6F
:1075000030B5214A4B0087B05B0893421EDD1F4A0D
:10751000934205DD02000B0002F0D4FF07B030BD3E
:1075200002AA00F095F803231840049A059B01284D
:1075300013D002281DD0002814D00298039900F01F
:107540006FFB80231B069C466144E7E70023002273
:107550000093002301F0DEF8E0E70298039900F0C1
:107560005FFBDBE7012402980399009401F0D2F855
:10757000D4E7012402980399009401F0CBF880230A
:107580001B069C466144C9E7FB21E93FFFFFEF7FF3
:10759000F0B54746CE4680B58DB004000D0000F032
:1075A00067FA294B06001B780F005BB2984601333F
:1075B00010D022002B002000290003F0CBFA8146D6
:1075C000002807D1002200232000290001F014FC2C
:1075D000002806D1300039000DB00CBC9046994609
:1075E000F0BD01230293194B0694079503934B4674
:1075F0000A93434604940595002B15D000230022DE
:107600001900100002F0E2F8434608900991022B9D
:107610000ED103F0B9FB212303600A9B0193002BD9
:107620000CD1089E099FD5E70023002408930994F4
:1076300002A801F0C1F90028EFD1EAE703F0A4FBAA
:107640000A9B01930360ECE77C00002060D70000F8
:10765000F0B54E464546DE465746E0B5E14B4C0098
:107660008FB09046894664089C4200DC87E0DE4B80
:107670009C4222DCDD4A002900DC92E0DC4B02F077
:1076800021FFDB4B06000F009C4200D17EE1D94A6E
:10769000D94B02F017FF02000B00414630000A6090
:1076A0004B60390002F00EFFD34BD24A02F00AFFC2
:1076B000434601259860D9606BE0D04B9C4200DCCA
:1076C0008FE0CF4B9C4200DD55E1CE4A2315924618
:1076D0009A4451460905631A19001D00040003F07D
:1076E00055FA03F089FA02000B00200029000892E5
:1076F000099302F0E7FE0022C34B02F071FC0F0079
:10770000060003F043FA03F077FA04000D000200CC
:107710000B00300039000A940B9502F0D3FE0022D2
:10772000B94B02F05DFC002200230C900D9101F09A
:107730005DFB002800D192E10023002220002900F7
:1077400001F054FB434243410133B04A41460192A8
:10775000022208A80092524600F07CFB4B4605002E
:10776000002B16DA802243461206944642465B6896
:10777000454263445360D3686344D36009E00B001F
:10778000020041460A604B600022002300258A6007
:10779000CB6028000FB03CBC90469946A246AB4651
:1077A000F0BD934B01F0F6FC914B06000F009C429C
:1077B00000D13DE18F4A904B01F0ECFC02000B0040
:1077C000414630000A604B60390002F07BFE894A76
:1077D000894B01F0DFFC012543466D429860D9607A
:1077E000D7E701F049F88A4A8A4B06000F0002F0F9
:1077F000F7FB0022884B01F0CDFC03F0C7F9050030
:1078000003F0FAF9794A7A4B0490059102F0E8FB0B
:1078100002000B003000390002F054FE754A0600E9
:107820000F0004980599744B02F0DAFB0290039163
:107830001F2D00DCC7E0029A039B3000390002F0E4
:1078400041FE83468A4653465B0024155B0DE31ACE
:10785000102B6CDD04980599D322674B520502F07A
:10786000BFFB02000B00300039000292039302F0CC
:1078700029FE0A0001001300069107920200390058
:10788000300002F01FFE029A039B02F01BFE06006E
:107890000F0004980599614A614B02F0A1FB320088
:1078A0003B0002F00FFE069E079F0B00020039000E
:1078B00030000292039302F005FE4B005B0D8346FD
:1078C0008A46E41A312C32DD04980599B822544BCB
:1078D000920502F085FB03000C0002000293039462
:1078E0000B000698079902F0EDFD02000B00060060
:1078F0000F000698079902F0E5FD029A039B02F03B
:10790000E1FD484A0290039104980599464B02F024
:1079100067FB029A039B02F0D5FD02000B003000CA
:1079200039000292039302F0CDFD83468A465A46FF
:107930005346414630000A604B60390002F0C2FDF8
:10794000029A039B02F0BEFD44460B000200A260B7
:10795000E3604B46002B00DB1BE75B462360802384
:107960001B065344636080231B069C466144A06051
:10797000E1606D420DE70B00020002F0A3FD4346FB
:1079800000259860D9601860596002E7D3221A4B2D
:10799000520502F097FD214A214B0D00040002F030
:1079A00091FD02000B00414620000A604B60290057
:1079B00002F088FD1A4B194A02F084FD4346012566
:1079C0009860D960E5E602000B003000390002F053
:1079D00079FD6B1E154A9B009B5883468A46A3423D
:1079E000A5D130E7FB21E93F7BD90240000040549C
:1079F000FB21F93F3163621A61B4D03DFB2139416B
:107A0000FFFFEF7FEAFBFFFF00007041E8D70000B7
:107A100083C8C96D305FE43F0000E03F7370032E00
:107A20008A19A33BC14920259A837B3968D7000076
:107A3000D3220C4B520501F0ADFB0B4A0B4B04005B
:107A40000D0001F0A7FB02000B00414620000A6078
:107A50004B60290002F036FD034A044BB9E60323CC
:107A600073E6C04661B4D03D7370032E8A19A33B00
:107A7000F8B54746CE46674B80B50A000F0019009F
:107A800005003940994200D19BE004000100002F1D
:107A900069DD3F1500D1B4E05F4B12039C468023A3
:107AA000120B5B0313435B00CA0F67449B184A0029
:107AB000F80703D5D20F5B009B188A0079108C461B
:107AC000002180201624894680030D189D4202DC87
:107AD00029185B1B8144D50F5B00013C5B195200E8
:107AE0004008002CF1D1002080468020202500276E
:107AF000000609E08B425CD0D40F5B00013DE31827
:107B000052004008002D16D0C4198B42F2DD271810
:107B10000E00002C49DB5B1AA242894149425B1AE4
:107B2000121BD40F5B00013D80443100E31852006A
:107B30004008002DE8D113434ED143465B08374936
:107B40004A468846494652104244C90702D5802118
:107B500009060B4361460F05BD18180029000CBC2F
:107B600090469946F8BD7B005B0803433900002B23
:107B7000F5D0002F3CD1E30A153A6405002BFAD06A
:107B80008020400303423FD1002700E00F005B004C
:107B9000791C0342FAD0250020208D40401A29008C
:107BA000D71B2200C2401A4376E7FE43F60F8E1918
:107BB000B1E79442A0D82718002CF6DB1E00002362
:107BC000AEE702003B002800390002F009FA2A0063
:107BD0003B0001F0DFFAC2E74346013303D04346DE
:107BE00001335B08ABE7012398460023C144A6E7B5
:107BF0003B00020002F066FC02000B0001F0E6FD13
:107C0000ADE713000022BBE70127210020207F42BF
:107C1000C6E7C0460000F07F01FCFFFF0000E03F28
:107C2000F0B54746CE4680B587B000920193754BBC
:107C30004F00814688467F089F4263DC02F0A6FF22
:107C4000002800D1D4E04A4643464846414602F067
:107C5000C7F904000D006C4A6C4B02F0C1F96C4A84
:107C60006C4B01F097FA22002B0002F0B9F96A4A36
:107C70006A4B02F027FC22002B0002F0B1F9684A9F
:107C8000684B01F087FA22002B0002F0A9F9664A3E
:107C9000664B02F017FC22002B0002F0A1F9644AA7
:107CA000644B01F077FA22002B0002F099F9029060
:107CB00003910022604B2000290002F091F9029A02
:107CC000039B06000F002000290002F089F9009AAA
:107CD000019B04000D004846414602F081F9020074
:107CE0000B002000290002F0EDFB02000B00300029
:107CF000390002F0E7FB02000B0000204F4902F0C0
:107D0000E1FB70E002000B0002F06AF904000D00D4
:107D10003D4A3E4B02F064F93D4A3E4B01F03AFACF
:107D200022002B0002F05CF93B4A3C4B02F0CAFBFC
:107D300022002B0002F054F9394A3A4B01F02AFA9A
:107D400022002B0002F04CF9374A384B02F0BAFB04
:107D500022002B0002F044F9354A364B01F01AFAA2
:107D60002B00220002F03CF9354B029003919F4218
:107D70009FDD344B00229F423DDC334900207B18BD
:107D80002E4916001F0002F09DFB04900591002271
:107D9000294B2000290002F023F932003B0002F0B9
:107DA00091FB029A039B06000F002000290002F0BD
:107DB00017F9009A019B04000D004846414602F065
:107DC0000FF902000B002000290002F07BFB0200EB
:107DD0000B003000390002F075FB02000B00049824
:107DE000059902F06FFB07B00CBC90469946F0BDB8
:107DF00000201249F7E7154B002604920593144F13
:107E0000C5E7C046FFFF3F3ED43888BEE9FAA8BDAB
:107E1000C4B1B4BD9EEE213EAD529C804F7E923ED9
:107E20009015CB19A001FA3E7751C1166CC1563F8F
:107E30004C5555555555A53F0000E03F0000F03F1B
:107E40003233D33F0000E93F0000E0FF0000E73F8E
:107E50000000D23FF0B5DE464E4645465746E0B5F7
:107E6000DC4CA5440D9114001900A49A0993DA4B37
:107E70009200D6584D1E03901821E01E06960295DA
:107E800000F0AAFEC3430100DB1719404B1C9A0007
:107E90009B1ADB001B190B9105934C1B771918D407
:107EA000A59BA5009C463F1922AE6544013707E01B
:107EB000286802F0A1FE013403C60435BC4208D094
:107EC000002CF5DA00200021013403C60435BC4241
:107ED000F6D1069B002B01DA00F0FDFB069B03990F
:107EE0000133DB009A46099BDA0094460092002297
:107EF000914672AA0492B94A6144934688469AAB65
:107F000063449B44029B002B00DABCE15D460026E3
:107F10000027039C4D442A686B6803CC02F060F88C
:107F200002000B003000390001F034F9083D060072
:107F30000F004445EFD1049B4B441E605F60082353
:107F40009C46E144D145DDD10EA804218446494236
:107F500061448C46069A93009C44614684460A918B
:107F60000399083B63448C460C93009B0092634446
:107F70009B46009A0498D10003008C466344089104
:107F80001E685F68002A33DD954980468C4662444E
:107F9000D300984470AB9A460EAB99460022914BA1
:107FA0003000390002F01CF802F0F0FD02F024FE6F
:107FB00000228D4B04000D0002F012F802000B00AD
:107FC0003000390002F07EFA02F0E0FD4B4601C3BA
:107FD0009946434620001A685B68290001F0DAF8E8
:107FE00008235B429C46E04406000F00D045D5D1F3
:107FF000059B30001A003900984600F0DFFCFF2393
:1080000000229B0504000D0001F0EAFF00F038FC9F
:108010000022764B01F0E4FF02000B002000290053
:1080200002F050FA0D00040002F0B0FD814602F0AB
:10803000E3FD02000B002000290002F043FA0600D5
:1080400040460F00002800DCEEE0009B18215A1E7D
:1080500092000EAB9B58091A1D000D41A9448D409A
:108060005D1B0EAB9D5017231B1A1D41002D2DDDEE
:1080700001239C46009BE144002B00DC1CE20E9C8B
:108080000123002C00D0B5E0009A012A09D0990004
:108090000EAA54580133002C00D0ACE0009A9A424A
:1080A000F5D1059B002B0EDD012B00D1A8E1022BA1
:1080B00009D1009B0EA95A1E92000EAB9B58079344
:1080C0009B029B0A8B50022D00D1C1E000230022AD
:1080D0003000390000F08AFE009B002800D194E2B5
:1080E000069A591E8A4210DC414A0A9894460EAA02
:1080F0006344944600229B0063441C68043B224373
:108100008342FAD1002A00D0C0E0069B0EAA013BB0
:108110009B00D358002B00D0B3E001220C9B043B02
:10812000596801320029FAD0009B9C466244110034
:1081300007921A0001338B4246DC0B986346804657
:10814000A59C4344A046099C9B00A1464A449844F0
:10815000D30022AA9146049A99449446089BA59A72
:1081600063448446614494469A468B00634400937A
:108170004346586802F040FD4B4618605960029B28
:10818000002B24DB4D46039C0026002701E02868D5
:1081900069680CCC01F024FF02000B0030003900AC
:1081A00000F0F8FF083D06000F005C45EFD1534694
:1081B0009E60DF6004239C460433E0449C46009BA1
:1081C000E144E2449845D3D1079B0093D1E60026D1
:1081D0000027ECE794FDFFFF30D9000018FEFFFFF9
:1081E000FFFFFF1F0000703E0000704100002040B4
:1081F000FFFFFF3F002180225204141B0EAA54509F
:10820000009999420EDD0EA884469B000EAA8900B3
:10821000D25861446344CF4800E01A68821A04C30C
:108220008B42FAD101243CE7059B002B06D1009B31
:108230000EAA013B9B00D558ED1517E70022C64B4F
:10824000300000F0F7FD002800D024E100253DE7D4
:1082500032003B000020C14902F034F906000F0053
:10826000002C00D132E7059A0020BC4900F0A6FBA3
:1082700002000B003000390002F024F906000F0064
:1082800024E7012250E70026002754E64B46059AD2
:10829000079388468B000EA9CB58183A089505928B
:1082A000002B0DD18C464146AD4B43449B006344AB
:1082B000043B58680139183A0028F9D088460592DD
:1082C000059A0020A54900F079FB434604000D0003
:1082D000002B00DA05E29E000EAB9C464346DB0015
:1082E00066449C46059370AB9946049F674400978B
:1082F000306802F081FC22002B0001F071FE0022A8
:1083000038607960974B2000290001F069FE083F32
:1083100004000D00043EB945EAD14AAB03939B46E5
:1083200000239A46069B42469946434601320292F2
:1083300004934B46002B00DAAAE080208A4B009D74
:108340009846C005894900260027002408E0082334
:108350009C460835E044544511DC4346186859688A
:108360002A686B6801F03CFE02000B003000390007
:1083700000F010FF013406000F00A145E7DA5B466C
:10838000C0C39B4601239C46009BE244083B0093EC
:10839000029B9A45CDD1049B9846A49B022B00DDFD
:1083A0008EE0002B37DC1FD1059B00271D00039BAF
:1083B00000249C461E006544083E2A686B6838000D
:1083C000210000F0E7FE083D07000C00AE42F4D1AA
:1083D000089B002B03D080231B069C4664443A0074
:1083E00023000D990A604B600720079B18409B23D0
:1083F0009B009D443CBC90469946A246AB46F0BDCE
:10840000009B0EA95A1E92000EAB9B5807935B026D
:108410005B0A8B5057E64346002B00DA70E10020E0
:108420000021DB004AAAD61848AF32687368083EBC
:1084300000F0B0FEB742F8D1089B002B00D025E138
:108440000B0002004A984B990D9C2260636002F079
:1084500039F8434607000C00002B13DD01254CAE14
:10846000B14638002E0021004C4601360CCC00F0FD
:1084700091FEA146B045F7DA089B07000C00002BDF
:1084800000D015E13A0023000D998A60CB60ABE77C
:108490000026002773E701239C46009BE144022548
:1084A000002B00DDEBE532003B0000202B4902F001
:1084B00009F806000F0009E60024F2E54AAB039331
:1084C000A49B032B00D08FE74346002B00DC14E174
:1084D000039ADB009B46130091465B441E685F686D
:1084E000234B43440293DB00994448AB9A464B46E6
:1084F0005C681B681800210032003B00009001916D
:1085000000F048FE04000D0002000B0000980199E5
:1085100001F0D8FF3B00320000F03CFE4B46986073
:10852000D9601C605D6008235B429C46E1442600E4
:108530002F00CA45DBD14346012B00DCE3E0039A60
:1085400013005B441E685F68029BDB0099464A4447
:10855000904610E0FFFFFF000000E03F0000F03F0A
:10856000FFFFFF3F0000703EF0D80000FB21F93F05
:10857000FFFFFF1F984643465C681B6818002100F8
:1085800032003B000090019100F004FE04000D0059
:1085900002000B000098019901F094FF32003B00AB
:1085A00000F0F8FD4346039A9860D9601C605D6056
:1085B000083B26002F009A42DCD14D469446002607
:1085C00000244746083565442A686B68300021005E
:1085D00000F0E0FD083D06000C00AF42F4D1039B23
:1085E0004A9F5D689968D868089B002B65D08022F7
:1085F000120694460D9B6544604464441F605D60B0
:108600009960D8601E615C61EEE69A464B4607931E
:10861000059B30005A423900089500F0CFF900223E
:108620003A4B06000F0000F005FC002824D0384B20
:1086300000223000390001F0D3FC02F0A7FA5246C4
:108640000400950002F0D8FA0022304B01F0C8FC7B
:1086500002000B003000390001F034FF02F096FAFE
:108660000EAA50510122059B52441833904605939F
:1086700093000EAAD45023E65346300039009C00E4
:1086800002F084FA0EAB1851D04619E680230D9AF9
:108690001B06CB18106053600B0002004A984B99E0
:1086A00001F010FF434607000C00002B00DDD5E66B
:1086B00080231B069C466444E4E62B003A000D9D93
:1086C0002A606B600A000300AA60EB60320023009E
:1086D0002A616B6188E6099BDB00009372AB04930F
:1086E00032E4A49B022B00DDE8E6002B00DD92E6DD
:1086F00000D079E6002700246AE6002600246EE711
:108700000020002198E60026340068E70000704150
:108710000000703EF0B5CE46474680B587B0009267
:108720000193474A4B00814688465B08934207DC29
:108730004146484602F02AFA4146031E484666D0A2
:108740004A4643464846414601F04AFC04000D00B3
:1087500002000B004846414601F042FC394A3A4BC0
:1087600006000F002000290001F03AFC374A384B80
:1087700001F0A8FE22002B0001F032FC354A364BF6
:1087800000F008FD22002B0001F02AFC334A344B94
:1087900001F098FE22002B0001F022FC314B324AFE
:1087A00000F0F8FC0E9B02900391002B34D000984F
:1087B000019900222D4B01F013FC029A039B0490B7
:1087C00005913000390001F00BFC02000B00049809
:1087D000059901F077FE22002B0001F001FC009AC0
:1087E000019B01F06FFE224A04000D00214B300076
:1087F000390001F0F5FB02000B002000290000F019
:10880000C9FC02000B004846414601F05BFE07B080
:108810000CBC90469946F0BD02000B0020002900D8
:1088200001F0DEFB124A134B01F04CFE32003B001C
:1088300001F0D6FB4A46434600F0ACFCE7E7C046F1
:10884000FFFF3F3E7CD5CF5A3AD9E53DEB9C2B8AC2
:10885000E6E55A3E7DFEB157E31DC73ED561C1191D
:10886000A0012A3F1111813FA6F810110000E03F3E
:10887000495555555555C53F49004B081900704796
:10888000474AF0B54F4691464B005B0D994446462A
:10889000D6464A46C0B505000C000E0088460700C3
:1088A000132A27DC002A4BDB3E4B13419A460B0070
:1088B00052461340034318D03B4A3C4B280021004A
:1088C00000F068FC0022002300F0AAFA002847D03C
:1088D000002C04DA80234A465B0313419844464641
:1088E000534600279E43380031001CBC90469946F1
:1088F000A246F0BD332A08DD8023DB009945F4D180
:1089000002000B0000F046FCEFE7294A94460122E2
:1089100063445242DA4092460242E6D0224A234B56
:108920002800210000F036FC0022002300F078FA35
:10893000002815D0002C1EDB534646469F430FE00F
:10894000194A1A4B2800210000F024FC00220023C1
:1089500000F066FA002803D0002C04DB0027002674
:1089600038003100C1E76400640825430027002D6A
:10897000F6D0104EF4E74B46142B0BD03422D21A0B
:10898000012393405D19BD4208D201239C462F006C
:10899000E044D1E7133B9C46E044CDE72F00CBE712
:1089A00001FCFFFFFFFF0F009C7500883CE4377E51
:1089B000EDFBFFFF0000F0BF002070474B0070B5DB
:1089C0005B0D14000A00002B1AD14B005B08034317
:1089D00015D0234B002201F003FB224B9C422DDBE0
:1089E0000A004B005B0D363B1F4DE318AB422ADCFF
:1089F000002B0DDD1D4C1B0522401A43110070BDDC
:108A00001B4DAB42F0D102000B0000F0C3FBF6E7B8
:108A10001D00353519DA174B02009C4209DD0B00A9
:108A20001548164900F032F8134A144B01F0D8FAF1
:108A3000E5E70B001248134900F028F8104A114BE3
:108A400001F0CEFADBE70200E9E7084C36332240BA
:108A50001B051343190000220B4B01F0C1FACEE7AE
:108A600000005043B03CFFFFFE070000FFFF0F80F7
:108A7000FF07000050C300009C7500883CE4377E6F
:108A800059F3F8C21F6EA5010000903C30B54A00B2
:108A9000DB0FDB0752081A43110030BD02B47146E8
:108AA00049084900095C49008E4402BC7047C04631
:108AB00003B47146490840004900095A49008E44F0
:108AC00003BC7047002243088B4274D303098B42D6
:108AD0005FD3030A8B4244D3030B8B4228D3030C8E
:108AE0008B420DD3FF22090212BA030C8B4202D330
:108AF0001212090265D0030B8B4219D300E0090A58
:108B0000C30B8B4201D3CB03C01A5241830B8B4260
:108B100001D38B03C01A5241430B8B4201D34B0349
:108B2000C01A5241030B8B4201D30B03C01A5241AE
:108B3000C30A8B4201D3CB02C01A5241830A8B4233
:108B400001D38B02C01A5241430A8B4201D34B021C
:108B5000C01A5241030A8B4201D30B02C01A524180
:108B6000CDD2C3098B4201D3CB01C01A5241830934
:108B70008B4201D38B01C01A524143098B4201D36E
:108B80004B01C01A524103098B4201D30B01C01A99
:108B90005241C3088B4201D3CB00C01A5241830813
:108BA0008B4201D38B00C01A524143088B4201D340
:108BB0004B00C01A5241411A00D2014652411046A0
:108BC0007047FFE701B5002000F0F0F802BDC04695
:108BD0000029F7D076E7704703460B437FD4002285
:108BE00043088B4274D303098B425FD3030A8B4241
:108BF00044D3030B8B4228D3030C8B420DD3FF22AB
:108C0000090212BA030C8B4202D31212090265D078
:108C1000030B8B4219D300E0090AC30B8B4201D32B
:108C2000CB03C01A5241830B8B4201D38B03C01A72
:108C30005241430B8B4201D34B03C01A5241030BE9
:108C40008B4201D30B03C01A5241C30A8B4201D39A
:108C5000CB02C01A5241830A8B4201D38B02C01A45
:108C60005241430A8B4201D34B02C01A5241030ABC
:108C70008B4201D30B02C01A5241CDD2C3098B42A1
:108C800001D3CB01C01A524183098B4201D38B011E
:108C9000C01A524143098B4201D34B01C01A5241C1
:108CA00003098B4201D30B01C01A5241C3088B4206
:108CB00001D3CB00C01A524183088B4201D38B00F1
:108CC000C01A524143088B4201D34B00C01A524193
:108CD000411A00D201465241104670475DE0CA0F6A
:108CE00000D04942031000D34042534000229C462A
:108CF00003098B422DD3030A8B4212D3FC22890134
:108D000012BA030A8B420CD3890192118B4208D309
:108D1000890192118B4204D389013AD0921100E06B
:108D20008909C3098B4201D3CB01C01A524183097F
:108D30008B4201D38B01C01A524143098B4201D3AC
:108D40004B01C01A524103098B4201D30B01C01AD7
:108D50005241C3088B4201D3CB00C01A5241830851
:108D60008B4201D38B00C01A5241D9D243088B42A7
:108D700001D34B00C01A5241411A00D2014663464A
:108D800052415B10104601D34042002B00D54942AE
:108D9000704763465B1000D3404201B5002000F0ED
:108DA00005F802BD0029F8D016E770477047C046A5
:108DB000D0400B1C1141203A03D49C461341184368
:108DC00063465242934018437047C0468446101C85
:108DD00062468C46191C634600E0C0461FB501F090
:108DE00097F8002801D40021C8421FBD10B500F03B
:108DF000EFFF4042013010BD10B501F089F80028A6
:108E000001DB002010BD012010BDC04610B501F0EF
:108E10007FF8002801DD002010BD012010BDC046F4
:108E200010B501F011F8002801DC002010BD012070
:108E300010BDC04610B501F007F8002801DA002087
:108E400010BD012010BDC046F0B5CE464746150402
:108E50002D0C2E0080B50704140C3F0C9946030C12
:108E60007E435D43674363437F19340CE4199C469A
:108E7000A54203D980235B029846C4444B46434332
:108E80005143250C36046544360C2404A4195B199F
:108E9000591820000CBC90469946F0BDF0B54E46DE
:108EA00057464546DE46E0B543025B0A450083B0BF
:108EB0000F1C99462D0EC60F002D57D0FF2D24D024
:108EC0008020DB00C0041843002381469A469B465D
:108ED0007F3D7C027A00FB0F640A120E984623D075
:108EE000FF2A4BD0E30080240020E4047F3A1C4397
:108EF000AD186B1C47460193534677403A000F2B41
:108F000048D87D499B00CB589F46002B00D085E078
:108F100008339A46063B9B467C027A00FB0FFF25EE
:108F2000640A120E9846DBD1002C00D090E0524625
:108F300001231A4392460120DBE74C4658461700AE
:108F4000022824D0032800D1CFE0002200230128EA
:108F50004DD15802D205400AFF071043384303B0F1
:108F60003CBC90469946A246AB46F0BD002B5BD177
:108F700004239A46033B00259B46AAE7FF35002CB5
:108F800060D1524602231A4392460220B1E7FF22E3
:108F90000023DEE74B461B0C9C464B462604360C52
:108FA000180461463300220C6446000C43434E43D0
:108FB0005043544380191A0C1218964203D9802149
:108FC00049028C4664441B041B0C1004C018830126
:108FD0005E1EB341800E1843130C1B199B01034303
:108FE0001C00230179D5012362081C401443019A17
:108FF0007F32002A4DDD630704D00F232340042B6A
:1090000000D00434230103D53C4B019A1C4080322C
:10901000FE2ABCDCA3015B0AD2B29AE70C239A4673
:10902000093BFF259B4654E7180001F071FE4A46B4
:10903000431F76259A4000236D4291462D1A9A4689
:109040009B4646E7524603231A439246032050E7C5
:10905000200001F05DFE431F2D1A9C40763D00204C
:1090600047E780230027DB03FF2272E7424666E7DB
:109070004C463200584662E780234A46DB031A42D8
:1090800022D01C4220D123435B025B0A4746FF22C9
:109090005FE701239A1A1B2A21DC23000199D340A0
:1090A0009E318C401A0023005C1EA34113435A07D3
:1090B00004D00F221A40042A00D004335A0111D4DC
:1090C0009B015B0A002244E780234A46DB031343EB
:1090D0005B025B0A3700FF223BE7019587E700222E
:1090E000002336E70122002333E78023DB032343F9
:1090F0005B025B0AFF222CE740D90000FFFFFFF76D
:1091000070B500283DD0C317C5185D40C40F2800B6
:1091100001F0FEFD9E22121A962A07DCD2B2082820
:1091200033DD083885406802400A23E0992A0BDDC8
:10913000052329001B1AD94003001B339D402B0037
:109140005D1EAB4119430D00052801DD431F9D4005
:109150002B000F490B406E0709D00F263540042D18
:1091600005D004335D0102D59F220B40121A9B01EA
:10917000580AD2B24002D205400AE4071043204305
:1091800070BD002400220020F4E76802400AF1E7E5
:10919000FFFFFFFBF0B54F464646D6460C000903DD
:1091A000C0B5490A470F5E0039431F03DB0F9C46D9
:1091B00065007B0A570F1F436D0DE40F760DA14626
:1091C000C000B846D200AB1B64457BD0002B5FDDEE
:1091D000002E00D0A4E03E00164300D112E15E1E36
:1091E000002E00D09EE1871A4346B84280410125F7
:1091F000C91A4042091A0B0200D431E149024E0A51
:10920000002E00D16EE1300001F082FD0300083B2A
:109210001F2B00DD61E120223900D21A9E40D1408F
:109220009F400E439D4200DD51E15D1B6B1C1F2BD7
:1092300000DD7CE12021C91A3D0030008F408840CC
:10924000DD40791E8F41310007222843D940002597
:1092500007433A40002A09D00F233B40042B05D096
:109260003B1DBB42BF417F42C9191F000B0200D406
:1092700026E26A1CC64B55056D0D9A4200D106E1E7
:10928000C44AFF080A40530752023B43120B8EE0C8
:10929000002B00D0B8E06B1C5B055B0D012B00DCE4
:1092A00030E1871A4346B842B641CB1A76429E1B3C
:1092B000330200D54CE13B003343A1D1002200240E
:1092C000002570E0002B00DCE5E0002E00D183E0FB
:1092D000AF4EB54260D0802636043743B846382BAF
:1092E00000DC3EE1434613431F007A1E97413F18BE
:1092F00087428041404209180B0200D4B0E0A44BE1
:1093000001359D4200D1C3E0A24A7B080A400121F9
:109310000F401F435108D30707221F433A4099E7E4
:109320009B4EB54238D0802636043743B846382B9A
:1093300000DDDCE01F2B00DC30E11E004746203E54
:10934000F740BC46202B04D04026F31A46469E40E8
:109350003243170063467A1E97411F43CCE0002B2F
:1093600000D104E24346134300D159E14B07C00842
:1093700018438023C9081B03194208D04546ED084D
:109380001D4204D14346D008590708432900420F23
:10939000C9007F4D1143C0004B07CA087C49C00873
:1093A00003438D4268D012036D05120B6D0D002131
:1093B00012031800130B0A0D12051A43764B2D05E4
:1093C00013402B435B00E4075B08234319001CBCDC
:1093D00090469946A246F0BD3E00164312D05E1E4E
:1093E000002E00D000E1871887428041414440426E
:1093F000091801250B0233D5022585E764463300A1
:10940000414610001D00C7E7002D00D0DAE00C0037
:109410000443F3D05C1C00D19FE15D4CA64200D117
:109420002FE1DB43382B00DD66E11F2B00DD83E1FC
:1094300020240500E41A0F00DD40D940A040434637
:10944000A7405B1A441EA04198462F433843171A81
:10945000BA42924143465242991A64463500CAE6DE
:1094600007223A40002A00D0F6E64B07CA084849CE
:10947000FF083B438D4296D11900114300D19EE174
:10948000802109030A431203120B414D8FE7150097
:10949000002200238BE7002B00D0C7E06B1C5F0588
:1094A0007F0D012F00DCF1E0394DAB4200D1B9E076
:1094B00085180A00854289414244494251180722D1
:1094C000CF076D082F4349083A401D00C2E6072226
:1094D0003049ED1A31403A40BCE63E00283886401B
:1094E00000279FE6380001F013FC20308EE643464B
:1094F00013431F007A1E9741C71BB8428041404268
:10950000091A78E60E003B0006431343002D61D193
:10951000002E00D0F4E0002B00D11BE1644639009E
:10952000100039E71A4FBB427AD03300FFE6300013
:109530001F3DE840202B03D04021CB1A9E403743EB
:109540007B1E9F41072207433A400021002589E7FF
:10955000171A4346BA42B641591A76428E1B6446E0
:109560004EE61F2B00DDADE020264746F61AB74039
:10957000B9461700B246DF404E463E4337005646D6
:10958000B240561EB24117434246DA408918AEE651
:10959000FF070000FFFF7FFFFFFF0F8020264746E9
:1095A000F61AB740B9461700B246DF404E463E4372
:1095B00037005646B240561EB24117434246DA4083
:1095C000891A99E77F4CA6425BD0802424045B4231
:1095D000214327E7002E0CD1002B00D1CBE06446BD
:1095E00039001000774DD7E6764FBB4218D03300D4
:1095F00075E6002B14D04B07C00818438023C90818
:109600001B03194207D0FC081C4204D17907D0087B
:109610000843E14621004C46420FC9001143C000F7
:10962000684DB9E61D0000220023C0E6002D5BD185
:109630000D00054300D1E2E65D1C00D1B0E0614DB4
:10964000AE421FD0DB43382B71DC1F2B00DD96E0D0
:1096500020250F00ED1AAF40B9460700AA46DF40AB
:109660004D463D432F005546A840D940451EA841D0
:1096700088440743BF189742924151424144350004
:109680003AE6644635004146100085E60B00034388
:10969000002D00D063E6002BF5D04346134300D1E4
:1096A0007AE68718874280410722414440420918E0
:1096B0003A400B0200D4D5E6434B01351940C9E5C9
:1096C000380069E61E004746203EF740BC46202B86
:1096D00004D04026F31A46469E40324317006346A4
:1096E0007A1E97411F4302E6364DAE42CAD080250E
:1096F0002D045B422943A6E70843411E8841A6E6A4
:10970000002B00D148E6871A4346B842B641CB1A2F
:1097100076429E1B33024BD5171A4346BA429241FA
:10972000591A5242891A072264463A4092E5014387
:109730000F00791E8F419DE71C000F00203CE74081
:10974000202B03D04024E31A99400843411E88414E
:1097500038437CE60022002425E6171A4346BA4225
:109760009241591A5242891A6446350043E54146EE
:109770001000144D10E680220024120380E61D0024
:109780000F00203DEF40BC46202B03D04025EB1AB4
:109790009940084307006346781E87411F4369E7E5
:1097A000871897429B4141445B42C9183500A3E5A5
:1097B0003B003343CED0072231003A4052E600232B
:1097C0001A00F4E5FF070000FFFF7FFFF0B55746E2
:1097D000DE464E464546E0B5834607000E03480088
:1097E00085B092461C00360B400DCD0F002800D1ED
:1097F0009DE0954B984239D08023F6001B041E4310
:10980000924A7B0F33439946944603006344009386
:1098100000230026FF00029323031B0B98466300DE
:10982000E40F52465B0D019400D1B3E086498B42B0
:1098300000D19EE04246D100802212040A435146E4
:10984000490F11438B46814952468C460099634427
:10985000CB1A0021D20000932B0063409A460F2EB2
:1098600000D905E17A4BB6009B599F465B463343CE
:10987000994600D0B8E00223082600270090029302
:10988000CAE7CB463A0002990195019B9A46022904
:1098900027D0032900D180E2012944D06D49009BE3
:1098A0008C4663441C00002C38DD530700D013E2C3
:1098B000D2085B46DB0109D55946674B19408B46F8
:1098C0008021C9008C46009B63441C00634B9C4272
:1098D00007DC5B4664055F075B0217431B0B620DE9
:1098E00002E000230027584A00211B031C0B0B0D2C
:1098F0001B05234314055A4A380013401C435346A2
:109900006400DB0764081C43210005B03CBC9046A2
:109910009946A246AB46F0BD0122524201231B1BD1
:10992000382B00DCADE1002200230027DCE75B469A
:10993000334399465ED0002E00D18AE1300001F019
:10994000E7F903000B3B1C2B00DD7BE11D22D31A42
:109950005A460100DA4008398E4013005F4633430F
:1099600099468F403F4B00261B1A00930023029319
:1099700052E7414653460B433B499B468C46009B6E
:10998000634400935B46002B3BD1022300221E431D
:10999000022161E7434613439B4637D04346002BE1
:1099A00000D162E1404601F0B3F903000B3B1C2BF0
:1099B00000DD53E102004146083A914088461D21EE
:1099C000CB1A5146D9400B0041460B439B465346A8
:1099D00093401A00009B25499C46604403008C4636
:1099E00063440093002137E70323B14600900C261F
:1099F000029311E70023009301330426002702930A
:109A00000AE70323C3461E43032125E701331E4310
:109A10000022012120E700239A46802300271B0310
:109A2000094A61E7802349461B03194200D1E2E05D
:109A30005946194200D0DEE00B431B0317001B0BF5
:109A4000A246014A50E7C046FF07000001FCFFFFA5
:109A500080D90000FF030000FFFFFFFEFE070000AB
:109A6000FFFF0F800DFCFFFF01F8FFFFF303000075
:109A7000D94500D9CBE000D1C6E03C0048460027DC
:109A8000009B013B00935B46160E1B021E43130214
:109A9000984633041B0C9946310C0191FFF798F856
:109AA0004A4642430B04210C050019438A4207D958
:109AB0008919013D8E4203D88A4201D9851E891930
:109AC000881A0199FFF784F809048C464A46210454
:109AD00064464243090C030021438A4204D9891990
:109AE000013B8E4200D8F1E02D041D43AB464346B6
:109AF000891A4246280C12041D0C5B46140C2200E5
:109B00001B041B0C5A4303946B4344430295684364
:109B10001B19150CEB189C4203D980246402A4463F
:109B200060441C0C15041B042D0C20185D19814287
:109B300077D373D00C1AA24A7D1BAF42BF41944623
:109B4000009B7F426344E01B1C00864200D1DBE0A7
:109B50000199FFF73DF84A4642430B04290C0700E0
:109B600019438A4207D98919013F8E4203D88A4294
:109B700001D9871E8919881A0199FFF729F8090464
:109B80004A46894629044D464243090C03002943AD
:109B90008A4207D98919013B8E4203D88A4201D9EA
:109BA000831E89193F04891A3A00039F1A4338001B
:109BB00013041B0C584381460298150C6F43434312
:109BC00045434846000C8446DB1963449F4203D951
:109BD000802040028446654448461F0C00041B0454
:109BE000000C7D191818A94200D284E000D17FE052
:109BF00001231A4357E680234A461B0313431B03E2
:109C00001B0BAA466F4A6FE6BA4200D935E74B46AE
:109C1000DC0758087B081C43FF0734E70024AF42E9
:109C200089D247444745A4415B466442A41964185D
:109C3000013BA6421ED2A0426DD800D1B6E0241A44
:109C40009B4678E703005A46283B9A4000279146F6
:109C500088E6584601F05CF8203072E60300524670
:109C6000283B9A4093460022B4E6504601F050F853
:109C700020309AE6A642E2D1B845DCD9341A9B4698
:109C800059E71F2B65DC504C0099A4465C466144A3
:109C900008008C4011008240D940501E82410C4384
:109CA00014435A46DA401300620709D00F222240BB
:109CB000042A05D02200141D9442894149425B18B0
:109CC0001A0262D50122002300270DE68A4200D83D
:109CD0000AE7831E891907E70F231340042B00D1DD
:109CE000E6E5171D9742924153429B44FA08E0E58E
:109CF000002800D1D7E57118531EB14227D3A942DD
:109D000015D358D01A0073E7002B00DC04E60123BA
:109D100000229B44CDE502234744474589415B42ED
:109D20009C46494289190C19E344241A03E7434627
:109D30005F0047459B41B8465B429E19023A89192C
:109D4000A94200D054E7404500D051E7ABE51A00E6
:109D5000F6E71F215F4649420C1BE740202B07D046
:109D60001A49009B8C46634418005B4683401A43A3
:109D7000501E82413A4307270023174009D00F2184
:109D8000002311401400042995D122005F075B02D3
:109D90001B0BD20817430022A6E5802359461B035C
:109DA0000B431B0317001B0B064A9DE5BD42B2D8AF
:109DB0009B460024BFE68045B9D31A00C3E7C046DE
:109DC000FF030000FF0700001E0400003E04000027
:109DD000F0B54F464646D6468446C0B58046194E35
:109DE00018030F034D00000B5C0082463F0B6D0D06
:109DF000C90F9146640DDB0F0120B5420AD0B44271
:109E000003D0A54201D157450CD01CBC90469946C1
:109E1000A246F0BD66463E43F7D1AC42F5D154466A
:109E20001443F2D10120C845EFD1994207D0002D4B
:109E3000EBD163461F433800471EB841E5E70020D9
:109E4000E3E7C046FF070000F0B54F464646D6465A
:109E50004D00C0B50E03C90F8A462C491F035C0094
:109E60008046360B6D0D91463F0B640DDB0F8D4226
:109E70001ED08C4216D0002D1ED130438446002CBB
:109E800001D13A4323D06246002A1AD09A4529D0FC
:109E9000514602200139084001381CBC90469946C1
:109EA000A246F0BD39001143E5D002204042F4E75C
:109EB0003043FAD1AC420FD0002C0FD13A43E7D057
:109EC0000CE00122013B934318000130E5E76346B3
:109ED0000020002BE1D0DBE73A43E6D19A45D7D109
:109EE000A542D5DCA54205DBBE42D1D808D0002072
:109EF000BE42D2D250460123013898430130CCE70C
:109F0000C845C5D80020C845F4D3C6E7FF07000000
:109F1000F0B54F464646D6464D00C0B50E03C90FB4
:109F20008A462E491F035C008046360B6D0D914614
:109F30003F0B640DDB0F8D4218D08C4211D0002DE9
:109F400018D130438446002C1ED13A431CD16346BD
:109F50000020002B30D05146022001390840013842
:109F60002AE039001143EAD0022025E03043FBD13A
:109F7000AC4226D0002C26D13A4324D151460220AF
:109F800001390840013817E06246002A0FD09A458F
:109F9000E1D1A54205DBBE42DDD819D00020BE428A
:109FA0000AD25046012301389843013004E00122CF
:109FB000013B9343180001301CBC90469946A246D1
:109FC000F0BD3A43D0D19A45C5D1A542C3DCE0E704
:109FD000C845C0D80020C845E3D3EDE7FF0700001F
:109FE000F0B55746DE464E464546E0B58346060088
:109FF0000F03480087B092461D003F0B400DCC0F69
:10A00000002800D16FE0DE4B984238D08023FF005B
:10A010001B041F43730F3B430193DA4B0027994600
:10A0200000239B46F60081442B0369001B0B52461C
:10A030009846490DED0F002900D185E0D04B99429B
:10A0400000D173E04346DA0080231B0413435246D9
:10A05000CC48520F84461343524600206144D2003C
:10A0600089442100694000918C46012149448A4677
:10A070000F2F00D990E0C449BF00CF59BF465B46BF
:10A080003B43019300D06AE1022308270026814662
:10A090009B46C9E732005846019B61460091022861
:10A0A00000D175E0032800D1FEE1012800D02CE1A9
:10A0B00000230027002600253F032A0D3F0BB3484D
:10A0C00012053A4302401B051343009A5B00D10777
:10A0D0005B080B433000190007B03CBC9046994622
:10A0E000A246AB46F0BD5B463B43019300D12FE156
:10A0F000002F00D1A5E1380000F00AFE03000B3B61
:10A100001C2B00DD96E11D22D31A5A460100DA40CD
:10A110005E4608398F4013008E403B4301939C4BB1
:10A1200000271B1A994600239B467DE7414653466C
:10A130000B4393498C46E144002B00D01AE10222E4
:10A140000220174300228CE7134300D10DE1434660
:10A15000002B00D181E1404600F0DAFD02000B3A0D
:10A160001C2A00DD72E10100434608398B40984605
:10A170001D239A1A5346D3401A00434613435246AE
:10A180008A404946081A824989468144002068E786
:10A190007B4B002700268EE7140C1204120C1100D2
:10A1A000370C3604350C794328008C462E0060436A
:10A1B0006044834656432100300C8046584679431C
:10A1C00040440291844506D98846802149028C4644
:10A1D000E044414602913604010C360C00048B46E3
:10A1E00081191E0C1B041B0C0391190079438C462A
:10A1F000280075436544A8465843050C45447743F9
:10A20000A94203D9802149028C466744290C8C4617
:10A2100039000004000C2D042D186144AB44059155
:10A220005946049101990F043F0C080C3900514321
:10A230004243904602008C46090C8B4662437C43A5
:10A2400044445C44A04503D98021490288464244E5
:10A25000210C884661460904090C8C463900594393
:10A26000434370437E430F0CF6182404BE19644424
:10A2700042448C46B34203D980235B029846404453
:10A28000029B61469846049B370443449B46AB457A
:10A29000AD416B420D0405992D0C8C467F19674426
:10A2A000FD18A8465D462D19A542A4419346644277
:10A2B000A446C344DC448F42BF4198459B4193452B
:10A2C0009241A445A4415B427F421F43360C524257
:10A2D0006442BF192243BF18624638184302D20DA8
:10A2E000039913436A020A43501E82416146ED0DF1
:10A2F0002A434E023243D90100D4B3E0012650086C
:10A3000032400243DE0732435B08224C5444002CA7
:10A3100062DD510709D00F201040042805D0101D20
:10A320009042924152429B180200D90104D58024E8
:10A330001948E400034054441848844200DD27E7EC
:10A340005E075B02D2081F0B630516435B0DB2E686
:10A35000002399460133042700269B4664E6032325
:10A36000019781460C279B465EE601220120174398
:10A37000002276E6032303201F43434671E6C046CE
:10A38000FF07000001FCFFFFC0D90000FFFF0F80A6
:10A390000DFCFFFFFF030000FFFFFFFEFE070000B4
:10A3A0000023802700933F030026434B83E6019B55
:10A3B0003200A446584670E6AC466EE68027019906
:10A3C0003F0339422DD03B422BD11F433F033F0B6C
:10A3D00000951600384B6EE601252D1B382D00DD4B
:10A3E00066E61F2D40DC35481C00504416008240B4
:10A3F0008440EE40501E824134431443EB406207D8
:10A4000009D00F222240042A05D02200141D9442B4
:10A41000804140421B181A023ED501230027002626
:10A4200049E68027019B3F031F433F033F0B0094F6
:10A43000214B40E603005A46283B9A4000260192F1
:10A440006DE6584600F064FC203057E603005246A3
:10A45000283B9A401300002293E6504600F058FC37
:10A4600020307BE6CA4650E71F201E004042041BF6
:10A47000E640202D03D0124C5444A3401A43501EF2
:10A480008241324307260027164009D00F200023BF
:10A49000104014000428B9D122005E075B021F0B94
:10A4A000D2081643002306E680273F031F433F03DD
:10A4B0003F0B1600004BFEE5FF0700001E040000E6
:10A4C0003E040000F8B557464E464546DE460C00B1
:10A4D0000903E0B5490A460F5F0031431E03DB0F55
:10A4E000760A9B46530F3343C84E6500C000E40F05
:10A4F000D2006D0DA24681467F0D9C469046B74224
:10A5000000D1B9E05B46012673409B46EE1BA34594
:10A5100000D183E0002E63DD002F00D0B1E0634660
:10A52000134300D123E1731E002B00D0BAE1861A39
:10A530006346B04280410125C91A4042091A0B0204
:10A5400000D447E149024B0A98464346002B00D10C
:10A5500089E1404600F0DCFB0300083B1F2B00DDD7
:10A560007CE120223000D21A4146D04099400200BE
:10A570009E400A439D4200DD6AE15D1B6B1C1F2B60
:10A5800000DD94E1202110003500C91A8E40DA4028
:10A590008840DD40711E8E411100072228430025AE
:10A5A00006433240002A09D00F233340042B05D044
:10A5B000331DB342B641764289191E000B0200D406
:10A5C0003DE26A1C914B55056D0D9A4200D119E18F
:10A5D0008F4AF6080A40570752023743120B9BE096
:10A5E000002E00D0C5E06E1C7605760D012E00DC35
:10A5F00048E16746861ACB1BB042BF417F42B8464E
:10A600001F004346FF1A3B00B8461B0200D55FE11E
:10A6100037439AD100220024002579E0002E00DC87
:10A62000FAE0002F00D18DE0784B9D4267D0802367
:10A6300067461B041F43BC46382E00DC52E16346CC
:10A6400013435A1E93411E18864280414042091806
:10A650000B0200D4BEE06D4B01359D4200D1D2E02B
:10A660006B4A73080A4001210E401E435108D3076C
:10A6700007221E43324095E71E00164300D045E7EF
:10A6800040E7624B9D423AD0802367461B041F433C
:10A69000BC46382E00DDEBE01F2E00DC3AE1330033
:10A6A0006746203BDF403B00202E05D04027BF1BE4
:10A6B0006646BE40324390464646721E964133433C
:10A6C000DAE0002B00D114E26346134300D168E1C5
:10A6D00080234E07C008C9081B030643194208D04F
:10A6E0006046C008184204D163460100D2085E07E4
:10A6F0001643F3009946C900720F444D11434B466F
:10A70000DE08424B4F073743CA089D4200D16EE036
:10A7100012036D05120B6D0D00211203130B0A0DB0
:10A7200012051A433B4B2D0513402B435B00E407F6
:10A730005B082343380019003CBC90469946A2466A
:10A74000AB46F8BD6346134311D0731E002B00D0F7
:10A7500007E186188642804161444042091801257C
:10A760000B0237D502257BE73E0061469146350056
:10A77000C5E75C46002D00D0E1E00B000343F3D0B9
:10A78000731C00D1ACE1214B9F4200D13AE1F3436D
:10A79000382B00DD6FE11F2B00DD8CE120250E0042
:10A7A000ED1AAE40B0460600AA46DE4045463543A7
:10A7B0002E005546D940A8406346451EA8415B1A65
:10A7C0009C463043161AB242924163465242991A4D
:10A7D0003D00B4E607223240002A00D0E4E60B4BED
:10A7E000F6084F073743CA089D4200D090E73B0068
:10A7F000134300D1A6E180231B031A431203120B5B
:10A80000024D89E715000022002785E7FF070000B9
:10A81000FFFF7FFFFFFF0F80002E00D0C7E06B1C03
:10A820005E05760D012E00DCF0E0C84DAB4200D194
:10A83000B9E085180A0085428941624449425118AD
:10A840000722CE076D082E43490832401D00A9E6B5
:10A85000BF49ED1A114007223240A3E632002838E2
:10A860008240002686E6300000F052FA203073E67F
:10A87000634613435A1E9341C61AB0428041404278
:10A88000091A5CE60E00674606431743002D5ED1A9
:10A89000002E00D0F3E0002F00D11EE15C4661469F
:10A8A00091462CE7A94FBE427BD01E00F1E6100076
:10A8B0001F3DE840202B03D04021CB1A9A4016437D
:10A8C000731E9E410722064332400021002583E784
:10A8D000161A6346B2428041591A40420B1A9846F2
:10A8E0005C4632E61F2E00DDABE02027BB1B9A46FC
:10A8F00063465746BB40994613004F46F3401F43FB
:10A900003B005746BA40571EBA4113436246F240D5
:10A91000891898E62027BB1B9A4663465746BB40DA
:10A92000994613004F46F3401F433B005746BA4039
:10A93000571EBA4113436246F240891A9CE7834B83
:10A940009F425FD080252D047342294320E7002ECB
:10A950000CD1002F00D1D0E05C46614691467B4D82
:10A96000CDE67A4FBE421CD01E0065E6002F18D0FF
:10A97000C0084E0706438020C9080003014208D0E2
:10A980006346DC08044204D12100DA46D2085E079F
:10A990001643F300994601245346C900720F114330
:10A9A0001C406A4DABE61D0000220027B4E6002DD6
:10A9B00059D10B00034300D1D6E6731C00D1B2E09D
:10A9C000624B9F421ED0F343382B6FDC1F2B00DD00
:10A9D00097E020250E00ED1AAE40B0460600AA46CC
:10A9E000DE40454635432E005546A840D940451E19
:10A9F000A8418C440643B6189642924151426144A4
:10AA00003D0025E63D006146914678E60B00034394
:10AA1000002D00D055E6002BF5D06346134300D13E
:10AA20006DE6861886428041614440420918002242
:10AA30000B0200D4D0E6464B01351940B2E5B146D1
:10AA40005DE633006746203BDF403B00202E05D00B
:10AA50004027BF1B6646BE40324390464646721EA4
:10AA600096413343EFE5394B9F42CBD080252D04EF
:10AA700073422943A8E70843411E8841A2E6002FFC
:10AA800000D13CE66346861ACF1AB0429B415B4236
:10AA9000FB1A98461B024ED5161A6346B2429241E3
:10AAA000591A5242891A5C4600227BE501430E0086
:10AAB000711E8E419FE71D000E00203DEE40B04606
:10AAC000202B04D04025EB1A994008438146484684
:10AAD0004346411E8841184374E60022002417E6CD
:10AAE000161A6346B2429241591A5242891A3D00DF
:10AAF00025E561469146154D01E6802200241203AA
:10AB000079E61D000E00203DEE40B046202B04D01B
:10AB10004025EB1A9940084381464E464346711E34
:10AB20008E411E4367E7861896429B4161445B4213
:10AB3000C9183D008CE547463743CED00722414631
:10AB4000324049E600273A00E6E5C046FF0700002C
:10AB5000FFFF7FFF70B50C4E0D031C0349005B0027
:10AB60002D0B490D240B5B0DB14208D00649002086
:10AB70008B4203D114432000441EA04170BD054305
:10AB80000120002DFAD1F1E7FF07000030B5144D88
:10AB90000A034B00120B5B0DC90F0024AB4211DD01
:10ABA000104CA34210DC8024640322430E4CE41AB0
:10ABB0001F2C0CDD0D48C31ADA4013005C4200293B
:10ABC00000D11C00200030BD094BCC18FAE7094D1C
:10ABD000E040AC4663449A4013000343EEE7C046AE
:10ABE000FE0300001D0400003304000013040000F5
:10ABF000FFFFFF7FEDFBFFFF70B500282DD0C317CF
:10AC0000C5185D40C40F280000F082F8154B1B1AD0
:10AC10005B055B0D0A2815DD0B38854000222D03EE
:10AC20002D0B002110002D030A0D2D0B12052A43B8
:10AC30000D4D1B052A4013435B00E4075B082343CB
:10AC4000190070BD02002900153291400A000B2145
:10AC5000081AC5402D032D0BE3E70024002300252F
:10AC60000022DEE71E040000FFFF0F804100090EF6
:10AC70004B1C70B5DBB24602750AC40F012B14DD04
:10AC8000E0239B006D07360BCB1800210A0D28002E
:10AC900012051C4D32435B052A405B0813435B00E1
:10ACA000E4075B082343190070BD002914D1002D6F
:10ACB0001ED0280000F02CF80A281CDC0B232A00E8
:10ACC0001B1ADA40030015339D400F4B12031B1A69
:10ACD0005B05160B5B0DD8E7002D06D0320B8026E6
:10ACE00036036D071643094BCFE7084B0026CCE728
:10ACF00000230026C9E703002A000B3B9A400025E9
:10AD0000E3E7C046FFFF0F8089030000FF07000054
:10AD10001C2101231B04984201D3000C10391B0A8B
:10AD2000984201D3000A08391B09984201D300094F
:10AD3000043902A2105C40187047C04604030202A6
:10AD400001010101000000000000000030B51C00FE
:10AD5000094B05001B6885B0D868084B002A01D153
:10AD6000074B1A000292019300912B002200054923
:10AD700000F026F800F0A6FD8000002000DA0000B8
:10AD80004FC800000DDA0000014B18687047C0463C
:10AD900080000020084B10B50400002B02D00021D9
:10ADA00000E000BF054B1868836A002B00D098476D
:10ADB000200001F05DFBC046000000003CDA00000E
:10ADC0000EB403B5010003AB044804CB0068019343
:10ADD00000F076F802B008BC03B0184780000020ED
:10ADE00070B500260C4D0D4C641BA410A64209D171
:10ADF000002601F03FFB0A4D0A4C641BA410A6423A
:10AE000005D170BDB300EB5898470136EEE7B300AB
:10AE1000EB5898470136F2E750020020500200201C
:10AE20005002002060020020002310B59A4200D199
:10AE300010BDCC5CC4540133F8E710B5884202D988
:10AE40008B18984203D3002307E08B5C8354013AAC
:10AE5000FBD210BDCC5CC45401339A42FAD1F8E75E
:10AE600003001218934200D1704719700133F9E7BB
:10AE7000936810B5013B9360002B04DA9469A342F8
:10AE800007DB0A2905D01368581C106019700800E8
:10AE900010BD00F04BFC0100F9E7F8B506000F000B
:10AEA0001400D518AC4201D1002007E021783A0007
:10AEB0003000FFF7DDFF0134431CF3D1F8BD000083
:10AEC000F0B59FB002900F0016000593002805D042
:10AED00083690493002B01D100F0F4FD7B4B9F426A
:10AEE0005BD1029B5F68BB891B0762D53B69002B66
:10AEF0005FD0002306AC6361203363761033A37602
:10AF000035002B78002B01D0252B5CD1AB1B049393
:10AF10000CD0320039000298FFF7BFFF431C00D16C
:10AF2000C4E06269049B9446634463612B78002B00
:10AF300000D1BBE0012200235242626002A95432D8
:10AF400052186E1C2360E360A3601370A365317810
:10AF500005225F4800F0D4FE751C002835D1226818
:10AF6000D30604D5532302A95B18202119701307B7
:10AF700004D5532302A95B182B21197033782A2B8F
:10AF80002CD0350000210A20E3682A786E1C303A64
:10AF9000092A64D900292ED026E04E4B9F4202D1C7
:10AFA000029B9F689FE74C4B9F429CD1029BDF68AE
:10AFB00099E73900029800F00FFC002899D0012091
:10AFC00040421FB0F0BD01359BE7414B2268C01ADB
:10AFD00001238340134323602E00B8E7059B191D0E
:10AFE0001B680591002B01DB099304E05B42E360E1
:10AFF0000223134323602B782E2B0AD16B782A2B44
:10B0000035D1059B02351A1D1B680592002B2BDBE1
:10B010000793324E29780322300000F071FE002899
:10B0200006D04023801B83402268013513432360F0
:10B03000297806222A486E1C217600F061FE00283D
:10B040003AD0284B002B25D10722059B0733934389
:10B05000083305936369039A9B18636150E7434380
:10B0600001219B18350090E701235B42D0E70023C4
:10B070000A201A000135636029786E1C30390929CD
:10B0800003D9002BC5D00792C3E7424301235218CE
:10B090003500F1E705AB00933A00134B210002980D
:10B0A00000E000BF0390039B0133D3D1BB895B0653
:10B0B00000D584E70B9884E705AB00933A000A4B70
:10B0C0002100029800F080F8ECE7C04694DA000016
:10B0D00040DA0000B4DA000074DA000046DA00005A
:10B0E0004ADA0000000000009BAE0000F7B5150032
:10B0F00001938A680B6900900C00934200DA1300F8
:10B1000022002B6043321278002A01D001332B60D9
:10B1100023689B0602D52B6802332B600627236821
:10B120001F4027D0230043331B785A1E93412268C7
:10B13000920630D42200019943320098089EB0470D
:10B14000431C25D0062320682A68E16803400025B7
:10B15000042B03D18D1AEB43DB171D40A368226932
:10B16000934201DD9B1AED180027BD4220D100203B
:10B1700010E00137E3682A689B1ABB42D2DD220047
:10B180000123193201990098089EB047431CF0D161
:10B1900001204042FEBD3020E118433108702100FB
:10B1A0005A1C45310978A218433202331170C1E7A5
:10B1B000220001231A3201990098089EB047431CCF
:10B1C000E6D00137D1E70000F0B589B004920A005B
:10B1D00043320593039002920A7E0C000E9B6E2A66
:10B1E00000D186E01FD8632A33D008D8002A00D1C6
:10B1F0008CE0582A4DD0250042352A7030E0642A70
:10B2000001D0692AF7D1196825680A1D280629D5B1
:10B2100008681A60002803DA2D23029A404213704E
:10B220006B4E0A274FE0732A74D008D86F2A1FD0BC
:10B23000702AE0D1202209680A43226003E0752ABF
:10B2400016D0782AD7D12200782145321170614E6C
:10B2500022E025001A684235111D196013682B7011
:10B26000012365E008681A606906D3D500B2D1E70A
:10B2700019682568081D186008682E0605D5544E03
:10B2800008276F2A1BD00A2719E06D06F7D580B270
:10B29000F5E745314E4E0A7018682268011D0068B6
:10B2A0001960150621D5D30702D520231A43226041
:10B2B0001027002803D1202322689A43226023000C
:10B2C000002243331A706368A360002B58DB04220A
:10B2D000216891432160002854D1029D002B5AD04F
:10B2E0002500337842352B7055E05506DBD580B20A
:10B2F000D9E71A680D68101D4969186013682E0691
:10B3000001D5196002E06D06FBD519800023029D6E
:10B3100023614FE01A68111D1960156800216268E9
:10B32000280000F0EDFC002801D0401B606063683D
:10B3300023610023029A13703CE023692A000499D8
:10B340000398059DA847431C3ED023689B0715D44E
:10B35000079BE068984239DA180037E022000123A1
:10B36000193204990398059EB047431C2CD001352F
:10B37000E368079A9B1AAB42F0DCE9E70025F7E7A0
:10B380000028ADD0029D3900FDF722FC735C013D21
:10B390002B700028F7D1082F09D12368DB0706D5C9
:10B3A00063682269934202DC3023013D2B70029BCB
:10B3B0005B1B2361059B07AA00932100049B039854
:10B3C000FFF794FE431CB8D10120404209B0F0BD04
:10B3D00051DA000062DA00000D4B70B51C68050000
:10B3E000A36B002B0FD1182000F06EFC094BA0635B
:10B3F0000360094B01224360084B83600B23838168
:10B400000023026143610022A36B1D615A6170BD7C
:10B41000800000200E33CDAB34126DE6ECDE05006B
:10B42000124B10B51C68A36B002B0FD1182000F035
:10B430004BFC0F4BA06303600E4B012243600E4B8D
:10B4400083600B238381002302614361A46B0B4A59
:10B45000206961690A4BFDF7F7FC0122002380187F
:10B460005941206161614800400810BD8000002002
:10B470000E33CDAB34126DE6ECDE05002D7F954C1E
:10B480002DF451580CB430B5164B9DB00C1E1D68F0
:10B4900008DA8B2301202B6040421DB030BC08BC71
:10B4A00002B01847822302A99B008B8100230290DF
:10B4B00008619C4200D0631E8B604B6101235B429C
:10B4C000CB81209A21AB2800019300F055FD431C4D
:10B4D00001DA8B232B60002CDFD00023029A13703B
:10B4E000DBE7C046800000200EB400B50B499CB0DD
:10B4F0001DAB02900690079104910948094904CBBD
:10B500000591006802A9019300F036FD0023029A1C
:10B5100013701CB008BC03B01847C046FFFFFF7F84
:10B52000800000200802FFFF020010B51378541CB1
:10B53000002B05D1CC5CD4540133002CFAD110BDC2
:10B540002200F3E7C9B20378002B04D08B4200D16C
:10B5500070470130F7E74B42594149420840F7E74D
:10B5600002780B78002A03D0013001319A42F7D0DB
:10B57000D01A70470023C25C0133002AFBD1581E49
:10B580007047002330B59A420AD0013AC45CCD5CC2
:10B59000AC4204D1934202D00133002CF6D1631B9C
:10B5A000180030BD30B50500002A00D130BD0C7840
:10B5B000013A6B1C2C700131002C05D19A189A426B
:10B5C000F4D01C700133FAE71D00EDE710B50378E5
:10B5D000002B0FD10B785A4253415B42184010BDEB
:10B5E0000023CA5C002AFAD0C45C944201D1013322
:10B5F000F7E701300378002BF2D11800EFE70000E5
:10B60000F0B51F000E0087B00590019102920C98D2
:10B61000347800F0EAFA082200194378751C1340C8
:10B6200036D12D2C36D1B51C74780126002F62D06E
:10B63000102F09D1302C07D120222B789343582B7F
:10B6400054D110276C7802352D4B3900F3181800AF
:10B650000393FDF7BDFA0491012100234942020042
:10B660008C4618002100303909291AD80C00A7424D
:10B6700023DD591C09D06346824206D302D10499C6
:10B68000A14202DB0123784320182C780135E9E739
:10B690002E00BCE72B2C01D01E00C7E7B51C747828
:10B6A000FAE721004139192901D8373CDFE72100A9
:10B6B0006139192901D8573CD9E75A1C08D1059A94
:10B6C00023331360029B0398002B09D107B0F0BD10
:10B6D000002E00D04042029A002AF7D0002B01D061
:10B6E0006B1E0193029B019A1A60EFE73024002F32
:10B6F000AAD10827A8E7302C9ED00A27A4E7C04685
:10B70000FFFFFF7F37B51300064A05001068046A83
:10B71000002C00D1044C0A0000942900FFF770FFB0
:10B720003EBDC04680000020E4000020F8B50500C2
:10B730000E001400002804D08369002B01D100F012
:10B74000C1F9224B9C422DD16C68A369A360A389E7
:10B750001B0731D52369002B2ED023682269F7B24D
:10B76000981A6369F6B2834205DC2100280000F0D4
:10B770003BF9002826D1A3680130013BA360236870
:10B780005A1C22601F706369834204D0A389DB07BF
:10B790001AD50A2E18D12100280000F025F900281A
:10B7A00012D00FE00A4B9C4201D1AC68CDE7094BA7
:10B7B0009C42CAD1EC68C8E72100280000F00CF8D0
:10B7C0000028CAD0012676423000F8BD94DA000085
:10B7D000B4DA000074DA0000364B70B51D6806005C
:10B7E0000C00002D05D0AB69002B02D1280000F021
:10B7F00069F9314B9C420FD16C680C23E25E93B225
:10B8000019072DD4D90611D4092301203360373309
:10B810001343A381404270BD284B9C4201D1AC68C8
:10B82000EBE7274B9C42E8D1EC68E6E75B0713D5D2
:10B83000616B002908D023004433994202D03000C4
:10B8400000F06AFA002363632422A3899343A3814F
:10B8500000236360236923600823A2891343A38123
:10B860002369002B0BD1A0218022A389890092009B
:10B870000B40934203D02100300000F0E1F9012396
:10B88000A289134011D00023A36063695B42A361C6
:10B89000002023698342BED10C23E25E1306BAD591
:10B8A00040231343A3810138B5E7920700D46369AD
:10B8B000A360EDE78000002094DA0000B4DA000015
:10B8C00074DA000010B5062000F090FC012000F0B2
:10B8D000CFFD0000F7B58A8905000C00130760D47E
:10B8E0004B68002B04DC0B6C002B01DC0020FEBD40
:10B8F000E76A002FFAD000232E682B6080235B01BB
:10B90000216A1A4034D0606DA3895B0706D563684D
:10B91000C01A636B002B01D0236CC01A0200216A8D
:10B9200000232800E76AB847A189431C06D12B6889
:10B930001D2B30D82B4ADA40D3072CD50023636067
:10B9400023692360CB0405D5431C02D12B68002B4F
:10B9500000D16065616B2E600029C7D0230044339D
:10B96000994202D0280000F0D7F900206063BEE7BA
:10B9700001232800B847431CC6D12B68002BC3D035
:10B980001D2B01D0162B01D12E60AFE74023A289D9
:10B990001343A381ABE740230B430120A381404223
:10B9A000A5E70F69002FA1D00B680F60DB1B019387
:10B9B0000023920700D14B69A360019B002B00DCA0
:10B9C00094E7019B3A00216A2800A66AB047002844
:10B9D00003DC4023A2891343DFE7019B3F181B1AB6
:10B9E0000193EAE7010040200B6970B505000C00E7
:10B9F000002B01D1002070BD002804D08369002BEA
:10BA000001D100F05FF80B4B9C4209D16C680C220D
:10BA1000A35E002BEED021002800FFF75BFFEAE7D2
:10BA2000054B9C4201D1AC68F1E7044B9C42EED13E
:10BA3000EC68ECE794DA0000B4DA000074DA000095
:10BA4000002310B504000360436083608181436676
:10BA5000C281036143618361190008225C30FFF7F2
:10BA6000FFF9054B24626362044BA362044BE3625B
:10BA7000044B236310BDC0462DC2000055C2000018
:10BA80008DC20000B9C2000010B5024900F08CF868
:10BA900010BDC046E9B9000070B568254A1E55437F
:10BAA0000E002900743100F081F9041E08D0002135
:10BAB0002A00016046600C30A0606832FFF7D0F9C0
:10BAC000200070BD836913B50400002B28D1836466
:10BAD000C3640365134B144A1B6882620193984246
:10BAE00001D101238361200000F020F86060200074
:10BAF00000F01CF8A060200000F018F80022E060C0
:10BB000004216068FFF79CFF01220921A068FFF76C
:10BB100097FF02221221E068FFF792FF0123A36141
:10BB200013BDC0463CDA000089BA0000F8B51C4BD2
:10BB300007001E68B369002B02D13000FFF7C2FF77
:10BB40004836B4687368013B04D53368002B07D0CE
:10BB50003668F6E70C22A55E002D0DD06834F2E7BA
:10BB600004213800FFF798FF30600028F0D10C2343
:10BB700004003B602000F8BD20000A4B656625608C
:10BB80006560A560E36025616561A5610822290003
:10BB90005C30FFF765F96563A563A564E564E9E7D3
:10BBA0003CDA00000100FFFFF7B5040007000026A3
:10BBB00001914834002C01D13000FEBD6368A568B6
:10BBC0000093009B013B009301D52468F2E7AB8909
:10BBD000012B08D90E22AB5E013304D029003800B6
:10BBE000019B984706436835EBE7EC3000687047E7
:10BBF00070B50E001D000E23C95E96B0140000291A
:10BC000007DA00232B60B3891B0611D48023DB00E5
:10BC10000FE06A4600F088FB0028F2DBF022019B6F
:10BC200012021340054A9B185A4253412B60EDE71C
:10BC300040230020236016B070BDC04600E0FFFF27
:10BC4000F7B502268B8905000C00334206D023008D
:10BC500047332360236101236361F7BD01AB6A466B
:10BC6000FFF7C6FF00990700280000F09FF80028A2
:10BC700008D10C22A35E9A05EFD4032293431E43FE
:10BC8000A681E4E70F4BAB628023A28920601343B7
:10BC9000A381009B20616361019B002B0DD00E23CB
:10BCA000E15E280000F052FB002806D00322A389A1
:10BCB00093431A0001231343A381A0893843A08131
:10BCC000CBE7C04689BA000010B5034B01001868E5
:10BCD00000F06CF810BDC0468000002082B0002942
:10BCE00000D101A9101E06D0002B06D013780B60DE
:10BCF0001078431E984102B0704702204042FAE794
:10BD0000C9B28218904201D10020704703788B425B
:10BD1000FBD00130F6E7000070B50500002910D017
:10BD20000C1F2368002B00DAE418280000F034FB15
:10BD30001D4A1368002B05D163601460280000F0D1
:10BD40002CFB70BDA34209D9216860188342F3D14E
:10BD500018685B6841182160EEE713005A68002AF2
:10BD600001D0A242F9D919685818A0420BD1206815
:10BD70000918581819608242E0D1106852684118B9
:10BD800019605A60DAE7A04202D90C232B60D5E78C
:10BD900021686018824203D11068526841182160FE
:10BDA00062605C60CAE7C0461C1C0020032370B5BB
:10BDB000CD1C9D43083506000C2D1ED20C25A94232
:10BDC0001DD8300000F0E8FA254A14682100002947
:10BDD00019D1244C2368002B03D1300000F0CAF99C
:10BDE00020602900300000F0C5F9431C2BD10C2342
:10BDF0003000336000F0D1FA03E0002DDFDA0C23CD
:10BE00003360002070BD0B685B1B19D40B2B03D96A
:10BE10000B60CC18256003E04B688C420DD1136099
:10BE2000300000F0BAFA200007220B30231D9043A7
:10BE3000C31AE7D05A42E250E4E763600C00EFE730
:10BE40000C004968C3E70323C41C9C43A042E1D013
:10BE5000211A300000F08EF9431CDBD1C7E7C04641
:10BE60001C1C0020201C0020F8B507000D00160047
:10BE7000002905D11100FFF799FF04002000F8BD4B
:10BE8000002A03D1FFF748FF3400F7E700F086FAF5
:10BE90002C00B042F2D231003800FFF787FF041EB9
:10BEA000ECD029003200FEF7BFFF29003800FFF771
:10BEB00033FFE3E7F0B58E6885B007000C0003920E
:10BEC00001939E423CD890238A89DB001A4234D0E9
:10BED0000325096923685B1A0293636902985D432D
:10BEE000EB0F5D19019B6D1001331B18AB4200D99C
:10BEF0001D00530532D529003800FFF757FF061EF5
:10BF000009D10C233B6040230120A2894042134306
:10BF1000A38105B0F0BD029A2169FEF785FFA389D0
:10BF2000144A1A4080231343A381029B2661F6180A
:10BF300026606561019EED1AA560019B9E4200D9B5
:10BF4000019E320003992068FEF777FFA368002066
:10BF50009B1BA36023689E192660DAE72A0038003D
:10BF6000FFF782FF061EE0D121693800FFF7D4FEFB
:10BF7000C7E7C0467FFBFFFFF0B59FB00290059377
:10BF80008B890F0016001B0611D50B69002B0ED1F3
:10BF90004021FFF70BFF38603861002805D10C23E2
:10BFA000029A013813601FB0F0BD40237B6100236B
:10BFB00006AC6361203363761033A37635002B78AB
:10BFC000002B01D0252B46D1AB1B04930CD03200A3
:10BFD00039000298FFF76EFF431C00D1AEE06269A2
:10BFE000049B9446634463612B78002B00D1A5E049
:10BFF000012200235242626002A9543252186E1C80
:10C000002360E360A3601370A36531780522544870
:10C01000FFF776FE751C00281FD12268D30604D5D1
:10C02000532302A95B1820211970130704D5532349
:10C0300002A95B182B21197033782A2B16D03500F2
:10C0400000210A20E3682A786E1C303A092A4ED96A
:10C05000002918D010E00135B1E7414B2268C01A21
:10C0600001238340134323602E00CEE7059B191D57
:10C070001B680591002B01DB099304E05B42E36040
:10C080000223134323602B782E2B0AD16B782A2BA3
:10C0900035D1059B02351A1D1B680592002B2BDB41
:10C0A0000793304E297803223000FFF729FE00283D
:10C0B00006D04023801B8340226801351343236050
:10C0C0002978062228486E1C2176FFF719FE0028E1
:10C0D0003CD0264B002B25D10722059B07339343E9
:10C0E000083305936369039A9B18636166E74343CA
:10C0F00001219B183500A6E701235B42D0E700230E
:10C100000A201A000135636029786E1C303909292C
:10C1100003D9002BC5D00792C3E74243012352182D
:10C120003500F1E705AB00933A00114B210002986E
:10C1300000E000BF0390039B0133D3D1BB890B9870
:10C140005B0600D42FE7012040422CE705AB0093AB
:10C150003A00074B21000298FFF736F8EAE7C0469D
:10C1600040DA000046DA00004ADA00000000000071
:10C17000B5BE0000002370B5064C05000800236022
:10C1800000F060F9431C03D12368002B00D02B6022
:10C1900070BDC046982F002070B504000D001F2907
:10C1A00004D9162303600120404270BD436C002B6C
:10C1B00004D08A009B181A68002A08D1200000F0D9
:10C1C00031F82A000100200000F01AF8EDE7002005
:10C1D000012AEAD0511C03D1162301302360E4E781
:10C1E000002428001C6090472000DEE710B5034BB8
:10C1F00001001868FFF7D0FF10BDC0468000002086
:10C20000002370B5064C050008001100236000F003
:10C2100001F9431C03D12368002B00D02B6070BDB3
:10C22000982F002010B500F0E5F810BD70B50C0097
:10C230000E25495F00F0BAF8002803DB636D1B1878
:10C24000636570BDA389024A1340A381F9E7C04624
:10C25000FFEFFFFFF8B51F008B8905000C001600EB
:10C26000DB0505D50E23C95E0022022300F080F80D
:10C27000A389054A28001340A38132000E23E15E02
:10C280003B0000F02BF8F8BDFFEFFFFF70B50C008E
:10C290000E25495F00F06CF8A389421C03D1054AC2
:10C2A0001340A38170BD802252011343A3816065B6
:10C2B000F8E7C046FFEFFFFF10B50E23C95E00F0A0
:10C2C00021F810BD0B1E04D0FF2A04D98A23036075
:10C2D0008B3B180070470A700123FAE770B5050020
:10C2E000080011000022064C22601A0000F0B8F885
:10C2F000431C03D12368002B00D02B6070BDC046C7
:10C30000982F0020002370B5064C0500080023601C
:10C3100000F060F8431C03D12368002B00D02B6091
:10C3200070BDC046982F0020002370B5064C050054
:10C3300008001100236000F055F8431C03D1236866
:10C34000002B00D02B6070BD982F0020002370B50B
:10C35000064C05000800236000F054F8431C03D18C
:10C360002368002B00D02B6070BDC046982F0020A2
:10C3700070B50500080011000022064C22601A006A
:10C3800000F050F8431C03D12368002B00D02B6031
:10C3900070BDC046982F0020704770470B1F1B6868
:10C3A000181F002B01DA0B58C018704770B5050034
:10C3B000080011000022064C22601A0000F03AF832
:10C3C000431C03D12368002B00D02B6070BDC046F6
:10C3D000982F002058220120014B40421A607047DC
:10C3E000982F002058220120014B40421A607047CC
:10C3F000982F002058220120014B40421A607047BC
:10C40000982F00205822024B00201A607047C04627
:10C41000982F002058220120014B40421A6070479B
:10C42000982F002058220120014B40421A6070478B
:10C43000982F002058220120014B40421A6070477B
:10C44000982F0020044A1368002B00D1034B1818C2
:10C45000106018007047C046241C0020A02F002048
:10C4600058220120014B40421A607047982F00204B
:10C47000FEE7C046F8B5C046F8BC08BC9E4670470B
:10C48000F8B5C046F8BC08BC9E467047646174614C
:10C490000000000008C50000EB01000011C500000D
:10C4A0001704000019C500002907000020C500007E
:10C4B0003908000025C50000DF02000030C500007B
:10C4C0008304000035C50000B109000041C500002B
:10C4D0001B0200004BC500003106000059C50000DA
:10C4E0009F05000072616E646F6D00616C6C006C82
:10C4F0006173740066616C73650074727565002504
:10C500002E3135732E2E2E006D616B654C69737460
:10C51000006164644C6173740064656C65746500EB
:10C520006A6F696E00636F707946726F6D546F0049
:10C5300066696E64006A6F696E537472696E6773C0
:10C5400000756E69636F6465417400756E69636F31
:10C550006465537472696E6700667265654D656DDA
:10C560006F727900E80F0000F80F00001210000051
:10C5700090100000C8100000FE10000036110000EE
:10C580005C11000098110000DA1100003012000068
:10C5900074120000E0120000281300004E13000087
:10C5A00086130000CC130000F213000020140000DA
:10C5B000521400008A1400000E150000D615000069
:10C5C0004C160000B81600000C1700002C170000D5
:10C5D0004E1700000018000046180000BE180000AA
:10C5E000E80F0000E80F0000EC18000054190000EC
:10C5F000D81900001E1A0000661A0000D81A0000A0
:10C600004A1B0000921B0000D81B00000E1C0000FB
:10C61000541C00009A1C0000E21C0000361D0000A3
:10C62000941D0000D21D00003C1E0000721E000080
:10C63000BA1E0000021F00004A1F0000841F0000F5
:10C64000CC1F000014200000E80F0000E80F0000DD
:10C65000E80F00007C200000E80F0000B22000007E
:10C66000DE2000001421000040210000E80F00003F
:10C67000E80F0000E80F0000E80F0000762100003E
:10C68000C2210000E80F0000E80F000008220000AF
:10C69000582200007E220000E80F0000E80F000092
:10C6A000E80F0000AC220000DC2200000C23000098
:10C6B000422300006C230000A2230000CC230000D2
:10C6C000F42300001C2400004C2400007C24000003
:10C6D000A6240000D0240000002500002A25000028
:10C6E000E80F0000E80F0000E80F0000E80F00006E
:10C6F000E80F00005A250000A0250000CC2500000E
:10C70000F8250000242600005A260000902600008C
:10C71000C6260000FC260000282700005427000041
:10C720008A270000E80F0000E80F0000E80F000073
:10C73000E80F0000E80F0000E80F0000E80F00001D
:10C74000E80F0000E80F0000E80F0000E80F00000D
:10C75000E80F0000E80F0000E80F0000B627000017
:10C76000EC270000282564206974656D206C6973CE
:10C77000742900286F626A65637420747970653A61
:10C780002025642900537461636B20756E646572A3
:10C79000666C6F77000000000700000003000000D7
:10C7A000E2C700000D290000EAC70000BD29000013
:10C7B000F3C70000552A0000FCC700001129000043
:10C7C0000000000001000000020000000300000063
:10C7D000040000000A0000006D6963726F3A62692C
:10C7E0007400686173546F6E6500706C6179546F8A
:10C7F0006E6500686173536572766F00736574537C
:10C800006572766F00474320746F6F6B202564203C
:10C8100075736563733B20667265652025642077B8
:10C820006F726473003C496E74656765723E003CCC
:10C830004F626A6563743E003C4C6973743E000D40
:10C840000A564D2050616E69633A2025730D0A0027
:10C850006D697363000000008DC80000D9360000C8
:10C8600096C80000713600009AC80000C535000067
:10C87000A2C800006B350000ACC800000135000004
:10C88000B8C80000033400006E756C6C00686578F1
:10C89000546F496E740073696E006A736F6E4765FA
:10C8A00074006A736F6E436F756E74006A736F6E97
:10C8B00056616C75654174006A736F6E4B657941A2
:10C8C0007400000038C900004537000040C900006E
:10C8D000493700004AC900006737000053C900000B
:10C8E000713700005EC900007B3700006AC9000094
:10C8F000853700007AC900008F3700008AC9000020
:10C90000993700009FC90000A3370000B4C9000098
:10C91000AD370000C0C90000B7370000D0C9000023
:10C92000C1370000DCC9000053370000E9C900002E
:10C930005D3700006E657400686173576946690071
:10C940007374617274576946690073746F705769C4
:10C9500046690077696669537461747573006D790F
:10C9600049504164647265737300737461727448F2
:10C970007474705365727665720073746F70744866
:10C980007474705365727665720068747470536560
:10C99000727665724765745265717565737400725D
:10C9A0006573706F6E64546F4874747052657175FE
:10C9B0006573740068747470436F6E6E65637400A1
:10C9C000687474704973436F6E6E65637465640058
:10C9D00068747470526571756573740068747470EE
:10C9E000526573706F6E73650068747470436C6F1A
:10C9F0007365001A1B1C03040607090A171819009F
:10CA00000000000008080800080A4A4000000A5F09
:10CA1000EA5FEA0ED92ED36E19324489330C924C58
:10CA2000924D080800000004880808040804848463
:10CA300088000A448A4000048EC4800000000488F4
:10CA400000000EC000000000080001224488100C05
:10CA50009252524C048C84848E1C824C901E1EC2B6
:10CA600044924C06CA525FE21FF01EC13E02448E41
:10CA7000D12E1FE24488100ED12ED12E0ED12EC4FD
:10CA800088000800080000048004880244880482AA
:10CA9000000EC00EC008048244880ED126C0040EC9
:10CAA000D135B36C0C925ED2521C925C925C0ED06B
:10CAB00010100E1C9252525C1ED01C901E1ED01CD8
:10CAC00090100ED013712E12525ED2521C8808089C
:10CAD0001C1FE242524C1254981492101010101E57
:10CAE000113B75B131113935B3710C9252524C1C56
:10CAF000925C90100C92524C861C925C92510ED01B
:10CB00000C825C1FE4848484125252524C113131E5
:10CB10002A44113135BB7112524C9252112A44846D
:10CB2000841EC488101E0EC808080E100804824116
:10CB30000EC242424E048A400000000000001F085E
:10CB400004800000000ED2524F10101C925C000EA8
:10CB5000D0100E02424ED24E0C925C900E06C81CB3
:10CB600088080ED24EC24C10101C925208000808C1
:10CB700008024002424C1014981492080808080653
:10CB8000001B75B131001C925252000C92524C00A5
:10CB90001C925C90000ED24EC2000ED01010000607
:10CBA000C8049808080EC807001252524F001131ED
:10CBB0002A4400113135BB00124C8C9200112A44DA
:10CBC00098001EC4881E06C48C84860808080808BD
:10CBD00018080C881800000C83600000000000009A
:10CBE000010000000200000003000000040000003B
:10CBF000050000000600000007000000080000001B
:10CC0000090000000A0000000B0000000C000000FA
:10CC10000D0000000E0000000F00000010000000DA
:10CC200012000000140000001600000018000000B0
:10CC30001A0000001C0000001E0000002000000080
:10CC40002300000026000000290000002C00000046
:10CC50002F00000032000000360000003A00000003
:10CC60003E00000042000000460000004B000000B3
:10CC700050000000550000005A0000006100000054
:10CC8000680000006F000000760000007D000000DA
:10CC9000840000008B00000092000000990000005A
:10CCA000A0000000A7000000AE000000B5000000DA
:10CCB000BC000000C3000000CA000000D10000005A
:10CCC000D8000000DF000000E6000000ED000000DA
:10CCD000F4000000FB000000FF0000002CCD00006D
:10CCE000E537000037CD0000293D000041CD0000B0
:10CCF000A13900004ECD0000993B000055CD000049
:10CD0000E93B00005ECD0000393C00006ACD000028
:10CD1000353B00007BCD0000113A000088CD0000BB
:10CD2000CD3A0000646973706C6179006C69676862
:10CD3000744C6576656C006D62446973706C6179E2
:10CD4000006D62446973706C61794F6666006D6254
:10CD5000506C6F74006D62556E706C6F74006D6214
:10CD6000447261775368617065006D6253686170E9
:10CD700065466F724C6574746572006E656F5069BC
:10CD800078656C53656E64006E656F506978656C8C
:10CD900053657450696E004E6F7420656E6F7567D1
:10CDA0006820726F6F6D206576656E2061667465B0
:10CDB0007220636F6D70616374696F6E00436F6D95
:10CDC00070616374656420466C61736820636F648E
:10CDD000652073746F72650A2564206279746573C7
:10CDE000207573656420282564252529206F662019
:10CDF000256400426164207265636F726420666F0F
:10CE0000756E6420647572696E6720696E697469F5
:10CE1000616C697A6174696F6E00256420256420F5
:10CE200025642028256420776F72647329002564A7
:10CE3000207265636F7264732C20256420776F7293
:10CE400064732C206D617849442025642C20636F25
:10CE50006D70616374696F6E206379636C657320B4
:10CE6000256400526573746F7265642025642073B5
:10CE700063726970747300537461727465640072D4
:10CE80006164696F0000000026CF0000F1460000D9
:10CE900033CF00008D49000043CF00000D49000052
:10CEA00051CF0000214B00005CCF0000194700006B
:10CEB0006CCF0000A147000080CF00008947000030
:10CEC0008FCF0000034D00009BCF0000814C00007D
:10CED000A4CF0000254C0000AFCF00006D4B000038
:10CEE000BACF0000A94B0000C3CF0000DD4B00000B
:10CEF000CCCF000029470000DBCF0000094700002D
:10CF0000E4CF0000394700006E756D626572006EF7
:10CF10006F6E65006F74686572007061697200738E
:10CF20007472696E670064697361626C65526164F2
:10CF3000696F006D657373616765526563656976D6
:10CF40006564007061636B657452656365697665DD
:10CF5000007061636B657453656E64007265636530
:10CF600069766564496E74656765720072656365AC
:10CF7000697665644D6573736167655479706500A2
:10CF80007265636569766564537472696E67007370
:10CF9000656E64496E74656765720073656E645092
:10CFA0006169720073656E64537472696E670073B1
:10CFB00065744368616E6E656C0073657447726F6B
:10CFC000757000736574506F776572007369676E72
:10CFD000616C537472656E6774680064657669632A
:10CFE000654944006C6173744D657373616765498D
:10CFF0004400000000000000963007772C610EEE20
:10D00000BA51099919C46D078FF46A7035A563E99F
:10D01000A395649E3288DB0EA4B8DC791EE9D5E0C6
:10D0200088D9D2972B4CB609BD7CB17E072DB8E7C5
:10D03000911DBF906410B71DF220B06A4871B9F31A
:10D04000DE41BE847DD4DA1AEBE4DD6D51B5D4F453
:10D05000C785D38356986C13C0A86B647AF962FDB8
:10D06000ECC9658A4F5C0114D96C0663633D0FFA05
:10D07000F50D088DC8206E3B5E10694CE44160D50B
:10D08000727167A2D1E4033C47D4044BFD850DD2F5
:10D090006BB50AA5FAA8B5356C98B242D6C9BBDB08
:10D0A00040F9BCACE36CD832755CDF45CF0DD6DC03
:10D0B000593DD1ABAC30D9263A00DE518051D7C8AA
:10D0C0001661D0BFB5F4B42123C4B3569995BACF35
:10D0D0000FA5BDB89EB802280888055FB2D90CC656
:10D0E00024E90BB1877C6F2F114C6858AB1D61C1CF
:10D0F0003D2D66B69041DC760671DB01BC20D298EE
:10D100002A10D5EF8985B1711FB5B606A5E4BF9F7A
:10D1100033D4B8E8A2C9077834F9000F8EA809966D
:10D1200018980EE1BB0D6A7F2D3D6D08976C6491D8
:10D13000015C63E6F4516B6B62616C1CD8306585F1
:10D140004E0062F2ED95066C7BA5011BC1F40882CE
:10D1500057C40FF5C6D9B06550E9B712EAB8BE8B0F
:10D160007C88B9FCDF1DDD62492DDA15F37CD38C98
:10D17000654CD4FB5861B24DCE51B53A7400BCA396
:10D18000E230BBD441A5DF4AD795D83D6DC4D1A4C8
:10D19000FBF4D6D36AE96943FCD96E34468867AD9F
:10D1A000D0B860DA732D0444E51D03335F4C0AAA3E
:10D1B000C97C0DDD3C710550AA41022710100BBE41
:10D1C00086200CC925B56857B3856F2009D466B988
:10D1D0009FE461CE0EF9DE5E98C9D9292298D0B0BD
:10D1E000B4A8D7C7173DB359810DB42E3B5CBDB76A
:10D1F000AD6CBAC02083B8EDB6B3BF9A0CE2B603EB
:10D200009AD2B1743947D5EAAF77D29D1526DB049F
:10D210008316DC73120B63E3843B64943E6A6D0DEA
:10D22000A85A6A7A0BCF0EE49DFF099327AE000A35
:10D23000B19E077D44930FF0D2A3088768F2011EC8
:10D24000FEC206695D5762F7CB67658071366C195F
:10D25000E7066B6E761BD4FEE02BD3895A7ADA1080
:10D26000CC4ADD676FDFB9F9F9EFBE8E43BEB71761
:10D27000D58EB060E8A3D6D67E93D1A1C4C2D838EB
:10D2800052F2DF4FF167BBD16757BCA6DD06B53F51
:10D290004B36B248DA2B0DD84C1B0AAFF64A033690
:10D2A000607A0441C3EF60DF55DF67A8EF8E6E310F
:10D2B00079BE69468CB361CB1A8366BCA0D26F2558
:10D2C00036E2685295770CCC03470BBBB9160222A5
:10D2D0002F260555BE3BBAC5280BBDB2925AB42BBA
:10D2E000046AB35CA7FFD7C231CFD0B58B9ED92CCF
:10D2F0001DAEDE5BB0C2649B26F263EC9CA36A7534
:10D300000A936D02A906099C3F360EEB85670772EA
:10D3100013570005824ABF95147AB8E2AE2BB17B51
:10D32000381BB60C9B8ED2920DBED5E5B7EFDC7CD8
:10D3300021DFDB0BD4D2D38642E2D4F1F8B3DD682F
:10D340006E83DA1FCD16BE815B26B9F6E177B06F2A
:10D350007747B718E65A0888706A0FFFCA3B066617
:10D360005C0B0111FF9E658F69AE62F8D3FF6B61A4
:10D3700045CF6C1678E20AA0EED20DD75483044E46
:10D38000C2B30339612667A7F71660D04D476949D4
:10D39000DB776E3E4A6AD1AEDC5AD6D9660BDF40E7
:10D3A000F03BD83753AEBCA9C59EBBDE7FCFB2479A
:10D3B000E9FFB5301CF2BDBD8AC2BACA3093B3537F
:10D3C000A6A3B4240536D0BA9306D7CD2957DE5488
:10D3D000BF67D9232E7A66B3B84A61C4021B685D61
:10D3E000942B6F2A37BE0BB4A18E0CC31BDF055ADA
:10D3F0008DEF022D416C6C207461736B732073741C
:10D400006F707065640076303737002025732025F3
:10D4100073004D656D6F727920636C656172656430
:10D42000004E6F2066726565207461736B20656EB7
:10D43000747269657300000080D40000E15F000031
:10D440008DD400006D5C000099D4000017600000CE
:10D450009FD4000027600000A5D4000037600000C2
:10D46000ABD40000A15C0000B5D40000496000000E
:10D47000BDD40000E15D000073656E736F727300D0
:10D48000616363656C65726174696F6E0074656D6C
:10D4900070657261747572650074696C745800749B
:10D4A000696C74590074696C745A00746F756368A0
:10D4B0005265616400693263526561640069326378
:10D4C00057726974650000003CD50000D16000000F
:10D4D0004AD50000D560000053D50000E16000008F
:10D4E0005DD50000E560000066D50000E960000041
:10D4F0006BD50000ED60000070D50000F160000009
:10D500007CD50000F560000083D50000F9600000C4
:10D510008CD50000FD60000091D500000161000085
:10D520009CD5000005610000A6D50000D960000070
:10D53000B0D50000DD60000074667400656E616245
:10D540006C65446973706C617900676574576964D0
:10D55000746800676574486569676874007365740A
:10D56000506978656C006C696E6500726563740063
:10D57000726F756E6465645265637400636972638B
:10D580006C6500747269616E676C650074657874AF
:10D5900000746674546F75636865640074667454CF
:10D5A0006F7563685800746674546F7563685900CA
:10D5B000746674546F7563685072657373757265C1
:10D5C0000057656C636F6D6520746F204D696372E1
:10D5D0006F426C6F636B732100705F737069202101
:10D5E0003D204E554C4C002F686F6D652F62726F59
:10D5F0006D61676F73612F2E706C6174666F726DF1
:10D60000696F2F7061636B616765732F6672616DFF
:10D6100065776F726B2D61726475696E6F6E6F7274
:10D620006469636E7266352F6C69627261726965D6
:10D63000732F5350492F5350492E6370700053502D
:10D6400049436C6173733A3A535049436C61737345
:10D65000284E52465F5350495F547970652A2C20FA
:10D6600075696E74385F742C2075696E74385F74D8
:10D670002C2075696E74385F74290000000000006A
:10D6800000000000BD660000796600009F66000093
:10D69000A9660000B36600009D660000030000005C
:10D6A000020000000100000004000000050000006E
:10D6B000110000000C0000000B0000001200000030
:10D6C0000A000000060000001A000000140000001C
:10D6D00017000000160000001500000010000000F8
:10D6E000FFFFFFFFFFFFFFFF000000001E00000024
:10D6F00019000000180000000700000008000000EA
:10D70000090000000D0000000E0000000F000000E6
:10D710001C0000001B0000001D00000013000000A2
:10D7200000000000000000006D6B00009D72000012
:10D73000ED6B0000016C0000F76B0000696B0000EE
:10D740005D6B00000D6C0000896B0000596B0000E0
:10D75000000000000000304300000000000030C363
:10D760007371727400000000FB21F93FFB21094036
:10D770007CD91240FB2119407A6A1F407CD9224093
:10D78000BBFD2540FB2129403A462C407A6A2F40B8
:10D790005C4731407CD932409C6B3440BBFD354006
:10D7A000DB8F3740FB2139401BB43A403A463C40BE
:10D7B0005AD83D407A6A3F404C7E40405C474140E9
:10D7C0006C1042407CD942408CA243409C6B444048
:10D7D000AC344540BBFD4540CBC64640DB8F47409F
:10D7E000EB584840FB21494083F9A200444E6E00AB
:10D7F000FC291500D1572700DD34F50062DBC0009D
:10D800003C999500419043006351FE00BBDEAB00A4
:10D81000B761C5003A6E2400D24D42004906E000CF
:10D8200009EA2E001C92D100EB1DFE0029B11C005C
:10D83000E83EA700F535820044BB2E009CE9840039
:10D84000B4267000417E5F00D691390053833900C1
:10D850009CF439008B5F840028F9BD00F81F3B0061
:10D86000DEFF97000F980500112FEF000A5A8B007A
:10D870006D1F6D00CF7E360009CB2700464FB700E5
:10D880009E663F002DEA5F00BA277500E5EBC700F2
:10D890003D7BF100F739070092528A00FB6BEA00EA
:10D8A0001FB15F00085D8D00300356007BFC460011
:10D8B000F0AB6B0020BCCF0036F49A00E3A91D004A
:10D8C0005E619100081BE60085996500A0145F0069
:10D8D0008D40680080D8FF0027734D000606310098
:10D8E000CA561500C9A873007BE260006B8CC000AB
:10D8F00000000040FB21F93F000000002D44743E71
:10D90000000000809846F83C0000006051CC783B55
:10D9100000000080831BF0390000004020257A3889
:10D92000000000802282E336000000001DF369350C
:10D9300002000000030000000400000006000000D8
:10D94000948F00003E8F00003E8F00006C9000001E
:10D950003A8F00003A8F0000629000006C90000047
:10D960003A8F0000629000003A8F00006C90000037
:10D97000709000007090000070900000789000009F
:10D98000709A0000E2980000269900008A98000032
:10D9900026990000169A0000269900008A98000037
:10D9A000E2980000E2980000169A00008A980000B1
:10D9B000829800008298000082980000249A00005B
:10D9C00098A100009AA000009AA00000B8A300004F
:10D9D00094A0000094A00000A0A30000B8A3000041
:10D9E00094A00000A0A3000094A00000B8A3000031
:10D9F000AEA30000AEA30000AEA30000BCA30000D5
:10DA00002C2066756E6374696F6E3A2000617373C3
:10DA1000657274696F6E2022257322206661696CBD
:10DA200065643A2066696C6520222573222C206C7F
:10DA3000696E65202564257325730A008400002023
:10DA4000232D302B2000686C4C00656667454647E7
:10DA5000003031323334353637383941424344456A
:10DA600046003031323334353637383961626364D9
:10DA700065660000000000000000000000000000DB
:10DA80000000000000000000000000000000000096
:10DA90000000000000000000000000000000000086
:10DAA0000000000000000000000000000000000076
:10DAB0000000000000000000000000000000000066
:10DAC0000000000000000000000000000000000056
:10DAD000000000004300504F534958000020202010
:10DAE000202020202020282828282820202020200E
:10DAF00020202020202020202020202020881010DE
:10DB00001010101010101010101010101004040439
:10DB100004040404040404101010101010104141F7
:10DB200041414141010101010101010101010101E5
:10DB300001010101010101011010101010104242F9
:10DB400042424242020202020202020202020202B5
:10DB50000202020202020202101010102000000055
:10DB600000000000000000000000000000000000B5
:10DB700000000000000000000000000000000000A5
:10DB80000000000000000000000000000000000095
:10DB90000000000000000000000000000000000085
:10DBA0000000000000000000000000000000000075
:10DBB0000000000000000000000000000000000065
:10DBC0000000000000000000000000000000000055
:10DBD0000000000000000000000000000000000045
:04DBE0000000000041
:08DBE4002425FF7F0100000071
:10DBEC00FFFFFFFF4006000001000000E803DC051A
:10DBFC00DC05DC05DC050000FFFFFFFFFFFFFFFF7E
:10DC0C001800000019FCFFFFFFFFFFFFFF000000E2
:10DC1C000200000003000000FFFFFFFF00000000F7
:10DC2C00010000000000020001000000FFFFFFFFE8
:10DC3C0000000000020000000000040002000000D0
:10DC4C00FFFFFFFF000000000300000000000800C1
:10DC5C00030000000A0000000800000001000000A2
:10DC6C00840000200000000094DA0000B4DA000008
:10DC7C0074DA00000000000000000000000000004A
:10DC8C000000000000000000000000000000000088
:10DC9C000000000000000000000000000000000078
:10DCAC000000000000000000000000000000000068
:10DCBC000000000000000000000000000000000058
:10DCCC000000000043000000000000000000000005
:10DCDC000000000000000000000000000000000038
:10DCEC0000000000430000000000000000000000E5
:10DCFC000000000000000000000000000000000018
:10DD0C0000000000430000000000000000000000C4
:10DD1C0000000000000000000000000000000000F7
:10DD2C0000000000430000000000000000000000A4
:10DD3C0000000000000000000000000000000000D7
:10DD4C000000000043000000000000000000000084
:10DD5C0000000000000000000000000000000000B7
:10DD6C000000000043000000000000000000000064
:10DD7C000000000000000000000000000000000097
:10DD8C000000000043000000000000000000000044
:10DD9C000000000000000000000000000000000077
:10DDAC0000000000C5C20000DDBC00000000000047
:10DDBC00DCDA000006C500004FC800004FC80000A8
:10DDCC004FC800004FC800004FC800004FC80000EB
:10DDDC004FC800004FC800004FC80000FFFFFFFFF6
:10DDEC00FFFFFFFFFFFFFFFFFFFF0000010041539C
:10DDFC004349490000000000000000000000000042
:10DE0C000000000000000000000000000000415372
:10DE1C004349490000000000000000000000000021
:10DE2C0000000000000000000000000000000000E6
:10DE3C00E90000004966000091690000B96E00001D
:04DE4C00C100000011
:0400000300006A2D62
:00000001FF
